:020000040000FA
:1000000000040020E508000079050000C508000094
:10001000830500008D05000097050000000000002A
:1000200000000000000000000000000009090000BE
:10003000A105000000000000AB050000B5050000B0
:10004000BF050000C9050000D3050000DD05000064
:10005000E7050000F1050000FB05000005060000B3
:100060000F06000019060000230600002D06000000
:1000700037060000410600004B0600005506000050
:100080005F06000069060000730600007D060000A0
:1000900087060000910600009B060000A5060000F0
:1000A000AF060000B9060000C3060000CD06000040
:1000B000D7060000E1060000EB060000F506000090
:1000C000FF06000009070000130700001D070000DD
:1000D00027070000310700003B070000450700002C
:1000E0004F07000059070000630700006D0700007C
:1000F00077070000810700008B07000095070000CC
:100100009F0700001FB500F003F88DE80F001FBD2A
:1001100000F0DEBB1FB56FF00100009040100390AF
:10012000029001904FF010208069000B420900F00E
:100130001F045DF822300120A04083434DF8223097
:10014000684600F044F91FBDF0B54FF6FF734FF459
:10015000B4751A466E1E11E0A94201D3344600E080
:100160000C46091B30F8027B641E3B441A44F9D14B
:100170009CB204EB134394B204EB12420029EBD17E
:1001800098B200EB134002EB124140EA0140F0BD8F
:10019000DD4992B00446D1E90001CDE91001FF220A
:1001A0004021684600F03AFB94E80F008DE80F000C
:1001B000684610A902E004C841F8042D8842FAD12B
:1001C00010216846FFF7C0FF1090AA208DF8440068
:1001D000FFF7A0FF00F0F2F84FF01024A069102202
:1001E0006946803000F001F9A069082210A900F0EA
:1001F000FCF800F0D7F84FF080510A6949690068AF
:100200004A43824201D8102070470020704710B541
:10021000D0E900214FF0805002EB8103026944696C
:100220006243934209D84FF01022536903EB8103D4
:100230000169406941438B4201D9092010BD5069D1
:10024000401C01D0002010BD0F2010BD70B501680A
:100250000446AE4D4FF01020062951D2DFE801F0E0
:10026000320318283B1DD4E90265646829463046EC
:1002700000F0CDF82A462146304600F0B6F8AA0034
:100280002146304600F09EFA002800D0032070BDC1
:1002900000F050FB4FF4805007E0201DFFF7ABFF4C
:1002A0000028F4D100F046FB60682860002070BD93
:1002B000241D94E80700920000F084FA0028F6D08C
:1002C0000E2070BD8069401C12D0201DFFF79FFFDB
:1002D0000028F6D109E08069401C09D0201DFFF7F5
:1002E0008AFF0028EDD1606820B12046FFF750FF5B
:1002F000042070BDFFF70EFF00F060F800F052F828
:10030000072070BD10B50C46182802D001200860E7
:1003100010BD2068FFF79AFF206010BD4FF0102439
:10032000A069401C05D0A569A66980353079AA2846
:1003300008D06069401C2DD060690068401C29D03D
:1003400060692CE010212846FFF7FEFE31688142EB
:100350001CD1A16901F18002C03105E030B108CAA9
:1003600051F8040D984201D1012000E000208A429A
:10037000F4D158B1286810B1042803D0FEE728460C
:1003800000F057F861496868086008E000F016F866
:1003900000F008F84FF480500168491C01D000F0CB
:1003A000A3FAFEE7BFF34F8F59480168594A01F499
:1003B000E06111430160BFF34F8FFEE74FF0102063
:1003C0008169491C02D0806900F0ADB87047524A7B
:1003D00001681160121D416811604F4A8168103236
:1003E0001160111DC068086070472DE9F041174683
:1003F0000D460646002406E03046296800F0A6F8BF
:10040000641C2D1D361DBC42F6D3BDE8F08170B5CD
:100410000C4605464FF4806608E0284600F083F855
:10042000B44205D3A4F5806405F58055002CF4D1C1
:1004300070BD4168044609B1012500E000254FF078
:1004400010267069A268920000F0BCF9C8B120467D
:1004500000F01AF89DB17669A56864684FF4002031
:1004600084420AD2854208D229463046FFF7CFFFA0
:100470002A4621463046FFF7B8FFFFF79FFFFFF7F8
:1004800091FFFFF747FEF8E72DE9FF414FF01024F9
:10049000616980680D0B01EB800000F6FF70010BB5
:1004A00000200090019002900246039068460123CC
:1004B0000BE0560902F01F0C50F8267003FA0CFCF2
:1004C00047EA0C0740F82670521CAA42F1D30AE012
:1004D0004A0901F01F0650F8225003FA06F6354388
:1004E00040F82250491C8029F2D3A169090B4A091E
:1004F00001F01F0150F822408B409C4340F82240FD
:10050000FFF765FFBDE8FF815809000000000020EB
:100510000CED00E00400FA050006004014480168F4
:100520000029FCD07047134A0221116010490B6862
:10053000002BFCD00F4B1B1D186008680028FCD056
:100540000020106008680028FCD07047094B10B5E7
:1005500001221A60064A1468002CFCD00160106861
:100560000028FCD00020186010680028FCD010BDC6
:1005700000E4014004E5014008208F49096809585A
:10058000084710208C4909680958084714208A49EF
:100590000968095808471820874909680958084711
:1005A0003020854909680958084738208249096878
:1005B000095808473C2080490968095808474020E5
:1005C0007D4909680958084744207B49096809584A
:1005D0000847482078490968095808474C20764957
:1005E000096809580847502073490968095808479D
:1005F0005420714909680958084758206E4909680C
:10060000095808475C206C49096809580847602068
:100610006949096809580847642067490968095801
:100620000847682064490968095808476C206249EE
:1006300009680958084770205F4909680958084740
:1006400074205D4909680958084778205A490968A3
:10065000095808477C2058490968095808478020EC
:1006600055490968095808478420534909680958B9
:100670000847882050490968095808478C204E4986
:1006800009680958084790204B49096809580847E4
:10069000942049490968095808479820464909683B
:1006A000095808479C204449096809580847A02070
:1006B0004149096809580847A4203F490968095871
:1006C0000847A8203C49096809580847AC203A491E
:1006D000096809580847B020374909680958084788
:1006E000B4203549096809580847B82032490968D3
:1006F00009580847BC203049096809580847C020F4
:100700002D49096809580847C4202B490968095828
:100710000847C8202849096809580847CC202649B5
:10072000096809580847D02023490968095808472B
:10073000D4202149096809580847D8201E4909686A
:1007400009580847DC201C49096809580847E02077
:100750001949096809580847E420174909680958E0
:100760000847E8201449096809580847EC2012494D
:10077000096809580847F0200F49096809580847CF
:10078000F4200D49096809580847F8200A49096802
:1007900009580847FC2008490968095808475FF4C8
:1007A0008070054909680958084700000348044952
:1007B000024A034B70470000000000206809000057
:1007C0006809000040EA010310B59B070FD1042A15
:1007D0000DD310C808C9121F9C42F8D020BA19BA0C
:1007E000884201D9012010BD4FF0FF3010BD1AB171
:1007F000D30703D0521C07E0002010BD10F8013BC6
:1008000011F8014B1B1B07D110F8013B11F8014BEC
:100810001B1B01D1921EF1D1184610BD02F0FF033F
:1008200043EA032242EA024200F005B870477047EB
:1008300070474FF000020429C0F0128010F0030C42
:1008400000F01B80CCF1040CBCF1020F18BF00F8C3
:10085000012BA8BF20F8022BA1EB0C0100F00DB872
:100860005FEAC17C24BF00F8012B00F8012B48BFD0
:1008700000F8012B70474FF0000200B51346944674
:100880009646203922BFA0E80C50A0E80C50B1F1E8
:100890002001BFF4F7AF090728BFA0E80C5048BFFC
:1008A0000CC05DF804EB890028BF40F8042B08BF9A
:1008B000704748BF20F8022B11F0804F18BF00F896
:1008C000012B7047014B1B68DB68184700000020B4
:1008D00009480A497047FFF7FBFFFFF713FC00BD0B
:1008E00020BFFDE7064B1847064A1060016881F3F8
:1008F0000888406800470000680900006809000097
:100900001D030000000000201EF0040F0CBFEFF3D9
:100910000881EFF30981886902380078182803D12B
:1009200000E00000074A1047074A12682C3212689C
:100930001047000000B5054B1B68054A9B589847B7
:1009400000BD000005030000000000205409000065
:1009500004000000001000000000000000FFFFFF86
:040960000090D00330
:10100000881100207DB0010079960000CDAF01006D
:1010100079960000799600007996000000000000A3
:10102000000000000000000000000000D9B0010036
:101030007996000000000000799600007996000083
:1010400041B1010047B10100799600007996000096
:101050007996000079960000799600007996000054
:101060004DB10100799600007996000053B101005E
:101070007996000059B101005FB1010065B101002E
:101080007996000079960000799600007996000024
:101090007996000079960000799600007996000014
:1010A0006BB1010071B101007996000079960000E2
:1010B00079960000799600007996000079960000F4
:1010C00077B10100799600007996000079960000CA
:1010D00079960000799600007996000079960000D4
:1010E00079960000799600007996000079960000C4
:1010F00079960000799600007996000079960000B4
:10110000799600007996000000F002F819F093FF3C
:101110000AA090E8000C82448344AAF10107DA4552
:1011200001D119F088FFAFF2090EBAE80F0013F0F1
:10113000010F18BFFB1A43F00103184734A5010043
:1011400054A501000A4410F8014B14F00F0508BF24
:1011500010F8015B240908BF10F8014B6D1E05D083
:1011600010F8013B6D1E01F8013BF9D1641E03D05C
:10117000641E01F8015BFBD19142E4D3704700008B
:101180000023002400250026103A28BF78C1FBD890
:10119000520728BF30C148BF0B6070471FB500F031
:1011A0003DF88DE80F001FBD1EF0040F0CBFEFF3DC
:1011B0000880EFF30980014A10470000CB9400003B
:1011C0008269034981614FF00100104470470000BB
:1011D000D511000001B41EB400B510F085F901B4BA
:1011E0000198864601BC01B01EBD0000F0B4404627
:1011F000494652465B460FB402A0013001B506488D
:10120000004700BF01BC86460FBC80468946924617
:101210009B46F0BC704700000911000019F008BFA0
:1012200070B51C4C054608202070A01C00F065F825
:101230005920A08029462046BDE8704006F067BBD3
:1012400010B506F06FFB13490020891E087010BD11
:1012500070B50C460F49891E097829B1A0F16001CB
:10126000532906D3012011E0602802D043F2010087
:101270000CE020CC084E94E80E0006EB8000A0F5B0
:101280008050241FD0F8806E2846B047206070BD83
:10129000012070470A000020BCB1010010B50446CF
:1012A0000021012000F03FF80021182000F03BF859
:1012B00000210B2000F037F80421192000F033F84A
:1012C00004210D2000F02FF804210E2000F02BF84F
:1012D00004210F2000F027F80421C84300F023F870
:1012E0000721162000F01FF80721152000F01BF839
:1012F0002046FFF795FF002010BD81210180704737
:10130000FFF79EBF10487047104A10B514680F4B86
:101310000F4A08331A60FFF79BFF0C48001D04605A
:1013200010BD704770474907090E002806DA00F023
:101330000F0000F1E02080F8141D704700F1E0205C
:1013400080F800147047000003F9004310050240C4
:101350000100000130B5FB4D044610280AD0112CC5
:1013600006D02846122C817806D0132C08D0FFDF37
:10137000AC7030BDFFDFFBE71129F9D0FFDFF7E7E5
:101380001129F5D0FFDFF3E770B50EF03CF9044604
:101390000FF072FE201AC4B206200CF0F9FA0546CE
:1013A00006200CF0FDFA2E1A07200CF0F1FA054683
:1013B00007200CF0F5FAE349281A32188878122829
:1013C0000DD000231A4413280BD0002002440878C3
:1013D000022808D000201044201AC0B270BD01239A
:1013E000F0E70120F2E70120F5E7D64810B5C17813
:1013F00094B0A9B15FF017018DF800104168CDF8E5
:1014000002100089ADF8060009A968460AF0D1F873
:101410000446112801D004B1FFDF14B0204610BDEE
:101420003221E9E702210CF008BB2DE9F04194B02C
:101430001D4690460E460746FFF7F4FF04000BD00A
:101440002078222804D3A07FC0F34010A84206D100
:10145000082014B0BDE8F08143F20200F9E737201C
:101460008DF80000ADF802703DB101208DF8040048
:101470008DF805608DF8068002E000208DF80400EC
:1014800009A968460AF095F8A07F65F34510A07792
:101490000020DEE730B50446A1F120000D460A2801
:1014A0004AD2DFE800F005070C1C2328353A3F44F8
:1014B000FFDF42E0207820283FD1FFDF3DE0A14858
:1014C0000178032939D08078132836D02078242851
:1014D00033D0252831D023282FD0FFDF2DE02078EE
:1014E00022282AD0232828D8FFDF26E020782228A7
:1014F00023D0FFDF21E0207822281ED024281CD012
:1015000026281AD0272818D0292816D0FFDF14E063
:101510002078252811D0FFDF0FE0207825280CD077
:10152000FFDF0AE02078252807D0FFDF05E02078DC
:10153000282802D0FFDF00E0FFDF257030BD30B586
:101540000B8840F67B444FF6FF72022801D093428D
:1015500004D09D1FA54224D2022802D04D88954276
:1015600003D04D88AD1FA5421BD24C88A34218D88A
:101570008B88B3F5FA7F14D2022802D0C888904233
:1015800005D0C88840F677450A38A84209D2C888ED
:10159000904208D0944206D05B1C6343B3EB800FAB
:1015A00001DB072030BD002030BD70B5044610F0CF
:1015B00003FA60BB207930B1082802D8217B0829C2
:1015C00005D9072070BD217B0029FAD0F6E718B1B4
:1015D000206810F0F1F9D0B9207B18B1A06810F0A4
:1015E000EBF9A0B9002507E0206850F8250010F0BD
:1015F000E3F960B96D1CEDB22079A842F4D800255A
:1016000009E0A06850F8250010F0D6F908B11020C4
:1016100070BD6D1CEDB2207BA842F2D8002070BDD9
:1016200010B5028943F6FD73111F994212D2418908
:1016300004290FD3B1F5804F0CD891420AD8017814
:10164000890705D5406818B1FFF7AFFF002800D122
:10165000002010BD072010BDF0B50024059D10B17D
:10166000A94203D851E009B90020F0BD0920F0BD1E
:10167000055D8DB107197E78112E3FD00FDC0A2E43
:101680003CD2DFE806F03B1624242A2A2C2C3333E4
:10169000025D72BB641CE4B28C42F9D3E4E71D2EF8
:1016A0002CDAA6F11206042E28D2DFE806F027274E
:1016B0001018022DDAD1BD781D70072D01D26D07EB
:1016C00001D40A20F0BD157845F0010515E0EE4380
:1016D000F60707E0012D07D010E00620F0BD2E0729
:1016E000A6F18056002EF5D06046F0BD1578AE0705
:1016F00001D50B20F0BD45F002051570055D641C99
:101700002C44E4B28C4202D9B0E74FF4485C8C42DE
:10171000AED3A9E710B504784CB1012243F20223FD
:10172000012C07D0022C0FD0032C17D112E000227D
:101730000A7015E00A7082790324B4EB921F0DD170
:101740000EE00000A80100200A708479B2EB941F1B
:1017500004D105E00A708279920901D0184610BDC3
:1017600050F8012F41F8012F80888880002010BD9B
:1017700008B538B1FEA06B4600680090487903EBCD
:10178000901000781070086842F8010F88889080E7
:1017900008BD30B50C46097895B0222902D2082040
:1017A00015B030BD28218DF80010ADF80200132AC5
:1017B00003D03B2A01D00720F2E78DF8042009A9C5
:1017C000684609F0F6FE050003D121212046FFF707
:1017D00061FE2846E4E700B595B023218DF800109E
:1017E000ADF802001088ADF804005088ADF806008E
:1017F000D088ADF80A009088ADF808000020ADF858
:101800000C00ADF80E0009A9684609F0D2FE15B02B
:1018100000BD70B50E46050003D00021092010F070
:1018200088F8D44C0120022EE0701CD0032E00D08A
:10183000FFDF0621201D0FF071FD607A20F0C0004F
:1018400084F80900FFF7D1FD608A00280AD0002D36
:1018500008D083000122002109200FF0CDFF0928C4
:1018600000D0FFDF70BD0321E01D0FF057FD607A4F
:1018700020F0C00040F040006072E01C02F03BFC31
:10188000E0E72DE9FF410220BA4E8DF80400002761
:10189000F08AADF80600B84655E001A80CF037F81C
:1018A000050006D0F08AB0B3A6F81680ADF8068021
:1018B00047E0039C2078212843D0A07F01072BD547
:1018C00004F123000090A28EBDF80800214604F127
:1018D000360301F02BFD050003D011282AD0FFDFCD
:1018E00028E0A07F20F00800A077E07F810861F366
:1018F0000000C10861F34100E07794F8210000F096
:101900001F0084F820002078282824D1292120468F
:10191000FFF7C0FD1FE01CE0400712D5BDF808002E
:10192000214604F10E02FFF756FF050004D01128EE
:1019300000D0FFDF00250EE0A07F20F00400A0779C
:1019400009E07F1CFFB202200CF022F8401CB842D4
:10195000A3D8052D07D0BDF80600F082052D04D0D0
:10196000284604B076E5A6F816800020F9E72DE9B0
:10197000F047040000D1FFDF20787E4E20F00F00FA
:10198000801C20F0F0007030207060680178091F22
:1019900011290BD2DFE801F0F1090A4FF00A0CF02F
:1019A000F0360A0A0A0AF174F100FFDFBDE8F08799
:1019B00087883846FFF736FD050000D1FFDF6078E5
:1019C000212140F008006070307D40F00400307547
:1019D0002846FFF75FFD384606F089FD384603F0DC
:1019E00021FC384604F03BFC394602200FF0A1FFF1
:1019F000A87F20F01000A877FFF743FF0028D5D07C
:101A0000FFDFD3E785882846FFF70CFD00B9FFDF2D
:101A100060688078012800D0FFDF606881792846FF
:101A200006F0D8FE0028C1D0617841F0080161704D
:101A30006168C880BAE786883046FFF7F3FC050086
:101A400000D1FFDF6078314640F0080060706068C8
:101A5000C088288160680089688160684089A881A1
:101A600002200FF066FF0020A875A87F00F0030099
:101A700002289BD1FFF705FF002897D0FFDF95E7ED
:101A800080783C2803D0002502280AD000E00125F8
:101A9000002720B13C2802D0022800D0FFDF17B178
:101AA0007EE00127F5E7607840F008006070307D47
:101AB00040F008003075EDBB606802218788384629
:101AC0000BF0B2FF0546032138460BF0ADFF82460E
:101AD000052138460BF0A8FF8146042138460BF05B
:101AE000A3FF804605B9FFDFBAF1000F00D1FFDF89
:101AF000B9F1000F00D1FFDFB8F1000F00D1FFDF17
:101B000022212846FFF7C6FC60688079012837D07B
:101B10004FF00208A87F68F30100A8776068C08AC8
:101B200028816068008B68816068408BA88160684C
:101B3000C07900E027E0E87560688168A961808964
:101B4000A8836068807B6870606850F80F1FC5F8D4
:101B500002108088E880A87F00F00301384606F074
:101B6000B8FCB8F1010F0ED0B8F1020F18D005E0A3
:101B70000302FF01A80100201FE023E0FFDF15E7BB
:101B80004FF00108C6E73078032800D0FFDF0021BE
:101B900008460FF0CEFEBDE8F047012000F087BFF9
:101BA000B078132800D0FFDF002107200FF0C1FE1E
:101BB000BDE8F0471120FFF7CDBB2046BDE8F04758
:101BC00001F08CBE607840F008006070EEE62DE910
:101BD000F0470546007800270009DFF894A69146F3
:101BE0000C463E46012871D0BC464FF6FF710228D4
:101BF0006DD0072809D00A286AD0FFDFA9F8006055
:101C00000CB1278066800020D0E6686804F10802E5
:101C100003780D2B40D006DC042B7DD0072B44D05D
:101C20000A2B7AD106E0122B46D0132B51D0142B5D
:101C3000F7D1C0E011270926002C6FD0B0F804803E
:101C4000A4F804806868807920729AF814104046DD
:101C500021F004018AF8141004210BF000FF052183
:101C600040460BF0FCFE002140460BF0F8FE01213F
:101C700040460BF0F4FE032140460BF0F0FE02213B
:101C800040460BF0ECFE062140460BF0E8FE072133
:101C900040460BF0E4FEB1E701270926002CCCD02A
:101CA0008088A080686880790EE0122710268088DE
:101CB000214600F01EFFA1E71C270926002CBCD0FE
:101CC0004088A08068680079207297E78AE0B3E0D6
:101CD00082E081783C2938D010272026002CACD017
:101CE0008088A0806868C08A60836868C08A208312
:101CF0006868008BA0836868408BE0836868417FD8
:101D0000E07D61F30000E0756968497F490861F38F
:101D10004700E075696802E022E05CE08BE0C8798A
:101D20000831FFF725FD696804F10F0201F10F008A
:101D30008B7B01461846FFF71BFD6868807910B160
:101D40000120A07507E00220FBE71B270926002CD5
:101D500071D084F808C09AF8141021F008018CE0C2
:101D60001D273026002C66D0A1806868411D0079AF
:101D7000FFF7FEFC686890F82B00E0736868C07895
:101D80000428207C14D020F00100207469681F22F0
:101D9000C97861F3420020746968C97A61F3C700A9
:101DA0002074696804F111000C3119F043F825E73B
:101DB00040F00100E9E720271026E4B3A18068681D
:101DC00004F10902407A20726968CB1C88781946B0
:101DD000FFF7CEFC12E74A4621462846BDE8F04709
:101DE00001F001BF287E012803D0022813D0FFDFB5
:101DF00004E71F271026F4B16888A080688B208133
:101E0000A88B6081E88BA081288CE0819AF814105F
:101E100021F0200131E012271026688800F069FEC9
:101E20004CB1687800F007000328C0D19AF814106C
:101E300021F0020121E027E0287E062822D2DFE8F7
:101E400000F0040F0F030303C5E71B270926DCB1CD
:101E5000A18084F808C09AF8141021F001010CE068
:101E60001B27092684B1A180287E012808D00320E1
:101E700020729AF8141021F010018AF81410BDE6AF
:101E80000220F5E7FFDFB9E6A9F80060BBE610B570
:101E9000F74894B08078132802D0082014B010BD01
:101EA00022208DF8000009A9684609F082FB04464B
:101EB000002107200FF03DFD2046EFE700B5EC487C
:101EC00095B08078122801D00820A0E41E208DF85B
:101ED000000000208DF802008DF8030009A9684673
:101EE00009F067FB0028F0D1002107200FF021FD49
:101EF0001120FFF72FFA002089E400B5DC4895B0E7
:101F00000078022803D0032801D008207FE41B209A
:101F10008DF8000000208DF8020009A9684609F03C
:101F200048FB0028F2D1002108460FF002FD0120F5
:101F300000F0BDFD00206AE42DE9F0410027CC4C03
:101F40000A287CD2DFE800F0057B1C7B7B7B7B448E
:101F50003B6AFFF7D2FF002831D105F01FFC0028B3
:101F60002DD0017821F00F01891C21F0F0012031E2
:101F70000170077605F0F0FB207D40F001001DE0C8
:101F80008EB23046FFF74EFA050000D1FFDF287809
:101F9000212814D005F002FC98B1017821F00F013E
:101FA000891C21F0F0011031017002210176468078
:101FB000AF7505F0D1FB207D40F002002075BDE833
:101FC000F08129463046BDE8F0411322FFF7E1BB1E
:101FD000A578122D03D0132D04D0FFDFEFE7FFF714
:101FE0006DFF01E0FFF753FF0028E8D105F0D6FBB5
:101FF0000028E4D0017821F00F01891C21F0F001C4
:1020000020310170122D07D00221017605F0A4FBCA
:10201000207D40F01000D1E70121F6E7607A012130
:10202000B1EB901F02D1022104E008E0800900D04A
:10203000FFDF0321BDE8F0410020FFF7EABBFFDF2F
:10204000BDE72DE9F04114460D00074600D1FFDF42
:102050002878012803D0022821D0FFDFAFE73846D7
:10206000FFF7E0F9060000D1FFDF0220B07520780D
:1020700020F00F00801C20F0F000103020706078FD
:1020800040F0080060702868A0616868E0612889F5
:1020900020847748017D41F0200101758FE73846A3
:1020A000FFF7C0F9060000D1FFDF69884FF6FF7027
:1020B000814209D1AA88824206D131463846BDE81C
:1020C000F0411322FFF765BB814201D1A88898B186
:1020D000207820F00F00801C20F0F00010302070DD
:1020E000607840F0080060702868A0616868E0616E
:1020F00028892084002006E0782300223946022027
:102100000FF07AFB0120B07559E730B5054695B060
:102110000C4608460FF050FC78BB00200121203D02
:10212000062D5FD2DFE805F0032540444A57002121
:1021300008200FF0D7FB10B1112015B030BD2420BE
:102140008DF80000D4F80200CDF80200A0798DF8D7
:10215000060009A9684609F02CFA05002CD10823CD
:102160000022114618460FF047FB082824D0FFDF55
:1021700022E060680FF062FC08B11020DDE73C202F
:102180008DF800002088ADF802006088ADF80400EA
:1021900009A9684609F00DFA05000DD1606858B12B
:1021A000BDF82810018007E0206801F0E2FF02E09E
:1021B000204600F0B1FC05462846BEE73D220BE074
:1021C0008DF8021002E000BF8DF8020009A96846F0
:1021D00009F0EFF9EFE734228DF800202278D207DA
:1021E000F2D0EDE70720A8E730B5054695B00C46DC
:1021F00008460FF005FC70BB203D052D35D2DFE809
:1022000005F00323232523002088FFF70BF920B1D5
:102210000078222804D208208FE743F202008CE7DE
:1022200025208DF800002088ADF8020009A9684635
:1022300009F0BFF9002880D1DDF82A10C4F8021097
:102240009DF82E10A17178E7062076E7206838B156
:102250000FF0F4FB08B110206FE7206801F07DFF5C
:102260000348408AA080002067E7072065E7000058
:10227000A8010020FE487047FD4810B518210A3813
:1022800018F04FFE012000F012FC1120FFF762F859
:10229000F74C00200A3C211D60744FF4617060828D
:1022A000E01C05F043FBD4F80300C4F80A00B4F8BE
:1022B0000700E081607A2074FFF797F800B1FFDF34
:1022C00000F09CFCBDE8104001F0C2BA10B50C460D
:1022D0003E21204618F025FEA07F20F00300A077C5
:1022E000202020700020A07584F8220010BD7047C7
:1022F0002DE9FC4105460E4608460FF05DFB10B186
:102300001020BDE8FC81DA4C0A3C15B1012D38D112
:102310002CE0D4F803000090B4F80700ADF80400F6
:102320008046677A8DF80670E11C3046FFF7F2F9B7
:102330000028E6D1FFF759F830B10099C4F803102E
:10234000A4F807806772DCE7307808B1012808D16B
:10235000D4F80300C4F80A00B4F80700E081607AFA
:102360002074002109200FF0E4FA0FE0317841B128
:10237000012906D0022906D0032904D043F2022005
:10238000BFE70720BDE70120FFF743FA657400208F
:10239000B7E710B504460FF033FB08B1102010BDAD
:1023A000B34922460A39C878091DFFF7E1F9002030
:1023B00010BD2DE9F0419AB0054600208DF85C0073
:1023C0008DF858008DF828008DF860001E461446E0
:1023D000884628460FF03BFB18B920460FF037FB24
:1023E00010B110201AB0EAE555EA040018D01F27F2
:1023F0000AAB17AA414628460097FFF72DF9002897
:10240000F0D118AB16AA314620460097FFF724F901
:102410000028E7D19DF85800C00703D00A20E1E763
:102420000720DFE701AF7DB11A208DF804008DF899
:10243000068042462946F81C18F0FCFC0BA901A8AE
:1024400009F0B7F80028CDD17CB120208DF8040028
:102450008DF8066032462146F81C18F0EBFC0BA9FB
:1024600001A809F0A6F80028BCD181499DF82800F0
:102470000A3948700020B5E770B506460A200C46B8
:10248000087015461146204609F093F830B93821F6
:1024900021702046294609F08CF820B1082801D186
:1024A00043F2032070BD2A462146304600F05BFB14
:1024B0000446082800D1FFDF204670BD2DE9F04119
:1024C0006CA196B00446D1E90001CDE914010027C2
:1024D00020460FF071FA30B92078012806D16068E3
:1024E0000FF06AFA10B1102016B068E5604D0A3D91
:1024F0002878012801D00820F6E707200BF050FAD1
:1025000018B9207848B1012807D0FEF73DFF30B157
:10251000287D10F00C0F09D103E01220E4E713200E
:10252000E2E7C10702D1A846800701D51120DBE709
:10253000208A43F6E172A0F120019142217807D36D
:10254000012942D1002840D1618A00293DD10FE004
:10255000022901D0032901D1A02836D3012907D0AF
:1025600098F80110C90703D0618A71B3B4292CD837
:10257000217831B1012908D0022904D0032924D1BE
:1025800015E0002516E0022514E008B9608A60B164
:1025900004256068007868B101280AD0022808D0B4
:1025A000032806D043F202209EE70125F1E7032528
:1025B00000E00127207A30B1012807D0022807D097
:1025C00003286AD106E0002605E066E0012602E065
:1025D000022600E003260DB1022D13D196B1E0686A
:1025E00018B1FEF7E2FF002886D198F801008007B5
:1025F00002D043F2012077E7022D03D1022E4CD006
:10260000032E4AD018208DF82C00208AADF82E0019
:10261000208AADF830008DF8325098F80310002071
:102620004FF0010811B1012968D102E08DF83300A3
:1026300001E08DF833808DF834702178012925D0A0
:10264000CDF83500ADF839008DF83C60207DC0F341
:102650004002014662F35F01C0F3800041EA80005E
:1026600014A9085C8DF83B00B8B169460BA805E0D9
:10267000B2010020070605040302010008F099FFDB
:10268000002891D15DB1022D09D011E0606850F8A9
:10269000011FCDF835108088D4E7072024E73EB12C
:1026A000E06828B16A460BA9FFF7E6FE0028A2D130
:1026B0001B208DF82C008DF82E8069460BA808F0A1
:1026C00078FF002897D19DF801001B2816D1052D11
:1026D00009D2DFE805F0030305050300032000E04D
:1026E000022000F0E4F9012D0AD0608A40B10022F6
:1026F0008300114610460FF07FF808B10320F3E67F
:102700000020F1E62DE9FC4107460D460326084668
:102710000FF09DF9002863D13846FEF783FE0400D0
:1027200004D02078222804D20820EAE543F20200EF
:10273000E7E5A07F00F0030C2DB129466046FEF7C7
:10274000FEFE0600F1D1F948BCF1010F05D0BCF145
:10275000020F17D0FFDF3046D3E5A27D2946012ABC
:1027600002D0007D800701D51120CAE529B968464D
:1027700000F0FDFA0028D8D16946384605F0A7FFD9
:102780000646E8E7A17D022914D1007D800611D418
:1027900025B1A07F40070BD4002100E0012138467D
:1027A00005F0E0FF0600D6D1A075002DD3D002E0E1
:1027B0001126D0E7A5B12A4621463846FFF70BF887
:1027C00006461128C7D1A07F4107C4D4296844F820
:1027D0000E1F6968616040F0040020740026BAE7AB
:1027E00010208EE570B50C460546FEF71BFE010075
:1027F00005D022462846BDE87040FEF7CABF43F226
:10280000020070BD00B595B031218DF800108DF833
:10281000020009A9684608F0CCFE15B000BD0123EE
:10282000FEF703BE00231A461946FEF7FEBD70B53B
:1028300094B004460FF0C0F810B1102014B070BD71
:102840002046FEF7EDFE0028F8D1B84DA8781128F3
:1028500001D00820F2E7FEF797FD20B1287DC006E1
:1028600003D51120EAE71320E8E71D208DF80000CA
:10287000207800F001008DF802002089ADF80400F6
:102880006089ADF806002078C0F340008DF809009B
:10289000E8780025012618B1012804D00320CDE7EF
:1028A0008DF8085001E08DF8086009A9684608F025
:1028B00080FE0028C2D12078800707D5606828B143
:1028C00009AA6946FFF7D8FD0028B7D11E208DF868
:1028D00000008DF802608DF8035009A9684608F0E1
:1028E00068FE0028AAD1A08900F0F5F80400A5D15F
:1028F0001220FEF72FFD2046A0E7F0B595B0154653
:102900000C4607460FF0A3F838B920460FF054F8EC
:1029100018B928460FF050F810B1102015B0F0BDCE
:10292000824E307D10F0180F01D1400701D51120E3
:10293000F4E72046FEF774FE0028EFD12078C0F3BC
:102940004001394302D0800702D50FB10720E5E7E7
:1029500029460220FEF7F3FD0028DFD1B0781128C8
:1029600003D0122801D00820D8E706200BF018F871
:1029700018B1B078122802D005E01220CEE7FFF798
:102980009DFA0028CAD1FEF7FFFC022801D21320CD
:10299000C4E72078800707D5606828B109AA69468E
:1029A000FFF76AFD0028B9D121208DF800002089A9
:1029B000ADF802006089ADF8040020784FF0010105
:1029C000C0F340008DF80600207882074FF0000029
:1029D00015D43A7842B1012A09D0022A07D0032A35
:1029E00005D043F2022099E78DF8070001E08DF849
:1029F000071057F8012F0292BA88ADF80C20F27830
:102A00001AB1012A04D0032088E78DF80E0001E0F6
:102A10008DF80E102988ADF810106988ADF81210E5
:102A2000A988ADF81410E988ADF81800ADF81610B3
:102A3000ADF81A0009A9684608F0BBFD002886D148
:102A4000A08900F048F804008ED11320FEF782FC24
:102A5000204663E730B5054695B00C4608460EF0B3
:102A6000CFFF10B1102015B030BD2846FEF7DAFCBC
:102A700038B10178222902D3807F800604D408204F
:102A8000F1E743F20200EEE713208DF80000ADF805
:102A9000025009A9684608F08CFD0028E3D19DF991
:102AA0002A107F2901D02170DDE70520DBE730B552
:102AB0001E4D040008D0012C04D0022C06D0032C9B
:102AC00004D0FFDF2C7030BDFFDFFBE72878012842
:102AD000F8D0FFDFF6E710B548B1830000221146B9
:102AE00007200EF089FE072801D0032010BD00202A
:102AF00010BD70B50C0006460DD0FEF793FC050026
:102B000000D1FFDFA680288920812889608168891B
:102B1000A081A889E08170BD10B50446006840B16D
:102B20000EF095FF20B1102010BD0000A80100207C
:102B3000206801F005FBA0882F4C6082607C012892
:102B40000FD1002109200EF0CDFE00B10120617AE5
:102B50000122B2EB911F01D1022100E00321FEF717
:102B600058FE0020E0E72DE9F047002592460C468C
:102B70000646A8464FF001090B2721E0306850F8BF
:102B80002500007820B1012805D00720BDE8F08796
:102B900084F8028001E084F80290306850F8250043
:102BA00050F8011FC4F803108088A4F807002770AC
:102BB0005146204608F0FDFC0028E7D16D1CEDB21F
:102BC0003079A842DAD8002539270FE0B068102202
:102BD00050F82510A01C18F02DF9277051462046FA
:102BE00008F0E7FC0028D1D16D1CEDB2307BA84283
:102BF000ECD80020CAE70000A8010020E848002126
:102C00000160818070472DE9FF41804692B01C46EB
:102C10000E4618460EF0D0FE18B1102016B0BDE8D2
:102C2000F08121460120FEF78AFC0028F6D101251B
:102C30008DF842504FF4C050ADF84000002210A96A
:102C4000284603F0AAFD0028E8D18DF842504FF441
:102C50002850ADF8400000271C216846099718F05D
:102C600082F99DF82400ADF8346020F00F00401C7C
:102C700020F0F00010308DF824009DF82500ADF80C
:102C8000367020F0FF008DF825009DF8260007AA79
:102C900020F00600801C40F001008DF826009DF811
:102CA00000000BA940F002008DF800001F20ADF8D5
:102CB000380009A80C9010A80B90CDF83C8068460D
:102CC00003F06EFB0028A9D1B54EBDF81C0007AA81
:102CD00030808DF8425042F60120ADF840009DF85A
:102CE00026000BA920F00600801C20F001008DF8C2
:102CF00026000220ADF83400ADF8380014A80F907B
:102D0000684603F04DFB002888D1BDF81C00708098
:102D1000311D204600F0ECF880E73EB5044608205F
:102D2000ADF8000020460EF047FE08B110203EBD71
:102D300021460120FEF703FC0028F8D12088ADF8D9
:102D400004006088ADF80600A088ADF80800E088AF
:102D5000ADF80A00924801AB6A468088002103F072
:102D600009FFBDF800100829E1D003203EBD1FB5C2
:102D70000446002002900820ADF80800CDF80CD0E1
:102D800020460EF019FE10B1102004B010BD84488A
:102D900002AA81884FF6FF7004F07BF80028F4D176
:102DA000BDF80810082901D00320EEE7BDF8001097
:102DB0002180BDF802106180BDF80410A180BDF82B
:102DC0000610E180E1E701B582B00220ADF8000015
:102DD000734802AB6A464088002103F0CBFEBDF881
:102DE0000010022900D003200EBD1CB50021009167
:102DF0000221ADF8001001900EF002FE08B1102083
:102E00001CBD67486A4641884FF6FF7004F041F8E0
:102E1000BDF800100229F3D003201CBDFEB5074603
:102E200014460E4608460EF0C7FD08B11020FEBD40
:102E30001F2C01D90C20FEBD38460EF0BDFD584DAB
:102E400018BB288801A903F021F80028F3D13878AD
:102E50008DF80500288801A903F06DFE0028EAD14D
:102E600000909DF800009DF8051040F002008DF8DC
:102E70000000090703D040F008008DF80000288802
:102E8000694603F0FBFD0028D5D1ADF8084028883D
:102E9000334602AA002103F06DFEBDF80810A142DE
:102EA000C9D00320FEBD7CB50546002000900190EE
:102EB0000888ADF800000C46284601950EF0BEFDCE
:102EC00018B920460EF09CFD08B110207CBD15B14C
:102ED000BDF8000050B132486A4601884FF6FF70D5
:102EE00003F0D7FFBDF8001021807CBD0C207CBD15
:102EF00030B593B0044600200D460090142101A87F
:102F000018F031F81C2108A818F02DF89DF80000E1
:102F1000CDF808D020F00F00401C20F0F000103059
:102F20008DF800009DF8010006AA20F0FF008DF842
:102F300001009DF8200001A940F002008DF820005A
:102F400001208DF8460042F60420ADF8440011A897
:102F500001902088ADF83C006088ADF83E00A08864
:102F6000ADF84000E088ADF842009DF8020020F086
:102F70000600801C20F001008DF802000820ADF84A
:102F80000C00ADF810000FA8059008A803F008FA8F
:102F9000002803D1BDF818002880002013B030BDF0
:102FA00010000020094810B504680A490848086064
:102FB0000DF08AFB0848046010BD08490020086035
:102FC0004FF0E0210220C1F8800270471005024056
:102FD000010000011805024014050240FC1F0040DA
:102FE00070B50C46054606F0BFFE21462846BDE8F2
:102FF000704007F09CBE704770477047704770473D
:1030000010FFFFFFDBE5B15100C001008100FFFFB1
:1030100010B504460EF0D0FC08B1102010BD207889
:10302000C0F30210042807D86078072804D3A178D9
:10303000102901D8814201D2072010BDE078410754
:1030400006D421794A0703D4000701D4080701D523
:10305000062010BD002010BD10B513785C08C37F9A
:1030600064F30003C3771478A40864F34103C377BF
:103070001078C309887863F34100887013781C09BD
:103080004B7864F347134B701378DB0863F300004D
:1030900088705078487110BD10B5C4780B7864F30F
:1030A00000030B70C478640864F341030B70C478A8
:1030B000A40864F382030B70C478E40864F3C303C8
:1030C0000B700379117863F30001117003795B08C9
:1030D00063F34101117003799B0863F3820111705E
:1030E0000079C00860F3C301117010BD70B51446BB
:1030F0000D46064604F052FB80B10178142221F0FF
:103100000F01891C21F0F001A03100F8181B2146A5
:1031100017F0D5FEBDE8704004F01EBB29463046CE
:10312000BDE870401322FEF734BB70B514460E465E
:10313000054604F033FB70B1017821F00F01891CC2
:1031400021F0F00120310170458021688161BDE8E6
:10315000704004F001BB31462846BDE870401322A0
:10316000FEF717BB10B5FE4C94F8300000280CD1C8
:1031700004F120014FF6FF72A1F110000CF0B9F834
:1031800000B1FFDF012084F8300010BD2DE9F047C9
:10319000064608A8894690E830041F469046142148
:1031A000284617F0E0FE0021CAF80010B8F1000F21
:1031B00003D0B9F1000F03D114E03878C00711D063
:1031C00020680EF01DFCE8BBB8F1000F07D12068A5
:1031D000123028602068143068602068A860216878
:1031E000CAF800103878800727D560680EF026FCF2
:1031F00040BBB9F1000F2CD0FFF73CF80168C6F8CE
:10320000B4118188A6F8B811807986F8BA01FFF761
:10321000A9FFDFF84C8308F12008C5F80C8062682C
:103220005AB196F8B40106F2B5111032FEF7A0FAC1
:1032300010224146606817F0FDFD3878400712D52E
:10324000A06800E002E00EF0DBFB50B11020BDE80A
:10325000F08760680028F9D0E8606068C6F8B001BF
:10326000EBE7A06828610020F1E730B50546087853
:103270000C4620F00F00401C20F0F00110312170AE
:103280000020607095F8220030B104280FD0052886
:1032900011D0062814D0FFDF20780121B1EB101FD8
:1032A00004D295F8200000F01F00607030BD21F0BE
:1032B000F000203002E021F0F00030302070EBE729
:1032C00021F0F0004030F9E710B510B190F8A940B6
:1032D00044B1A34890F8354000205CB1086010600C
:1032E000186010BD00F1A8040C6000F1D001F830A6
:1032F0001160F5E79A4C34340C60F0E700B58BB000
:103300000823CDE902128DF8013001919449002380
:1033100064310591099301468DF8103068460BF031
:10332000C0FF002800D0FFDF0BB000BD30B595B066
:103330000C462C2518998DF80050ADF80200B3B159
:103340001868019058680290ADF80C2010220DF119
:103350000E0017F06FFD09A9684608F02AF9002849
:1033600003D1A17F41F01001A17715B030BD00203D
:103370000190E8E72DE9F0470646008A8AB080B25E
:103380000D468146FEF74EF80446754F3078283FCB
:10339000DFF8CC814FF0000A122873D2DFE800F08A
:1033A00072E9350936777E98A8F3E7E6E5E4DF5B56
:1033B000DFDFA07F00F00300012806D0002148468F
:1033C0000AF03BFB050003D101E00121F7E7FFDF35
:1033D00098F85C10090602D5D8F860000BE00321CC
:1033E00005F121000DF09AFFD5F821005D49B0FBF1
:1033F000F1F201FB1200C5F8210070686866B06840
:10340000A8662078252800D0FFDFECE0A07F00F040
:103410000300012806D0002148460AF00EFB0600F2
:1034200003D101E00121F7E7FFDF7078810702D5C2
:103430002178252904D040F0010070700AB006E719
:103440000220287096F82000287106F121003136FC
:10345000C5E90206F2E7A07F00F00300012806D0CC
:10346000002148460AF0E9FA040003D101E00121F5
:10347000F7E7FFDF6078C10605D5142028704134D6
:103480006C60DBE7E2E140F008006070D6E73448AA
:10349000082128380DF042FF032016E02A208DF87D
:1034A000000010220DF10200716817F0C3FC102219
:1034B0000DF11200B16817F0BDFC294968462C399E
:1034C00008F077F800B1FFDF042028706F60B5E7DF
:1034D000E07FC00600D5FFDFB0680090B388062209
:1034E0000321484605F063F80028A7D0FFDFA5E7D1
:1034F00004B9FFDF716821B1102204F1230017F035
:1035000099FC28212046FDF7C5FFA07F00F00300AD
:1035100002280ED104F12300002300901A46214610
:103520004846FFF703FF112807D029212046FDF761
:10353000B1FF307A84F8200080E7A07F000700D533
:10354000FFDF14F81E0F40F008002070A4F816A04A
:10355000C4F818A0C4F81CA0617808460AE034E05A
:103560005C02002040420F006CE19AE090E062E0D3
:1035700009E03FE061F38200410861F3C30060703D
:10358000307AE0705AE7A07F00F00300012806D0EF
:10359000002148460AF051FA040003D101E001215C
:1035A000F7E7FFDF022104F175000DF0B7FE1120EF
:1035B000287004F5DA706860B4F875002882FD4858
:1035C0006C346C61C5E9028038E7A07F00F003002D
:1035D000012805D0002148460AF02FFA18B901E069
:1035E0000121F8E7FFDF0AB0324621464846BDE830
:1035F000F0477BE504B9FFDF207821289CD930799A
:10360000012802D002280AD103E0E07F40F0100038
:10361000E07798F85C1041F0010188F85C103246C0
:1036200021464846FFF762FD0AB02046BDE8F04754
:103630002321FDF72FBF327901230321484604F0EF
:10364000B7FD98B1122005F8040B327925F8042B48
:10365000281DA91E0095CDE901100023032148462D
:1036600004F023FE00288DD0FFDFE7E6A07F00F006
:103670000300012806D0002148460AF0DEF90400C4
:1036800003D101E00121F7E7FFDF30792070D5E6B3
:103690000321484605F02DF9002895D11320287004
:1036A000CCE6A07F00F00300012806D000214846A8
:1036B0000AF0C3F9050003D101E00121F7E7FFDFBC
:1036C00095F8740000F00300012878D1A07F00F085
:1036D0000307E07FC0F3400616B1012F04D02BE0B2
:1036E00095F89000C0072AD0D5F8AC0118B395F82A
:1036F0007320017C62F387010174E27FD5F8AC018D
:1037000062F341010174D5F8AC0166F30001017464
:10371000AEB1D5F8AC01102204F12301783517F0D1
:1037200089FB287E40F001002876287820F00100EF
:1037300005F8780900E016B1022F04D02CE095F8C6
:103740007800C00726D0D5F8A80118B395F87320E3
:10375000017C62F387010174E27FD5F8A80162F36E
:1037600041010174D5F8A80166F3000101748EB11E
:10377000D5F8A801102204F12301783517F05AFB7F
:10378000287840F0010005F8180B287820F0010097
:1037900005F89009022F51D05FF0000000EB4000C7
:1037A00005EBC00090F87800800708D5D5F8B02167
:1037B00095F86C0005F16D011032FDF7D9FF052079
:1037C00060F3070815F8740F00F0030060F30F288A
:1037D000287960F31748287F60F31F687548AC3874
:1037E000027822F00F02921C22F0F00220320270C6
:1037F000427822F00702D21C4270A0F80290C0F872
:10380000188004F033F92078252805D0212807D026
:10381000FFDF2078222803D922212046FDF73AFE37
:10382000A07F00F0030001280AD0002148460AF0DA
:1038300016F900283FF40EAEFFDFFFE50120ADE7EB
:103840000121F3E7716881F801A0F7E5FFDFF5E5F5
:1038500070B5584C0025103C14F85C0F20F0800027
:10386000207065600BF0E7FC5249A1F1100004F0F4
:103870008FF804F82C5C072060724E487C30206181
:103880005030A0611030E06170BD70B50D46FDF79D
:10389000C9FD040000D1FFDF4FF4DE71284617F0A8
:1038A00062FB44485430686104F123002861A07F22
:1038B00000F00300012809D05FF0020105F59070C7
:1038C0000BF0BAFC002800D0FFDF70BD0121F5E746
:1038D0000A46014602F590700BF0CCBC70B5054667
:1038E00040689AB0017808290DD00B2903D00C2923
:1038F00036D101218171686886883046FDF792FDD6
:10390000040035D133E046883046FDF78BFD0400D6
:1039100000D1FFDF2078212822D0282822D1686812
:1039200002210C3001F09CF9E0B168680821001D0B
:1039300001F096F9B0B12D208DF80000ADF80260CD
:10394000102204F1230101A817F074FA09A96846AE
:1039500007F02FFE00B1FFDF29212046FDF79AFD79
:103960001AB070BD687840F008006870F8E7FFDFB3
:10397000A07F00F00301022902D120F01000A077FF
:10398000207821280AD06868817909B1807898B1B7
:10399000A07F00F0030002285BD0FFDFA07F00F0D3
:1039A00003000228DCD1FDF76CFF0028D8D0FFDF30
:1039B000D6E700006C020020687840F008006870CC
:1039C000E07FC10720D0800701D5062000E0052058
:1039D00084F822002078292818D02428DED1314606
:1039E00006200DF0A6FF22212046FDF753FDA07F03
:1039F00000F0030001282AD0002130460AF02FF8F9
:103A00000028CBD0FFDFC9E70420E1E7A07F00F06A
:103A10000300012806D0002130460AF00EF8050008
:103A200003D101E00121F7E7FFDF25212046FDF763
:103A300031FD10208DF8500014A905F590700BF0A1
:103A400010FC0228AAD00028A8D0FFDFA6E7012199
:103A5000D3E7687840F0080068709FE72DE9F047E9
:103A60008CB01D46904689460646DDF850A0FDF70D
:103A7000D9FC040052D0207822284FD323284DD0DF
:103A8000E07FC0064AD4A07F00F00300012806D0E2
:103A90000021304609F0D1FF070002D00BE00121E0
:103AA000F7E7A07F00F00300012804D10121304690
:103AB00009F0BAFF074601AB02AA03A93846FFF78F
:103AC00003FC039800B9FFDF4FB1039807F5907727
:103AD00087612078222806D0242804D007E00399A3
:103AE0000020886103E025212046FDF7D3FC0398E0
:103AF0000C2141704662A0F80480C0F80890A0F83C
:103B000006A0C560029901610199416104A90BF009
:103B1000C8FB022802D0002800D0FFDF0CB0BDE8AF
:103B2000F08730B589B00546FDF77CFC0178222985
:103B300033D9807F00F00300012806D000212846F9
:103B400009F07BFF040003D101E00121F7E7FFDF6B
:103B5000227801230321284604F02AFB00281CD0E8
:103B600012208DF80C00227806A8811F05ABCDE944
:103B700000310290ADF8102000230321284604F004
:103B800094FB00B1FFDF03A904F590700BF069FB13
:103B9000022802D0002800D0FFDF09B030BD10B5E8
:103BA00086B00446FDF73EFC0178222919D9807FB2
:103BB00000F00300012806D00021204609F03DFF57
:103BC000040003D101E00121F7E7FFDF13208DF8A6
:103BD0000000694604F590700BF043FB002800D00C
:103BE000FFDF06B010BD2DE9F05F05460C4600274B
:103BF0000078904601093E46BB4604F1080A0229B6
:103C00007ED0072902D00A2909D141E068680178ED
:103C1000082905D00B292BD00C2929D0FFDFC5E1BD
:103C200014271C26002C6CD04088A080FDF7FAFBDE
:103C30005FEA000900D1FFDF99F81700524609F149
:103C40001801FDF795FD68688089208269684868D9
:103C5000C4F812008868C4F81600A07E20F00600A0
:103C600040F00100A07699F81E0040F040014DE0C0
:103C70001A270A26002CD6D08088A080FDF7D2FB18
:103C8000050000D1FFDF51462846FFF7EEFA8DE12F
:103C90000CB1288DA080287E0E287CD006DC01285F
:103CA0007AD0022808D0032804D135E0102874D037
:103CB000112873D0FFDF79E11E270926002CB2D02E
:103CC000A088FDF7AFFB5FEA000900D1FFDF287F86
:103CD00000F003000128207A1BD020F001002072A0
:103CE000297F890861F341002072297FC90861F3A7
:103CF00082002072297F090961F3C300207201E06C
:103D000049E116E199F81E0040F0800189F81E1083
:103D10004CE140F00100E2E713270D26002CAAD069
:103D2000A088FDF77FFB8146807F00F0030001281B
:103D300006D00021A08809F080FE050003D101E033
:103D40000121F7E7FFDF99F81E0000F00302012AC6
:103D500059D0A86E817801F003010129217A54D04D
:103D600021F00101217283789B0863F341012172E4
:103D70008378DB0863F38201217283781B0963F384
:103D8000C3012172037863F306112172437863F350
:103D9000C711217203E060E0A6E08EE09EE084F8A7
:103DA00009B0C178A172012A32D04279E17A62F376
:103DB0000001E1724279520862F34101E1724279F5
:103DC000920862F38201E1724279D20862F3C30180
:103DD000E1720279217B62F30001217302795208BA
:103DE00062F3410121730279920862F38201217327
:103DF0000079C00860F3C301217399F800002328FB
:103E00005AD9262168E0686EA4E741F00101A9E7CC
:103E10000279E17A62F30001E1720279520862F3F9
:103E20004101E1720279920862F38201E172027942
:103E3000D20862F3C301E1724279217B62F300018F
:103E400021734279520862F3410121734279920849
:103E500062F3820121734079CBE718271026002CEA
:103E600067D0A088FDF7DEFA8246807F00F003006D
:103E7000012807D00021A08809F0DFFD5FEA0009D2
:103E800003D101E00121F6E7FFDFE869A06099F8BE
:103E9000010040F0040189F8011099F80200800740
:103EA00008D5012020739AF8000023287ED9272105
:103EB000504663E084F80CB078E015270F26C4B3B1
:103EC000A088FDF7AFFA814606225146E86907F05F
:103ED000D6FB0120A073AEE048464FE01627092626
:103EE0003CB3287F207261E0287FFE4902280CD075
:103EF00019270E26ECB101280DD003281AD004286A
:103F00001BD0052819D0FFDF23E01B270926BCB3EF
:103F10000120207205E001202072607A20F0030069
:103F2000607211F85C0F4208520062F306000870DC
:103F30000FE02BE00220207207E0697F052801F0E6
:103F40000F0141F0800121721BD0607A20F0030044
:103F50006072A088FDF766FA05460078212825D012
:103F6000232800D0FFDFA87F00F00300012810D035
:103F70000021A08809F073FD22212846FDF78AFA66
:103F800014E0607A20F00300401CE1E7A8F800602C
:103F900011E00121EDE70CB16888A080287E03289C
:103FA0002BD004280AD005284BD0FFDFA8F80060EA
:103FB0000CB1278066800020BDE8F09F15270F26F2
:103FC000002CE3D0A088FDF72DFA807F00F00300DD
:103FD000012806D00021A08809F02FFD050003D19B
:103FE00001E00121F7E7FFDFD5F821000622514665
:103FF00007F045FB84F80EB0D8E717270926002CF8
:10400000C4D0A088FDF70EFA8146807F00F003003F
:10401000012806D00021A08809F00FFD050003D17A
:1040200001E00121F7E7FFDFA878800701D5022032
:1040300000E00120207299F800002328B6D927213A
:104040004AE719270E26002CA0D0A088FDF7EAF930
:104050005FEA000900D1FFDFC4F808B0A4F80CB093
:1040600084F808B0A07A40F00300A07299F81F10FD
:1040700061F38200A07299F81F1001EA510161F307
:10408000C300A072687E00F0030001288ED1607A20
:1040900040F00400607299F81E0000F0030001284F
:1040A00014D0E97E607B61F300006073AA7E217BFF
:1040B00062F300012173EA7E520862F341006073EB
:1040C000A87E400860F3410121736FE7E87E217B01
:1040D00060F300012173AA7E607B62F300006073CD
:1040E000EA7E520862F341012173A97E490861F317
:1040F000410060735AE730B504468079012591B0DC
:10410000B5EB901F00D0FFDFFFF72CF84FF6FF70E4
:10411000099074488DF8015020300190201D0290C4
:10412000601C0B900AA968460BF0BBF800B1FFDFDA
:104130000B980188A4F801108078E07011B030BDB0
:1041400010B5684C30B10146102204F1200016F081
:1041500071FE012084F8300010BD10B50446FFF751
:1041600001F8604920461022BDE81040203116F0C9
:1041700061BE70B55B4C06004FF0000514D00DF029
:104180001BFC08B110250DE00621304607F05EFA51
:10419000411C06D0206614F85C0F40F080002070AF
:1041A00000E00725284670BD14F85C0F20F0800061
:1041B000F5E72DE9F041804688B00D460027084616
:1041C0000DF045FCA8B94046FDF72CF9040003D0DA
:1041D0002078222815D104E043F2020008B0BDE89F
:1041E000F08145B9A07F010603D500F00300022845
:1041F00001D01020F2E7A07FC10601D4010702D54B
:104200000DB10820EAE7374991F85C10C90701D0E1
:104210001120E3E7E17FC90601D50D20DEE700F0BC
:104220000300022805D125B12846FEF7F1FE07005C
:10423000D4D1A07F00F00300012806D00021404621
:1042400009F0FBFB060002D00CE00121F7E7A07F9C
:1042500000F0030001280BD00021404609F0E4FBE8
:10426000060007D0A07F00F00300022804D009E078
:104270000121F2E70420B1E725B12A463146204664
:10428000FEF7EAFE07AB1A4669463046FFF71CF810
:10429000009800B9FFDF00990D20487006F5907076
:1042A000C1F82480486100200881A07F00F003004D
:1042B00001282BD0F5B302200871301D8861707879
:1042C00040090877B078C0F340004877287800F0BC
:1042D0000102887F62F301008877E27F62F3820047
:1042E000887701E05C020020E27F520862F3C3009D
:1042F0008877B27862F304108877A878C87701F1DC
:10430000210228462031FEF7C7FE22E00120087175
:10431000287800F00102087E62F3010008762A780E
:10432000520862F3820008762A78920862F3C3008A
:10433000087600E009E02A78D20862F304100876D3
:1043400024212046FDF7A6F80BE003200871052084
:10435000087625212046FDF79DF8A07F20F08000FB
:10436000A07701A900980AF09CFF022801D000B1B3
:10437000FFDF384632E72DE9FF4FF94A0D4699B085
:104380009A4607CA14AB002783E807001998FDF77F
:1043900049F8060006D03078262806D008201DB03F
:1043A000BDE8F08F43F20200F9E7B07F00F00309A7
:1043B000B9F1010F03D0B9F1020F07D008E03DB900
:1043C0001B98FEF725FE0028E9D101E01B9878BB79
:1043D000B07F00F00300012806D00021199809F0F1
:1043E0002CFB040003D101E00121F7E7FFDF852D5D
:1043F00025D007DCD5B1812D1BD0822D1BD0832D7C
:1044000008D11AE0862D1CD0882D1CD0892D1CD0F7
:104410008A2D1CD00F2020710F281AD001208DF872
:104420003400201D0E902079A8B158E10020F2E759
:104430000FE00120EFE70220EDE70320EBE7052086
:10444000E9E70620E7E70820E5E70920E3E70A2097
:10445000E1E70720A3E7B9F1010F17D0D4E919501C
:1044600080460220019001200090A87898F8021060
:10447000C0F3C000C1F3C00108405FEA000B5DD08B
:1044800050460DF099FA00286CD12DE0D4E9198539
:104490000120019002200090214630461B9AFEF731
:1044A000DBFD1B98007800F00101A87861F30100A2
:1044B000A870F17F61F38200A870F17F490861F371
:1044C000C300A870A17861F30410A8706078400957
:1044D0002870A078C0F3400068701B988078E8705E
:1044E000002068712871C0E7DAF80C000DF064FA5A
:1044F000C0BBDAF81C000DF05FFA98BBDAF80C00CC
:10450000A060DAF81C00E06098F80100A17800F0E3
:10451000010041EA4000A07098F80210C0B2C1F357
:104520000011891E0840A070002084F82000009926
:1045300006F1170002290BD001210AE098F80110BA
:10454000A07801F00101FD2242EA41010840E2E7C2
:10455000002104EB810188610199701C022902D0BD
:10456000012101E028E0002104EB81018861A878A5
:1045700000F00300012849D198F8020000F0030080
:10458000012843D1B9F1010F04D12A1D691D1B98DF
:10459000FEF782FD297998F8040001408DF82C106F
:1045A000687998F8052010408DF8300001432DD02F
:1045B00050460DF001FA08B11020F0E60AF11000A3
:1045C00004F5D47104F17C020490B9F1020F3CD0DF
:1045D0000090CDE9012100210BAB5A462046FEF7A1
:1045E000D5FD0028E9D104F5D67104F19402B9F1A2
:1045F000010F30D004980090CDE9012100210CABCF
:104600005A462046FEF7C2FD0028D6D1A078800782
:1046100040D4A87898F80210C0F38000C1F380015C
:10462000084337D0297898F8000014AAB9F1010F8F
:1046300017D032F810204B00DA4012F0030718D0E0
:10464000012F1ED0022F12D11DE0CDF800A0CDE920
:1046500001210121C0E7CDF800A0CDE90121012110
:10466000CDE732F811204300DA4002F00307032FB0
:1046700007D0BBF1000F0DD0012906D0042904D0CA
:1046800008E00227F5E70127F3E7012801D0042815
:1046900000D10427F07F40F001006BF34100F07778
:1046A000A07881074FF003000CD5A071BBF1000F7B
:1046B00015D100BF8DF85C0017AA31461998FEF796
:1046C00034FD0CE00221022F18D0012F18D0042F46
:1046D00022D00020A071F07F20F00100F07725218A
:1046E0003046FCF7D7FE0DA904F590700AF0B9FD2D
:1046F00010B1022800D0FFDF002050E6A171D9E7F9
:10470000A1710D2104F1240016F02DFC607840F019
:10471000020060700420CDE70120A071DFE72DE9E1
:10472000F04387B0914688460446FCF77BFE0700BD
:1047300006D03878272806D0082007B0BDE8F083D7
:1047400043F20200F9E7B87F00F00300012809D026
:104750000021204609F071F9040006D104E00000B0
:1047600008B301000121F4E7FFDFA679012E08D08C
:10477000B8F1000F0FD048460DF01EF9B8B1102067
:10478000DBE7B9F1000F25D1B8F1000F09D0B8F17E
:10479000010F1FD120E0022E05D0032E05D0FFDF30
:1047A00028E00C2526E0012524E0022522E0B8F1CE
:1047B000020F03D0B8F1010F0AD00BE0032E09D18C
:1047C00000251022494604F1210016F033FB11E0C8
:1047D000022E01D00720B0E70025102104F12100AE
:1047E00016F09FFB5FEA090004D0062106F02EFFB9
:1047F000C4F82100607840F002006070C10713D057
:1048000020F00100607002208DF8000004F121000A
:1048100002908DF804506946FF300AF022FD02280C
:1048200004D018B1FFDF01E084F82050252138467C
:10483000FCF730FE002080E730B587B00D46044617
:10484000FCF7F0FD88B1807F00F0030001280FD055
:104850000021204609F0F1F804000ED028460DF0A2
:10486000ABF838B1102007B030BD43F20200FAE7D0
:104870000121EEE76078400701D40820F3E72946DC
:1048800004F141002022054616F0D4FA607840F089
:104890001000607001070FD520F008006070142030
:1048A0008DF80000694604F5907001950AF0D9FC76
:1048B000022801D000B1FFDF0020D4E770B594B02A
:1048C0000D460646FCF7AEFD18B10178272944D104
:1048D00003E043F2020014B070BD807F00F00300DB
:1048E000012806D00021304609F0A7F8040003D1C2
:1048F00001E00121F7E7FFDFA07902282DD1A078A0
:10490000C0072AD0002302220321304603F050FCC6
:1049100028B30D208DF80D0007A80222811FADF8E5
:10492000142006ABCDE900310C9604F5907402908A
:10493000089400230321304603F0B7FC00B1FFDFE9
:1049400004208DF810008DF824500DA903A80AF05A
:10495000A8FC00B1FFDF0020BDE70820BBE7112065
:10496000B9E770B5064686B014460D4608460DF008
:1049700023F818B920460DF043F810B1102006B006
:1049800070BDA6F57F40FF380DD03046FCF74AFDDC
:1049900030B14378811C22461846FCF7E9FE07E057
:1049A00043F20200EBE72046FDF7F3FC0028E6D1D6
:1049B0001021E01D0CF0B2FCE21D29466846FEF70E
:1049C0009DFC102204F11700019916F033FA002023
:1049D000D5E72DE9F04104468CB0154688460027FE
:1049E00008460DF034F818B928460DF030F818B123
:1049F00010200CB0BDE8F0812046FCF713FD060046
:104A000003D03078272818D102E043F20200F0E703
:104A1000B07F00F00300012806D00021204609F0F5
:104A20000CF8040003D101E00121F7E7FFDF607813
:104A3000400702D5A078800701D40820D9E7B07FCD
:104A400000F00300012818D0D4E91901407800B122
:104A5000B5B1487810B1B8F1000F11D0C5B1EA1D59
:104A600006A8E168FEF74AFC102205F11700079935
:104A700016F0B4F930B104270AE0D4E91910E5E7DB
:104A80000720B6E71022E91D04F1310016F0D2F933
:104A9000B8F1000F06D0102208F1070104F121003F
:104AA00016F0C8F9607840F002006070C10715D0B8
:104AB00020F00100607002208DF8000004F1210058
:104AC0000290103003908DF804706946EF300AF0C0
:104AD000C8FB022804D018B1FFDF01E084F8207081
:104AE00025213046FCF7D6FC002082E7F8B51546B4
:104AF0000E460746FCF796FC040004D020782228D6
:104B000004D00820F8BD43F20200F8BDA07F00F0F9
:104B10000300022802D043F20500F8BD30460CF035
:104B20004BFF18B928460CF047FF08B11020F8BD1C
:104B300000953288B31C21463846FEF7F7FB112852
:104B400014D00028F3D1297C4A08E17F62F30001E8
:104B5000E1772A7C62F34101E177297C890884F8B6
:104B60002010A17F21F08001A177F8BDA17F090766
:104B7000FBD4D6F80200C4F83600D6F80600C4F814
:104B80003A003088A0861022294604F1230016F04E
:104B900051F9287C4108E07F61F38200E077297CAD
:104BA00061F3C300E077287C800884F82100A07FAF
:104BB00040F00800A0770020D3E770B594B00D4610
:104BC00006460BB1072086E6FCF72CFC040007D054
:104BD0002078222802D3A07F400604D408207AE659
:104BE00043F2020077E6C5B12D208DF80000ADF844
:104BF00002601022294601A816F01CF9287C410801
:104C0000E07F61F30000E077297C61F34100E07709
:104C1000287C800884F8200004E02E208DF8000015
:104C2000ADF8026009A9684606F0C3FCA17F21F037
:104C30004001A1774FE670B50D46FCF7F3FB040089
:104C400005D028460CF0DCFE20B1102070BD43F2E8
:104C5000020070BD29462046FEF707FB002070BD0C
:104C600005E000BF10F8012B0AB100207047491E73
:104C700089B2F7D20120704770B50D4600780499CB
:104C80001446042803D0052832D0FFDF70BDA88B5E
:104C90000E2200EB400002EB400018803320088019
:104CA000002CF3D0A88BA081002613E0A87F012858
:104CB00014D006EBC60005EB400106EB460204EB00
:104CC0004202088CD0811020223110320AF08AFB77
:104CD000761CB6B2A089B042E8D870BD05EB86015B
:104CE00006EB460204EB4202088CD0810220EBE77F
:104CF000A88B102200EBC00002EB4000188034208B
:104D00000880A87F012808D0022806D0FFDF002CE9
:104D1000E3D0A88BA081002613E0A073F7E7A87F5B
:104D2000012812D006EBC60005EB400104EB400061
:104D30000A8C028210221230223116F07BF8761C87
:104D4000B6B2A089B042EAD870BD05EB860106EB89
:104D5000C602088C04EB4202223110820220123279
:104D60000AF040FBEBE72DE9F04105780E20DDF875
:104D700018C001F1200402F10E074FF00008022DC7
:104D800006D0032D2DD0062D6AD0FFDFBDE8F081BF
:104D9000CD8B05EB850600EB460018803120ACF882
:104DA0000000002AF2D0087F9581801FC6B214E06F
:104DB00061682088388031F8020BF88031F8020BE6
:104DC0003881BA1C30460AF00DFB06B118B187F8DD
:104DD0000480A7F8028008340A376D1EADB2E7D20E
:104DE000D4E7CD8B05EB850600EB4600188032201A
:104DF000ACF80000002AC9D0087F9581401FC6B2D8
:104E00002AE06168228811F8010BFA803A79430898
:104E100060F3000263F34102830863F38202C30874
:104E200063F3C302030963F30412430963F34512F6
:104E3000830963F386123A71C009787131F8020B65
:104E400038813A4630460AF0CDFA18B187F8028028
:104E5000A7F8008008340A376D1EADB2D1D295E7AD
:104E6000087FCD8B801E86B206F1080068431030A3
:104E700018803520ACF80000002A87D0958102F117
:104E80001007D68107EBC5080BE020883880C7F8EB
:104E9000048032464046616815F0CCFF0834B044C7
:104EA00008376D1EADB2F0D270E72DE9F0471D4610
:104EB000089E0C4681462AB1607E00F58070D08045
:104EC000E08B108199F800000E274FF000084FF09A
:104ED000100A0C287ED2DFE800F096061521293151
:104EE0003F4E636B6B6B207F9146082802D00328EE
:104EF00000D0FFDF2F8030200BE000BFA9F80C802E
:104F0000BDE8F087207F9146042800D0FFDF2F8086
:104F100031203080B9F1000FF0D1F1E7207F9146C8
:104F2000042800D0FFDF2F803220F2E7207F914657
:104F3000022800D0FFDF2F803320EAE7207F1746CA
:104F4000022800D0FFDF3420A5F800A03080002F19
:104F5000D6D0A7F80C80D3E7207F1746042800D0CE
:104F6000FFDF3520A5F800A03080002FC8D04046D4
:104F7000A7F80C8012E0207F1746052802D00628EB
:104F800000D0FFDF1220288036203080002FB7D0DD
:104F9000E08BB881A7F81080B9F80200F881AFE77C
:104FA000207F9146072800D0FFDF2F803720B0E711
:104FB0004FF0140018804FF03800170030809FD059
:104FC000E08BB881A7F8128099F80000092807D073
:104FD0000A2800E017E009D00B280DD0FFDF8FE78B
:104FE000207F0C2800D0FFDF01200AE0207F0D2861
:104FF00000D0FFDF042004E0207F0E2800D0FFDF78
:105000000520B8737CE7FFDF7AE770B50C460546EC
:10501000FCF708FA20B10078222804D2082070BDDD
:1050200043F2020070BD0521284608F006FD20600D
:1050300008B1002070BD032070BDFFB585B00746E4
:105040001720ADF80C00089814460D46022628B922
:1050500008A93846FFF7D9FF00283ED15DB10023EB
:10506000BDF80C203146384603F0A2F8B8B30898D2
:105070000078A0BB05E02078092822D00F282FD087
:10508000FFDF002004A9CDE9001003460290BDF81F
:105090000C203146384603F008F900281DD1089845
:1050A00003A9801DC4E901072046049A04F017FBF8
:1050B00060B3072828D2DFE800F01E1C2727252030
:1050C000220007260023BDF80C203146384603F0A5
:1050D0006FF80028D5D143F2040009B0F0BD08E014
:1050E0000023BDF80C203146384603F061F8002853
:1050F000C7D11120F1E70020EFE70820EDE743F2E8
:105100000300EAE70720E8E70320E6E704980090B9
:10511000BDF80C3004223146384603F048FA002826
:10512000DBD1002DD9D008990D70D6E710B588B025
:105130001C46AAB104238DF800301388ADF80C305A
:105140005288ADF80E208A788DF812200988ADF8C3
:10515000101000236A462146FFF76FFF08B010BD0C
:105160001020FBE72DE9F041074600780C46122895
:1051700039D2DFE800F0383434141036090909094F
:10518000090909090909090904B9FFDF607840F034
:105190000800607028E0002CF8D1FFDFF6E7B8883F
:1051A000052186B2304608F048FC054604B1FFDF11
:1051B00005B9FFDF3146A81D04F08AFA02F0EEFAC5
:1051C000040007D0607840F008006070668002F04C
:1051D000C3FA0AE013213046FDF704FB16E0FFDFB7
:1051E00002E0FFDF00E0FFDF84B1607800070DD54B
:1051F0002078582220F00F00C01C20F0F0009030E2
:105200002070394604F1180015F059FE0020BDE564
:1052100000200870881D04F058BA0A460146901D07
:1052200004F05CBA70B50546052108F006FC0400E0
:1052300000D1FFDF2946A01DBDE8704004F048BA48
:105240002DE9FE4F4FF00009ADF80890ADF804903D
:1052500047880C46054693460521384608F0EDFB85
:10526000060000D1FFDF24B1A780A4F80690A4F8BF
:105270000890297E04F112003827C91E4FF001085A
:105280004FF0360A00900F2970D2DFE801F0F9FAEA
:105290006F6108AD6A70812CB6C9E59595003078CC
:1052A000012800D0FFDFA88B0E2101EBC001ADF873
:1052B00004103021ADF80810002C13D0A08100207C
:1052C0000DE004EBC00132790A747288CA8105EBE3
:1052D0008002401CD38B4B82128C8A8280B2A189BF
:1052E0008142EED8E8E03078012800D0FFDFE88B7B
:1052F0000E2101EBC001ADF804103021ADF808100B
:10530000297F091FC9B20091002CEBD0A081002792
:105310001AE000BF05EBC70A04EBC70808F10E024C
:10532000DAF8241000980AF05DF818B188F81090A7
:10533000A8F80E90BAF82010A8F81210BAF82210A7
:105340007F1CA8F81410BFB2A089B842E2D8B3E01D
:1053500002A8009001AB224629463046FFF78CFC9C
:10536000AAE03078072806D0FFDF04E0A3E0307819
:10537000072800D0FFDFE88BADF808A01230ADF8A9
:105380000400002C38D0A98BA1817188E18123E031
:105390003078082800D0FFDFA88B00F10E01ADF8AF
:1053A00004103721ADF80810002C25D0A081AA8B5D
:1053B00004F10E00296A4CE0E88B123080B23921EA
:1053C000ADF80400ADF80810F4B3A98BA181287ED4
:1053D000102807D00221A173E98B2182EA8B296A68
:1053E000009836E00121F6E702A8009001AB2246C2
:1053F00029463046FFF7B7FC5EE03078092800D038
:10540000FFDF1420ADF80400ADF808701CB3A98BC1
:10541000A181A4F81290A4F8109084F80E804BE0BB
:1054200030780A2800D0FFDF288CADF808701430DF
:10543000ADF804007CB10421A173A98BA181E98B93
:105440002182298C618200E032E02A8C04F1140070
:10545000696A15F0EFFC2FE030780B2800D0FFDFF1
:105460001420ADF80400ADF8087004B30521A17351
:10547000A4F80C90A4F81090A4F812901CE000E09E
:1054800008E002A8009001AB224629463046FFF70B
:105490000CFD11E00D203A21ADF80400ADF8081024
:1054A00034B1A4F80680A4F8089084F80C9003E0C6
:1054B000ABF8000014E0FFDFBDF80400ABF800001B
:1054C00074B1BDF808002080BDF804006080287E1B
:1054D000032805D0102803D0112801D086F80090A9
:1054E0000020BDE8FE8F2DE9F84356880F46804620
:1054F00015460521304608F0A0FA040000D1FFDF70
:10550000A41D33462A4639464046009404F064FA06
:10551000BDE8F8832DE9F0438DB00D461446814671
:1055200007A9FFF772FD002814D14FF6FF76012777
:105530004FF420588CB103208DF800001020ADF8F6
:10554000140008A802460690204605A909F069FF44
:1055500078B107200DB0BDE8F0830820ADF80C50FD
:105560008DF812708DF80000ADF80E60ADF8108067
:105570000CE00798A1780171218841808DF81270A4
:10558000ADF80C50ADF81080ADF80E606A46012100
:105590004846079BFFF751FDDCE708B501228DF86F
:1055A000022042F60202ADF800200A4602236946B4
:1055B000FFF7BCFD08BD08B501228DF8022042F6B8
:1055C0000302ADF800200A4603236946FFF7AEFD4B
:1055D00008BD00B587B079B102228DF800200A8895
:1055E000ADF80C204988ADF80E1000236A4604215E
:1055F000FFF723FD07B000BD1020FBE709B106232C
:1056000094E50720704770B588B00D4614460646ED
:1056100007A9FFF7FAFC00280ED17CB10620ADF8EF
:105620000C508DF80000ADF80E40079B6A4607212C
:105630005C803046FFF701FD08B070BD05208DF895
:105640000000ADF80C50F0E700B587B059B1072362
:105650008DF80030ADF80C20049100236A46082133
:10566000FFF7EBFCC6E71020C4E770B5002488B054
:10567000172391B10A78062A20D2DFE802F01F042E
:10568000041503171523DB1E9DB2CB880BB18E6862
:105690001EB1AB4203D90C20CEE71020CCE7042A80
:1056A00004D08B8853B901E00620C5E7012A13D046
:1056B000022A05D0042A1CD0052A2AD00720BBE7DD
:1056C00009228DF800204A88ADF80C20CA88ADF870
:1056D0000E208968049123E00C228DF800204A886E
:1056E000ADF80C20CA88ADF80E2089680924049111
:1056F00016E00D228DF800204A88ADF80C208A882B
:10570000ADF80E20CA88ADF8102089680A240591EA
:1057100006E00E228DF8002049788DF80C100B243D
:1057200000236A462146FFF788FC85E700B587B06D
:105730000F228DF80020ADF80C1000236A461946A0
:10574000FFF77BFC56E700B587B071B102228DF8F8
:1057500000200A88ADF80C204988ADF80E1000230F
:105760006A460521FFF769FC44E7102042E7000084
:1057700018B1817801293CD101E0102070470188DF
:1057800042F60213C81A4FF48072994233D01CDCDF
:1057900042F60103A1EB030099422CD00CDCF9B1D5
:1057A000B1F5C05F27D06FF4C050081823D0A0F522
:1057B0007060FF381DD11EE001281CD002281AD0CD
:1057C000FF2818D0904214D115E0904213D008DC85
:1057D000012810D002280ED0FE280CD0FF2808D1B6
:1057E00009E0A0F58070013805D0012803D0022817
:1057F00001D0002070470F2070470B2826D008DC0E
:105800001BD2DFE800F01C2025251A252923252797
:105810001E0011281CD008DC0C2817D00D281DD024
:105820000F2815D0102808D110E0822809D084282C
:1058300010D0852810D0872812D003207047002070
:1058400070470520704743F20300704707207047F8
:105850000F20704704207047062070470C207047C7
:105860004FF45050704707280DD2DFE800F00406CF
:10587000040C0C080A000020704711207047072014
:1058800070470820704703207047007810F00F021F
:1058900004D0012A05D0022A0CD110E0000909D158
:1058A0000AE00009012807D0022805D0032803D008
:1058B000042801D007207047087000207047062098
:1058C000704705282AD2DFE800F003070F171F00F2
:1058D000087820F0FF001EE0087820F00F00401C40
:1058E00020F0F000103016E0087820F00F00401C87
:1058F00020F0F00020300EE0087820F00F00401C6F
:1059000020F0F000303006E0087820F00F00401C56
:1059100020F0F000403008700020704707207047EA
:1059200038B50C46050041D06946FFF7AEFF0028A8
:1059300019D19DF80010607861F30200607069462B
:10594000681CFFF7A2FF00280DD19DF800106078B9
:1059500061F3C5006070A978C1F34101012903D04A
:10596000022905D0072038BD217821F0200102E06E
:10597000217841F020012170410704D0A978C9089D
:1059800061F386106070607810F0380F07D0A97846
:10599000090961F3C710607010F0380F02D1607808
:1059A000400603D5207840F040002070002038BD2C
:1059B00070B504460020088015466068FFF7B0FF08
:1059C000002816D12089A189884211D86068807882
:1059D000C0070AD0B1F5007F0AD840F20120B1FB20
:1059E000F0F200FB1210288007E0B1F5FF7F01D92B
:1059F0000C2070BD01F201212980002070BD10B57E
:105A00000478137864F3000313700478640864F373
:105A1000410313700478A40864F3820313700478BC
:105A2000E40864F3C30313700478240964F30413D3
:105A300013700478640964F34513137000788009C7
:105A400060F38613137031B10878C10701D1800764
:105A500001D5012000E0002060F3C713137010BDD2
:105A60004278530702D002F0070306E012F0380F25
:105A700002D0C2F3C20300E001234A7863F30202BA
:105A80004A70407810F0380F02D0C0F3C20005E031
:105A9000430702D000F0070000E0012060F3C502D8
:105AA0004A7070472DE9F04792B00D00804613D040
:105AB000B8F1000F14D01221284615F032FA03AACB
:105AC000FF21012005F0D3FB0024264637464FF482
:105AD00020596FF4205A6DE0102012B0BDE8F08715
:105AE0000720FAE79DF8160001280AD1BDF8140036
:105AF00048450BD010EB0A000AD001280CD0022830
:105B00000CD0042C0ED0052C0FD10DE0012400E0A8
:105B10000224BDF8126008E0032406E00424BDF866
:105B2000127002E0052400E00624BDF81210414581
:105B300040D12C7486B34FF007090DF134080EAA3A
:105B4000CDF80090CDE9012810230022FF21304636
:105B500005F029FCF0B9BDF834002A46C0B20EA900
:105B600009F040FCB0B9AE81B7B108AECDF80090F5
:105B7000CDE9016813230022FF21384605F013FC0C
:105B800040B9BDF83400F11CC01EC0B22A1D09F096
:105B900029FC10B10320A0E70AE0BDF82100E8814C
:105BA000062C05D19DF81600A872BDF814002881B6
:105BB000002092E703A805F062FB002892D0FFF7CF
:105BC0001CFE8AE72DE9F0438BB00E46DDE9129802
:105BD00005461C461746142103A815F0C4F90120F8
:105BE0008DF810008DF80C008DF81180ADF8147050
:105BF00064B1A178C90709D08DF81600E088ADF826
:105C00001A00A088ADF81800A068079001F0C6FD42
:105C1000040025D06580002009A9CDE900101722D5
:105C2000034601460290ADF82020284602F03DFBD5
:105C3000002812D108368DE8700008AA494603A84A
:105C4000099B04F042FE06466078000701D501F08A
:105C500083FD5EB13046FFF706FE0BB0BDE8F08372
:105C600013212846FCF7BEFD0320F6E709980090B3
:105C7000BDF8203004220021284602F098FCECE711
:105C800070B506468AB000200D46059007240490A2
:105C9000069003A900940790CDE901010246102364
:105CA0002946304605F07FFB68B904A9009108A891
:105CB000CDE90140BDF80C3000222946304605F000
:105CC00081F9002801D0FFF798FD0AB070BD05F0FA
:105CD0003CB82DE9FC470546002700780C46B8463D
:105CE000B9460C2873D2DFE800F0B8060D2FCE5F5E
:105CF0005F7F96B49AA504B1FFDF288980B201F0D6
:105D0000BFFEABE0A888042180B2814607F095FE73
:105D1000064604B1FFDF06B9FFDF494606F1080079
:105D200004F03CFA01F03AFD040008D0607840F03D
:105D300008006070A4F8029001F00EFD8FE01321BE
:105D40004846FCF74FFD9EE004B9FFDF6088042160
:105D500007F073FE060000D1FFDFA6F800900020D8
:105D600029791EE005EBC0029268D3B25FEA037C9A
:105D700007D5DB0605D505EBC10030F8020C3080F5
:105D800007E0120A52060AD5307105EBC000C08840
:105D900070806078022740F0080060705EE0401C70
:105DA000C0B28142DED859E0E888ADF8000004B9FD
:105DB000FFDF9DF80100000604D52878062807D0EB
:105DC00005282AD0607840F00800607046E044E082
:105DD0006088042107F031FE060000D1FFDF86F85D
:105DE0000490A888708018E004B9FFDF608804215F
:105DF00007F023FE060000D1FFDF06F1080004F0E3
:105E0000F8FF90F0010F02D1E879000626D56088EE
:105E10000227F080D6E704B9FFDF0227D2E704B9F2
:105E2000FFDF022761880122204601F06DFE4FF05E
:105E30000108C7E7A88986B204B1FFDF686800904F
:105E40002889ADF8040001226946304601F077FE4A
:105E500004E0002CB6D1FFDFB4E7FFDF9CB160782F
:105E6000000710D5B8F1000F0DD12078582220F08E
:105E70000F00001D20F0F00080302070294604F152
:105E8000180015F01CF83846BDE8FC873EB50C003C
:105E900008D06B4601AA002105F0F2FA20B1FFF705
:105EA000ACFC3EBD10203EBD00202080A0709DF8BF
:105EB000050002A900F00700FFF703FD50B99DF8A7
:105EC000080020709DF8050002A9C0F3C200FFF78A
:105ED000F8FC08B103203EBD9DF8080060709DF8F5
:105EE0000500C109A07861F30410A0709DF80510A9
:105EF000890961F3C300A0709DF80410890601D5DB
:105F0000022100E0012161F342009DF8001061F3DD
:105F10000000A07000203EBD70B5144606460D4638
:105F200051EA040005D075B108460BF087FD78B939
:105F300001E0072070BD2946304605F0FCFA10B19B
:105F4000BDE8704059E454B120460BF077FD08B12C
:105F5000102070BD21463046BDE8704096E7002015
:105F600070BD2DE9FE4F05460C46007E0A310091BA
:105F700004F108010027029190460C31821E3E4632
:105F8000BB464FF0010A0191082A7CD2DFE802F0FB
:105F9000F7047B32327EBCF86888042107F04DFD9F
:105FA0005FEA000900D1FFDFB9F8000010B1522705
:105FB0000726ECE051271026002C7CD06888A080B2
:105FC00084F806A099F80400002205EBC0000099AF
:105FD000C08BFFF7A1FF00286ED199F8040005EBF4
:105FE000C000C08B208199F8040005EBC000408CF4
:105FF000E081E6E0B5F82290062822D1E87F00068D
:106000001FD5512709F1140086B2002CD5D0A88BDA
:1060100000220099FFF780FF002873D16888A080D4
:106020000220A071A88B208184F80EA0288C2082E9
:10603000A4F812904A46696ADDF8040014F0FAFEEA
:10604000BFE0502709F1120086B2002C33D0A88B94
:1060500000220299FFF760FF002853D16888A080D2
:10606000A88BE080287E06280ED002202073288C82
:10607000E081E87F4A46C0096073A4F8109004F1FB
:106080001200696ADAE79BE00120EFE768880421E3
:1060900007F0D3FCB5F822A05FEA000900D1FFDFCA
:1060A00009F1080004F0A5FE90F0010F02D1E87F8D
:1060B000000626D501E076E024E00AF1140051271D
:1060C00086B2002C70D06888A080A88B002200992E
:1060D000FFF722FF002815D10220A071A88B208194
:1060E0000420A073288C2082A4F812A05246696A6A
:1060F000019814F09FFE89F804B0A98BA9F802104A
:106100005FE00320BDE8FE8F6888FBF78BF98246CD
:106110006888042107F091FC8146BAF1000F00D194
:10612000FFDFB9F1000F00D1FFDFB9F80600A0F5DD
:106130007F41FF3902D05127142601E05027122653
:106140008CB36888A080502F06D00220A071287FD1
:10615000029901F016F934E0287FA11D01F011F930
:106160009AF82210CDE9001BB9F8022068880023B4
:106170004946FFF727FD0028C4D122E000E016E0E1
:10618000FE49A88BC988814205D15427062654B1FF
:106190006888A08015E05327082624B16888A0806D
:1061A000A88BE0800DE0FFE7A8F800600EE055271F
:1061B0000726002CF8D0A88BA08084F806B000E059
:1061C000FFDFA8F800600CB127806680002099E707
:1061D000EA4900200870704730B587B00C4607F0D8
:1061E000F5FB0546FF2800D1FFDF0020208020714D
:1061F00060804FF6FF70E080294604F1080003F04C
:10620000BFFF02AA2946012005F031F81AE000BFBD
:106210009DF80B00000715D5BDF80E002946FFF7C5
:106220002FFD9DF80B00FF2340F010008DF80B00B0
:10623000BDF80B00ADF80400BDF80E002946019A28
:1062400005F047F902A805F01AF80028E0D007B0D9
:1062500030BD0A46014602F1080003F0A5BF70B543
:106260000546042107F0E9FB040000D1FFDF2946C1
:1062700004F10800BDE8704003F090BF2DE9F04143
:106280008AB00D468046FBF7CDF8060006D0307880
:10629000222806D208200AB0BDE8F08143F20200AD
:1062A000F9E70421404607F0C8FB07460DB1A8886E
:1062B00078B101208DF8140002208DF81800002418
:1062C0008DF819403DB1A888ADF8200028680790E6
:1062D00004E00920DFE7ADF82040079401F05EFA02
:1062E000050026D0A5F8028004A8CDE900041722F5
:1062F0000023ADF80C2019464046029401F0D5FF6A
:106300000028C8D107F108000095CDE9018096F872
:10631000221003AA05A8049B04F0D7FA0446687863
:10632000000701D501F018FA4CB12046FFF79BFA9F
:10633000B1E713214046FCF755FA0320ABE7049878
:106340000090BDF80C3004220021404602F02FF9E5
:106350004FF6FF71F9809EE72DE9FF5F83460E9EA1
:106360009846914677888A463846FBF75BF805469B
:106370000421384607F061FB044605B9FFDF04B984
:10638000FFDF0834CDE90274CDE9008695F82210CC
:106390004B465246584603F037FF04B0BDE8F09F25
:1063A0002DE9F04F99B004464FF000087348ADF85E
:1063B0004C80ADF82480ADF84880A0F80480ADF89A
:1063C0000C80ADF81080ADF81880ADF8148000781E
:1063D00016460D464746012809D0022807D0032853
:1063E00005D0042803D0082019B0BDE8F08F20465E
:1063F0000BF0E2FAD0BB28460BF0DEFAB0BB6068C7
:106400000BF025FB90BB606848B160892189884208
:1064100002D8B1F5007F01D90C20E5E7804608AA33
:1064200004A92846FFF7C4FA0028DDD168688078FF
:10643000C0F34100022808D19DF8110010F0380F78
:1064400003D028690BF0FAFA80B903A92069FFF795
:1064500067FA0028C8D1206950B1607880079DF89C
:106460000D0000F0380002D5E8B301E011E0D0BB28
:106470009DF80C0080060ED59DF80D0010F0380F29
:1064800003D060680BF0DAFA18B960680BF0DFFA35
:1064900008B11020A8E705A96069FFF741FA0028B4
:1064A000A2D1606940B19DF8150000F007010129F3
:1064B0003BD110F0380F38D006A9A069FFF730FAA9
:1064C000002891D19DF8140080062ED49DF8180064
:1064D00080062AD4A06950B19DF8190000F0070188
:1064E000012922D100E020E010F0380F1DD0E06833
:1064F00018B10078C8B11C2817D20CAA611C20461C
:10650000FFF77DFA0120B94660F30F27BA46074628
:106510008DF8460042F60300ADF844000DF1330259
:1065200015A9286808F07DFF08B107205CE79DF8F1
:10653000540014A9CDF80090C01CCDE9019100F0E1
:10654000FF0B00230BF20122514611A804F0D7FDE6
:10655000E8BBBDF850000B9008492A892869091D3D
:106560000092CDE901016B89BDF8202028680499CB
:1065700004F0C5FD01007CD1207801E05803002023
:10658000C1064FF0020A01D480062BD5ADF81C904D
:10659000606950B905A904A8FFF762FA9DF81500D3
:1065A00020F00700401C8DF815009DF814008DF8B0
:1065B000467040F0C8008DF8140042F60210ADF8A5
:1065C000440009A907AA0023CDF800A000E01CE0C0
:1065D000CDE9012140F2032211A8059904F08FFDB5
:1065E000010046D1F8484D464FF007098088ADF8C4
:1065F00031000CA9CDE900195B4600220295FF216C
:10660000BDF8500004F0DEFC10B1FFF7F6F8EBE641
:106610009DF83000000625D52946012060F30F21A2
:106620008DF846704FF42450ADF84400ADF8285072
:1066300062789DF82800002362F300008DF828009E
:106640006278520862F341008DF828000AAACDF85A
:1066500000A0CDE9012540F2032211A804F04FFD6E
:10666000010006D1606850B3206970B903A904A87D
:1066700000E07DE0FFF7F4F96078800705D49DF82D
:106680000D0020F038008DF80D008DF8467042F6B0
:106690000110ADF84400208940F20121B0FBF1F275
:1066A00001FB1202606812ABCDF80080CDE9010356
:1066B000002311A8039904F022FD010058D120788D
:1066C000C00729D0ADF81C50A06950B906A904A88C
:1066D000FFF7C6F99DF8190020F00700401C8DF85F
:1066E00019009DF818008DF8467040F040008DF8B4
:1066F000180042F60310ADF8440013A907AACDF81C
:1067000000A0CDE90121002340F2032211A806993F
:1067100004F0F5FC01002BD1E06868B329460120A4
:1067200060F30F218DF8467042F60410ADF8440076
:10673000E068002302788DF8582040788DF85900E1
:10674000E06816AA4088ADF85A00E06800798DF834
:106750005C00E068C088ADF85D00CDF80090CDE940
:1067600001254FF4027211A804F0C9FC010003D006
:106770000B9800F019FE37E693480321017056B1DB
:1067800080883080BDF848007080BDF82400B0805B
:10679000BDF84C00F080002026E670B501258AB0D7
:1067A00016460B46012802D0022816D104E08DF8C7
:1067B0000E504FF4205003E08DF80E5042F60100C9
:1067C000ADF80C0063B10024601C60F30F2404AA30
:1067D00008A9184608F025FE20B107200AB070BDB0
:1067E0001020FBE704A99DF820207748CDE900217F
:1067F000801C02900023214603A802F2012204F02B
:106800007EFC10B1FEF7F9FFE8E76F480EB1418852
:10681000318005700020E1E770B594B00446012690
:106820008DF83E6041F60100ADF83C0012AA0FA9B8
:106830003046FFF7B2FF002848D12078624CC007ED
:106840004FF0000544D01C2102A814F08CFB9DF8E9
:1068500008008DF83E6040F020008DF8080042F6F8
:106860000520ADF83C000E959DF83A00119520F0FA
:106870000600801C8DF83A009DF838006A4620F02A
:10688000FF008DF838009DF8390009A920F0FF00BD
:106890008DF839000420ADF82C00ADF830000EA8BA
:1068A0000A9011A80D900FA80990ADF82E5002A8DB
:1068B000FFF776FD002809D1BDF80000E080BDF8A3
:1068C00004002081401C60812570002014B070BD40
:1068D000E5802581BDF84800F4E72DE9F74F8B46A8
:1068E000394900269EB00A78012A04D0022A02D033
:1068F000082021B079E54A88824201D00620F8E7D5
:1069000089465A4501D10720F3E701214FF00008DD
:106910008DF86610ADF8401042464FF6FF71531CDB
:1069200063F30F220492ADF84210ADF84A10FF2035
:1069300042F6020A8DF86A801AAA8DF84800ADF86E
:1069400064A0ADF868801192CDF84C8010A804F0D6
:10695000BDFC0024254627460BAA072110A804F0F9
:10696000B8FC78B1822857D184B37DB3ADF85C40D0
:106970009DF85600ADF85E508DF80C8017AC0128DC
:106980005ED065E09DF832000FB3012853D1BDF809
:10699000301051451DD116AA07A907208DE8070020
:1069A000BDF82E0010230022FF2104F0FCFC98BB50
:1069B000BDF85800042801D0062847D1BDF81C10A6
:1069C000594538D10F2094E75803002036E00128BC
:1069D00031D1BDF83000B0F5205F03D042F601019F
:1069E000884228D1B9F80210BDF82E00814201D1A9
:1069F000012700E0002704B17DB158451BD116AB3B
:106A000007AA07218DE80E00044610230022FF216B
:106A100004F0C9FC00B902E02DE035460BE0BDF8FA
:106A20005800022801D0102810D1C0B215AA07A919
:106A300008F0D8FC50B9BDF82E608DE7052058E766
:106A400003A915A8221D08F0ECFC08B1032050E7AB
:106A50009DF80C000023001DC2B220988DF80C2078
:106A60000092CDE9014019A8049904F048FB10B93F
:106A7000022289F80020FEF7C0FE3AE710B50B4667
:106A8000401E86B084B203AA00211846FEF7B7FF65
:106A900004AA072103A88DE8070001230022FF2193
:106AA000204604F08FFA0446BDF81000012800D0FB
:106AB000FFDF2046FEF7A1FE06B010BDF0B5FC4F8B
:106AC000044687B038780E46032804D0042802D044
:106AD000082007B0F0BD04AA03A92046FEF768FF0E
:106AE0000500F6D160688078C0F3410002280AD121
:106AF0009DF80D0010F0380F05D020690AF09EFFB8
:106B000008B11020E5E7208905AA21698DE8070072
:106B10006389BDF810202068039904F0F0FA10B1E1
:106B2000FEF76BFED5E716B1BDF8140030800420E7
:106B300038702846CDE738B50C00054609D000234B
:106B40006A46FF2104F09CFC28B100BFFEF755FE09
:106B500038BD102038BD69462046FEF7E1FE00280A
:106B6000F8D1A078FF2100F001032846009A04F034
:106B7000B0FCEBE77FB5144603AA07250292CDE9E6
:106B800000350A462388FF2104F01CFABDF80C10DA
:106B90002180FEF732FE04B070BD2DE9F04192B0C5
:106BA0004FF000050C000746ADF8105019D0E06812
:106BB00028B1A068A8B10188ADF81010058038464A
:106BC000FAF730FC88B1007822286AD3384606F0FC
:106BD000FDFE80460421384606F02FFF060008D14E
:106BE00006E0102012B0BDE8F08143F20200F9E7A0
:106BF000FFDFA078012803D0022801D00720F1E7A9
:106C0000208838B1401C80B206AA414604F02FFB10
:106C100038BB02E043F20300E4E706A804F02FFBD0
:106C20009DF822204FF45051012A09D1BDF82020AF
:106C3000A2F52453023B03D1822801D088B901E098
:106C40000846CFE7E06898B1072204A9CDE9000221
:106C50000291A2882088BDF81030FF2104F0B2F91B
:106C600010B1FEF7CAFDBDE7A168BDF810000880AD
:106C70009DF81B00C00602D543F20140B2E70A9816
:106C800018B1BDF82400022801D00320AAE717227A
:106C90000A98ADF80C20A1780078012903D080076C
:106CA00010D408209EE7C007FBD0002307213846F8
:106CB00001F07EFA18B14FF00708022005E043F218
:106CC00004008FE74FF0010803208DF83000208882
:106CD000ADF834000BA8CDE9000500230295BDF8FE
:106CE0000C204146384601F0E0FA002887D1CDE972
:106CF00000570836029603AA07210CA80B9B03F045
:106D0000E4FD10B1FEF7AFFD6CE70B980090BDF805
:106D10000C3004224146384601F049FC62E770B568
:106D2000064615460C460846FEF722FD002805D10A
:106D30002A4621463046BDE870402EE570BDCCE5C0
:106D400070B51E4614460D0009D044B1616831B1DA
:106D500038B157494988814203D0072070BD1020BF
:106D600070BD2068FEF704FD0028F9D132462146A7
:106D70002846BDE87040FFF713BB70B515460C0000
:106D800006D038B14A498988814203D0072070BDB6
:106D9000102070BD2068FEF7EBFC0028F9D12946D1
:106DA0002046BDE8704089E670B5054686B00E46BF
:106DB000144610460AF024FEF0BB60680AF047FE55
:106DC000D0BBA5F57F40FF3803D02846FAF72AFB51
:106DD000A0B1284606F0FAFD054630466946FEF7A2
:106DE00061FE00280CD19DF810100F20082936D222
:106DF000DFE801F008060606060A0A0843F2020068
:106E000006B070BD0320FBE79DF80210012908D1F0
:106E1000BDF80010B1F5C05FF2D06FF4C052D1429E
:106E2000EED09DF80610012905D1BDF80410A1F59A
:106E300028510529E4D900E022E09DF80A10012933
:106E40000ED1BDF80810B1F5245FD9D0A1F52451B9
:106E50000239D5D00129D3D0022901D1D0E7FFDFF3
:106E6000606878B9002305AA2946304604F008FB7B
:106E700010B1FEF7C2FCC3E79DF81400800601D4F0
:106E80001020BDE76188224630466368FFF772FE36
:106E9000B6E72DE9F043074685B08946144610460B
:106EA0000AF0AEFD30B1102005B0BDE8F08300005F
:106EB00058030020384606F089FD4FF6FF76054658
:106EC000B74201D0FF2D0AD00146002304AA48464C
:106ED00004F0D6FA30B100BFFEF78FFCE4E743F2CE
:106EE0000200E1E79DF81000C00602D543F2014020
:106EF000DAE74FF0070803A90027CDF80080CDE9B5
:106F00000171628833462946484604F04CFA06006F
:106F100012D160680AF074FD58B96068CDF800803D
:106F2000CDE90107238862882946484604F03BFAE8
:106F30000646BDF80C0020803046CDE739B1FD4B48
:106F40000A881B899A4202D843F20300704724E65C
:106F500010B586B0F74C0423ADF81430E3883BB18C
:106F600024898C4201D2914204D943F20300A3E563
:106F70000620A1E5ADF81010002100910191ADF8B7
:106F8000003002218DF8021005A9029104A9039195
:106F9000ADF812206946FFF700FE8DE52DE9FC47AC
:106FA00081460F4608460AF007FDD0BB4846FAF76F
:106FB00039FA5FEA000811D098F80000222832D38D
:106FC000002317221946484601F0F2F850B1042177
:106FD000484606F032FD060007D105E043F2020004
:106FE000BDE8FC871120FBE7FFDF06F1080003F096
:106FF000F1F805463878012803D0022804D007208C
:10700000EEE7A8070FD502E015F0340F0BD0B879E2
:107010003C1DC00709D0E08838B1A0680AF0CCFC5C
:1070200018B11020DCE70820DAE73A782088002140
:1070300028B3A0F201130721112B18D20CD2DFE8DC
:1070400003F00B090D0B1D0B121D100B0B1D1D1D4D
:107050001D0B1D00022A11D10846C1E7012AFBD0F1
:107060000CE0EA0600E0AA06002AF5DA06E0A0F540
:10707000C0721F2A02D97D3A022AEDD8C1B298F80F
:107080002200CDE900017288234631464846FEF7CA
:1070900099FDA5E72DE9FF4F89B01E4615460C4620
:1070A0004FF000080F460998FAF7BCF930B10078A4
:1070B000222806D208200DB0BDE8F08F43F202006E
:1070C000F9E7B00801D00720F5E7032E00D100262C
:1070D000099806F07BFC83464FF6FF7ACCB1022D6F
:1070E0006AD320460AF0B3FC30B904EB0509A9F1D4
:1070F00001000AF0ACFC08B11020DCE7AD1EAAB21A
:107100002146504604F0CCFA39F8021C884253D18B
:10711000ADB28848B10702D50189491C00E00121C0
:107120001FFA81F9F10701D0068900E0564603AA4B
:107130005946484604F09BF84FF0070A0BE0788860
:10714000102839D808F1040108441FFA80F8A8452E
:1071500032D804EB08078FB339884945EFD34DE0A7
:107160009DF80F100A0749D54CB304EB080908F144
:107170000402B9F8023097B2102B1DD8DA19AA42CE
:107180001AD8B9F80020904216D1C80618D5E119CE
:10719000CDE9001A08AA0292B9F800000022594667
:1071A00003F010FF10B1FEF728FB84E7B9F80200E6
:1071B000BDF82010884203D00B207CE71EE005E0DC
:1071C000B9F8020038441FFA80F806E0C90604D571
:1071D0005946FEF755FD00288FD19DF80F00FF237B
:1071E00020F010008DF80F00BDF80F00ADF8000082
:1071F000BDF812005946009A04F06BF903A804F098
:107200003EF818B9BDF81200B042A9D90421099876
:1072100006F013FC040000D1FFDF22885AB10025DC
:10722000CDE900A52B4621460998FEF7CBFC0028A6
:10723000BBD125803FE700203DE72DE9F04F89B025
:107240001E4617000D464FF000041BD0B10802D0B7
:10725000072009B030E7032E00D1002606F0B6FB68
:107260008046FF2805D07DB128460AF0E7FB48B9E3
:1072700002E043F20200ECE73988681E08440AF095
:10728000DDFB08B11020E4E72A49B00701D54889A1
:1072900000E00120F2074FF6FF7902D04989491E2C
:1072A00000E049468EB204AA414603F0E0FF4FF0E9
:1072B000070A0DF10C0B33E09DF8131009072FD5C9
:1072C0000023CDE900A3CDF808B04B46002241468B
:1072D00004F069F8E8B9F5B1BDF80C103A8821441A
:1072E0002819091D8A4231D3BDF8162020F8022B37
:1072F000BDF80C2020F8022BCDE900A0CDF808B095
:10730000BDF81600BDF80C300022414604F04BF8E1
:1073100008B103209DE7BDF80C002044001D84B295
:1073200004A803F0ACFF38B1822809D0FEF765FA53
:107330008FE7000058030020BDF81600B042BBD90B
:1073400034B175B13988A01C814203D20C2080E78A
:1073500005207EE722462946484604F0A1F929196E
:107360000880A41C3C80002073E710B504460AF096
:1073700047FB08B1102010BD114840892080002033
:1073800010BD70B50C4605460E21204613F0C9FD10
:10739000002020802DB1012D01D0FFDF70BD06201F
:1073A00000E00520A07170BD10B50C4603F02EFF63
:1073B00000B1FFDF2046BDE81040FEF71EBA000016
:1073C000580300204FF0E0224FF400410020C2F8A3
:1073D000801120490870204990020860704730B53C
:1073E0001C4D04462878A04218BF002C02D000286B
:1073F00018BFFFDF2878A04208BF30BD2C701749A6
:10740000154A0020ECB1164DDFF858C0131F012CAF
:107410000DD0022C1CBFFFDF30BD086003200860C8
:10742000CCF800504FF400001060186030BD0860C8
:1074300002200860CCF800504FF0407010601860D7
:1074400030BD086008604FF06070106030BD00B55E
:10745000FFDF00BD1600002008F5014000F50040E8
:107460006403002014F5004010B50446007894B081
:10747000022805D0012803D043F2050014B010BD46
:10748000A07828B1032803D8607808B1032801D96F
:107490000720F3E73F208DF800002078022801D074
:1074A000012000E000208DF80200607800F095FDDA
:1074B000C01D8DF80300A078012800D1022000F043
:1074C0008CFD8DF80400607800F087FD8DF80500D4
:1074D000A07800F082FD8DF806002078012804D104
:1074E0009DF80300401C8DF8030009A9684604F0CC
:1074F00060F800B1FFDF0020C0E72DE9FF4F8DB03D
:10750000FA49DDE91AB90600D1E902010396CDE98D
:107510000901507A117A9A4608441546C7B20DD02F
:107520000024F01D20F00700B04200D0FFDF2888C3
:107530000399401C1FFA80F814B107E00124F0E71A
:1075400008F0FF0007F0F4FE00B1FFDF03993A46B0
:1075500001EB0810C01C20F00301D5F81080039146
:107560003CB9002008701FFA88F003F0F2FC00B16B
:10757000FFDF0399234601EB08000390A87A297ADC
:107580003A460844C1B203A800F071FD0398C01C3C
:1075900020F003000390697A00912B7AAA7A04B153
:1075A000002001A906F025F900B1FFDFBDF80410A5
:1075B0000398CDE900B90844C01C20F003001C99D1
:1075C000CDE902103A4604B10020534605A906F061
:1075D0009BFA00B1FFDFBDF8141003980844C01DEA
:1075E00020F007000E99821B03900A60002C35D111
:1075F000C04ABF491160111D401E086001232C22A2
:107600000BA9BD4806F076F800F0F1FC00211E221F
:10761000084602F053F8FAF72FFE00F034FFFEF7A9
:10762000D7FD09AB00220521B4A0FBF7ECFA00B1AD
:10763000FFDF05F10C00FFF7EFF800B1FFDF4FF4BB
:107640007F71B04813F08FFCAE48012180F8F91328
:10765000022180F8FA13062180F8FB1311B0BDE86F
:10766000F08F10B5A74CA078092800D3FFDF207851
:10767000C0EBC00004EB001010F8041F21F0FF0164
:107680000170417821F00701C91C21F018014170F7
:107690000121E17010BD2DE9F04105460C4600279F
:1076A0000078052190463E46B1EB101F00D0FFDF69
:1076B000287E58B1012810D0FFDF00BFA8F8006075
:1076C0000CB1278066800020BDE8F08102270926E2
:1076D0007CB1A88BA080A87F09E00327142644B1C1
:1076E0006888A080286AE060A88C2082287F2072A9
:1076F000E4E7A8F80060E6E700B5017895B001F08E
:1077000001018DF80210417801F001018DF803109C
:107710000178C1F340018DF804104178C1F34001B4
:107720008DF80510017889088DF8061041788908D0
:107730008DF8071081788DF80810C1788DF8091040
:1077400000798DF80A003E208DF8000009A96846EE
:1077500003F02FFF15B000BD70B56A4CE07800282B
:107760001BD020780025C0EBC00004EB001040794E
:1077700000F00700011991F8F803401E81F8F803A2
:107780002078401CC0B22070092800D12570A07854
:10779000401CA07009F0B1FCE57070BD594890F82C
:1077A000FB03002800D05CE770472DE9F043554DFE
:1077B0009BB00026D5F8F40368B1FFF7EFFF00286F
:1077C00075D07022D5F8F41313F079FBFFF7C4FFDE
:1077D000C5F8F463EEE795F8F903002867D0FFF7E2
:1077E00040FF0446444805F0B6FF606000B9FFDF83
:1077F000606803F029FF88B12046FAF7B8F860788E
:10780000010706D520F00700401C6070FFF7A4FFB9
:10781000D0E73948616805F0A7FFCBE736486168D3
:1078200005F0A2FF01A800F05BFC00286CD1032149
:10783000BDF8040006F001F98046BDF8040006F02A
:1078400062FA0746B8F1000F00D1FFDFD8F8040054
:1078500010B10078FF2857D0FFF703FF04463846E1
:10786000211D05F0B0FE00B9FFDFD4F8049089F8BF
:107870000060BDF804006080204600F0EAFE384653
:1078800005F0CDFE00B9FFDF3B208DF81000BDF8FC
:107890000400ADF8120004A805F050FB0EA804F097
:1078A0003CF96078010703D4C00607D409E02BE057
:1078B00020F00700801C6070FFF74EFFC8F80490AE
:1078C00078E7D8F8040038B10178491C11F0FF01BD
:1078D00001709DD1FFDF6DE700221146384600F0B0
:1078E0007AFB002894D1FFDF64E7000014B30100A5
:1078F0000000002000060240B40700206E5246350A
:1079000078000000B80300201BB0BDE8F08310B57C
:10791000FC4CA0600868E060AFF2711001F031FE2D
:10792000607010BDF74900200870704730B50546FB
:107930004FF080500C46D0F8A41095B0491C05D1EA
:10794000D0F8A810C9430904090C08D050F8A01FAA
:1079500001F0010129704168216080680EE02B2050
:107960008DF8000009A9684603F023FE00B1FFDF8F
:10797000012028700A982060BDF82C00A08028788B
:10798000002803D0607940F0C000607115B030BDB0
:10799000F0B54FF080540746D4F8800095B00D46FE
:1079A0002B26401C0BD1D4F88400401C07D1D4F8FE
:1079B0008800401C03D1D4F88C00401C0BD0D4F8B4
:1079C00080003860D4F884007860D4F88800B8600B
:1079D000D4F88C0016E08DF82C6069460BA803F0F3
:1079E000E8FD00B1FFDF01983860029878608DF8FB
:1079F0002C6069460BA803F0DCFD00B1FFDF0198A5
:107A0000B8600298F860D4F89000401C0BD1D4F80C
:107A10009400401C07D1D4F89800401C03D1D4F83E
:107A20009C00401C08D054F8900F28606068686083
:107A3000A068A860E06816E08DF8006009A96846B3
:107A400003F0B7FD00B1FFDF0A9828600B9868606B
:107A50008DF8006009A9684603F0ABFD00B1FFDFB7
:107A60000A98A8600B98E86015B0F0BD30B5A64C38
:107A70000546D4F8F40300B1FFDFC4F8F45330BD79
:107A80003EB50546032105F0D8FF0446284606F01A
:107A90003AF9054604B9FFDF606818B10078FF289D
:107AA00000D1FFDF01AA6946284600F094FA60B9C8
:107AB000FFDF0AE0002202A9284600F08CFA00B994
:107AC000FFDF9DF8080000B1FFDF9DF80000411EB8
:107AD0008DF80010EED260680199884201D1002033
:107AE0006060894C94F8FA03022800D3FFDF94F811
:107AF000FA03401CC0B284F8FA03012803D181487C
:107B0000407801F05DFD3EBD70B50446A1F57F40B3
:107B100016460D46FF3800D1FFDF012E01D0FFDFF2
:107B200070BD207820F00F00401D20F0F000503094
:107B3000207000202076A5830120A07770BD70B54D
:107B400015460C460646FFF729FE90B1017821F054
:107B50000F01491D21F0F0015031017046800121D3
:107B6000017621680162A18881840577BDE87040B3
:107B7000F2E53046BDE870401321FAF733BE70B528
:107B800005460C46084609F03BFF08B1102070BDC1
:107B90002846F9F747FC28B1284600F09DFE2070E2
:107BA000002070BD43F2020070BD2DE9F04F87B098
:107BB00005460020059053488946017811B10820F8
:107BC00007B04CE54F4851494160284609F018FF7D
:107BD000002868D1484609F013FF002863D16F7A66
:107BE0002B7AF818FF2870D82888FE286DD800B99D
:107BF0000A202880296909B94FF4B06129616A68AF
:107C0000B2B15478907804EB440420441478167987
:107C100004EB440400EB44005479D27804EB4404B0
:107C200006EB4606344402EB420204EB420406E053
:107C300007EB470003EB430200EB42042046C7EB8F
:107C4000C7021044C3EBC3021044184486B206EBCB
:107C5000C60000EB400A04EBC40000EB40000090BB
:107C6000D82901D20920ABE7A87AB8422DD84FF025
:107C70001208082F0DD8012B0BD807F0C4FC0746BB
:107C800009F0FAF93A1A297A687A521E0B189A42C0
:107C900001DA404694E76F6883468846BFB13846AC
:107CA00009F0D5FE08B110208AE7B9787878014448
:107CB00038780A180BEB0800904206D179793A79A6
:107CC0001144FA781144884201D0072078E70098DF
:107CD0001FFA8AF387B20097CDE901642A4603A907
:107CE0000020FFF70AFCDFF81C800399D9F8002078
:107CF000D8F80400014491420AD90420C9F80010C0
:107D00005EE7000018000020B80300208812002061
:107D10000097CDE901641FFA8AF32A4604A9FFF708
:107D2000ECFBDDE90301884200D0FFDF0498D8F8BE
:107D300004100844C8F80400C9F80000FF490120F5
:107D400088F80000087005983AE72DE9F0470746E3
:107D50000C46084609F054FE40B9384609F06EFE5C
:107D600020B9F81C20F00300B84202D01020BDE872
:107D7000F087F3484FF00008817899B14178824646
:107D8000C1EBC10100EB0115B4F8009015F8040F28
:107D9000234600F00F000022294600F0F0F906000B
:107DA00004D013E0A4F800800520E0E797B1218813
:107DB000494501D90C260DE02878234600F00F0034
:107DC0003A46294600F0DBF9060005D00C2E01D01A
:107DD000A4F800803046CAE79AF801005446401CD7
:107DE000C0B28AF80100092801D184F80180A07886
:107DF000401EA070687800F0070101290BD002290D
:107E000003D0032918D0FFDFE4E7C006E2D4688876
:107E1000FFF736FEDEE7CB48696805F0A5FC94F86D
:107E2000F903401CC0B284F8F9030128D2D1C64836
:107E3000407801F0C5FBCDE794F8FB03401C8AF8BD
:107E4000FB03C7E770B50D46044609F0B5FD18B948
:107E5000284609F0D5FD08B1102070BD29462046FE
:107E6000BDE8704007F09BBA70B5044615460E4653
:107E7000084609F0A1FD18B9284609F0C1FD08B16E
:107E8000102070BD022C03D0102C01D0092070BD31
:107E90002A463146204607F0A5FA0028F7D00520EB
:107EA00070BD70B514460D46064609F085FD38B91B
:107EB000284609F0A5FD18B9204609F0BFFD08B114
:107EC000102070BD22462946304607F0AAFA002845
:107ED000F7D0072070BD10B594B0044609F090FDAE
:107EE00010B1102014B010BD0F208DF8000009A9AA
:107EF000684603F05EFB0028F4D19DF82C0020704A
:107F0000BDF82E006080BDF83000A0800020E9E7B9
:107F100070B505460C46084609F090FD20B93CB105
:107F2000206809F06DFD08B1102070BDA08828B14F
:107F300021462846BDE87040FEF7A0B9092070BD73
:107F400070B504460D46084609F036FD30B9601E8E
:107F50001E2814D8284609F02FFD08B1102070BD46
:107F6000022C01D9072070BD04B9FFDF774800EB70
:107F7000840050F8041C2846BDE870400847A4F16E
:107F800020001F28EED829462046BDE87040FAF7A9
:107F9000BCB870B504460D46084609F031FD30B94D
:107FA000601E1E280DD8284609F006FD08B11020D5
:107FB00070BD012C01D0022C01D1062070BD07201C
:107FC00070BDA4F120001F28F9D829462046BDE83D
:107FD0007040FAF709B905F099B9032803D00228CF
:107FE00003D001207047062070470320704710B56A
:107FF00094B003F0CFFA54484178806803F0C0FC95
:10800000514801240C300178012916D130218DF816
:108010000010C0788DF8020010B1012803D005E0EF
:108020008DF8024002E000208DF80200684604F05E
:1080300085FF10B109A803F070FD02208DF824001F
:108040008DF825008DF8260009A8FFF70DFA00B17C
:10805000FFDF8DF8244003208DF825008DF82600E1
:1080600009A8FFF701FA002800D0FFDF3AE72DE961
:10807000F0410646022012B101EB4200401DC7B29A
:108080003068C01C20F0030232601BBB2C483B460A
:108090000A21283809F081FB002408E00A2C11D2BB
:1080A000DFE804F005070509090B0B05050528485D
:1080B00004E0284802E0284800E0284809F08CFB4A
:1080C000054600E0FFDFA54200D0FFDF641CE4B2FC
:1080D0000A2CE3D3306800EB07103060BDE8F08174
:1080E0002DE9F04395B081463A208DF82C00694681
:1080F0000BA803F05EFA00B1FFDF43F20406002490
:108100006D46DFF83C8032E02F19B87DC10706D0FC
:10811000400704D405EB4400C08800F0CEFB98F87B
:10812000FA0310B3B87D80071FD505EB4400C08863
:1081300000F055FAC8B105EB440011E0080000203A
:10814000B8030020B40700201800002014B3010079
:10815000391F0000F7840000E12F0000E9F0000063
:10816000C188A9F80010002605E0641CE4B29DF85F
:108170000400A042C8D815B03046BDE8F0832DE910
:10818000F041044600201880601E1D4616460F462A
:10819000052800D3FFDF05482A4600EB840031465E
:1081A00050F8043C3846BDE8F041184724B30100BC
:1081B0002DE9F0478A46984615460646032105F004
:1081C0003CFC0446304605F0B0FD0C35AFB200254E
:1081D00081462E4604B9FFDFB9F1000F00D1FFDF61
:1081E00004EB8A000189B94200D30125218CB942F0
:1081F00002D2BAF1060F00D3012638EA050104D0F5
:10820000817A41F0020181720BE038EA060108D060
:10821000817A41F00401817214F8220F40F00400C9
:10822000207005EA0600BDE8F0872DE9F047824698
:10823000DDE90854174605F10C0099460E461FFA71
:1082400080F800232A4639465046FFF7B1FF60B157
:10825000B07800061BD424F8045C24F8029C504635
:1082600005F063FD040008D106E0072F01D01120BE
:10827000D9E743F20400D6E7FFDF2D1D2046A9B25F
:1082800004F047FF00B9FFDF504603F0E5FA06EBC4
:108290008700062F0289A2EB0801018103D2318CED
:1082A000A1EB080030840020BDE72DE9F04385B044
:1082B0001E46DDE90D5491460F46DDF8308005F08D
:1082C00034FD60B309F10402694692B204F0BBFECA
:1082D00050B300980770BDF80800042800D2FFDFF3
:1082E000002701983A46394607808770019803F0C5
:1082F00075FB1EB1BDF80800001F3080B8F1000FFB
:1083000003D00198C01DC8F8000015B1BDF81000D9
:1083100028808CB1288870B1039820600CE043F26B
:10832000020005B0BDE8F083072F01D01120F8E767
:1083300043F20400F5E727600020F2E72DE9F04F53
:108340000F46054687B016465088032105F075FB99
:10835000040000D1FFDF4FF000098DF80C90A078E9
:10836000400600D1FFDF042F53D3297841F30000EA
:10837000401C06D162786B789A424AD12278120763
:1083800047D04FF0010B4FF00208142939DA4FF6AD
:10839000FF7A012933D0122902D0132931D11CE0F0
:1083A0000C2F2ED1A17801F07F01012929D020784E
:1083B00020F00F00401C2070687860708DF80CB0C1
:1083C000A888ADF80E00E888ADF810002889ADF84F
:1083D00012006889ADF8140016E0062F11D120783C
:1083E00020F00F0020707188012009F0A2FA8DF8AA
:1083F0000C80ADF80EA0A888ADF8100004E0062FA0
:108400000AD09DF80C10B9B17088324603A9F9F76B
:1084100018FE07B0BDE8F08F207820F00F00207024
:108420007188012009F085FA8DF80C80A888ADF8D4
:108430000E00ADF810A0E7E70028EAD0768806A87D
:10844000CDE9000927464C46002306220421304688
:10845000CDF80890FFF729FF00B1FFDF069805234C
:10846000042280F800B069784170A0F8028084800E
:108470000621CDE9001039463046FFF7D6FE002828
:10848000C7D0FFDFC5E70020FE49024621F81020D3
:10849000401C0828FAD3704770B50C46897821F043
:1084A000FF01A170217821F00F012170012161707D
:1084B0000021616005F039FC050000D1FFDF28468E
:1084C00004F0BFFDF53820852046BDE8704000F07F
:1084D00010BB70B50D46032105F0AFFA040000D1C2
:1084E000FFDFA07865F30600A07070BD70470146FD
:1084F000012009F01EBA3EB58DB20321284605F0D1
:108500009CFA040000D1FFDF2078002220F00F0049
:10851000207002208DF800004FF6FF70ADF80200C9
:10852000ADF8040069462846F9F78BFD3EBD2DE9FC
:10853000F04705460C4600784FF0000901219246AD
:108540004F46B1EB101F00D0FFDF287E032809D073
:10855000FFDF00BFAAF8007014B1A4F80090678094
:10856000002060E6AE8B4FF0700906F10A0087B27A
:10857000D4B16888A080688B2081E680A889A9682A
:10858000001F80B28046024604F10A00C91D12F0A5
:1085900051FC4645DED904EB0800A6EB08020A3080
:1085A000296912F047FCD5E7AAF80070D8E72DE951
:1085B000FC410F461C46164680460321089D05F0E7
:1085C0003CFA010008D033463A464046CDE9004522
:1085D000FFF72BFEBDE8FC8143F20200FAE770B51D
:1085E0000546A0F57F4086B0FF3811D0284605F03B
:1085F0008AFB040000D1FFDF2046694604F0E3FF58
:1086000000B9FFDF019CB4F80500E41C052802D086
:10861000012006B070BD2E460321284605F00DFA54
:10862000050000D1FFDF2079122807D120880C280F
:1086300004D1A87800F07F00022806D0002306228B
:1086400004213046FFF7B4FDE3E7002306220521AD
:10865000F7E7F8B5024680689489938A30F8031FDB
:108660001C444588241F8C421ED1042D1DD0052D8D
:1086700029D0062D1ED0402D16D30E46144628466E
:1086800000F0D7F908280FD0207820F00F00401C08
:1086900020F0F00010302070032020766583A68340
:1086A000607840F008006070F8BDBDE8F840001D3B
:1086B00000F0CBB90093548813690A46011D204687
:1086C000FBF7CCF9F8BDBDE8F840001D36E67FB5F4
:1086D0000D460646032105F0B0F904003DD0207890
:1086E00000F00F0001283BD0002003A9CDE90010C5
:1086F000034602900C2205213046FFF7D6FD0028E4
:1087000029D1039812210523017061781A46891C2A
:10871000417008214180298881806988C180A988A9
:108720000181E98841810C21CDE9001021463046C4
:10873000FFF77BFD00B1FFDFF0230022314601206F
:1087400009F05AF8207820F00F00401C2070607863
:10875000801C6070002004B070BD43F20200FAE794
:108760001120F8E77FB50D460646032105F065F9AF
:10877000040006D0207800F00F00012804D0082063
:10878000E9E743F20200E6E7002003A9CDE9001083
:1087900003460290062205213046FFF786FD002899
:1087A000D9D103981321052301706178417002210A
:1087B000418085800621CDE900101A4621463046C9
:1087C000FFF733FD00B1FFDF207820F00F002070AD
:1087D0000020C0E72DE9F84F0F468346032105F03E
:1087E0002CF90546584605F0A0FA80464FF0000ADD
:1087F00005B9FFDFB8F1000F56D1FFDF54E0404666
:108800006946002204F082FD9DF800408146082C54
:1088100000D3FFDF05EB840609F108003189062C3F
:108820000144318102D2298C08442884072C03D1C9
:108830000AF1010000F0FF0AB07AC0070CD021460F
:10884000284600F0DDF838B9B07A032C20F001009A
:10885000B07258462ED0FFDFB07A810706D520F0DF
:108860000200B0722146584600F0DAF8062C1BD8F8
:1088700095F82200410717D520F0040085F8220062
:10888000002401E0E407002005EB8401887A420718
:1088900006D520F0040088722146584600F0C0F842
:1088A000641CE4B2062CECD37F1EFFB2A7D2504664
:1088B000BDE8F88FFBF773F9CEE710B5032105F09B
:1088C000BCF8040000D1FFDF204600F012F9A078C8
:1088D00040F08000A07010BD10B5032105F0ADF888
:1088E000040000D1FFDF208D2321B0FBF1F0C0B2E6
:1088F00010BD70B50D46032105F09FF8040000D1AE
:10890000FFDF062D00D9FFDF2946204600F078F86A
:10891000002805D004EB85018A7A42F001028A72B0
:1089200070BD10B50446402801D2072010BD00F0EC
:1089300080F8082802D04FF4445010BD0021774839
:1089400002E0491C082903D230F81120002AF8D18E
:10895000082903D020F81140002010BD042010BDCC
:1089600010B5402801D2072010BD00F062F8082899
:1089700005D06A4A002122F81010084610BD0520D3
:1089800010BD70B588B015460C00064606D02DB156
:108990006088402804D2072008B070BD1020FBE793
:1089A000218849B300F045F8082827D003AA06A972
:1089B00005A88DE80700228804AB07213046FFF7A1
:1089C00074FC0028E8D1BDF810202946059812F063
:1089D00031FA2088BDF81010884204D9421A29447F
:1089E000039812F027FA05980090238862880721DF
:1089F0003046FFF7DCFDCFE70C20CDE70520CBE7C5
:108A0000072903D0464A32F8112000E0028D00EB1E
:108A100081000089904201D20120704700207047F8
:108A200010B5032901D0FFDF10BDBDE81040FBF7F2
:108A300078B801460020394A02E0401C082803D2D9
:108A400032F810308B42F8D170472DE9F0410F46D3
:108A50008046014686B014463846FCF744FDC0B255
:108A600008283CD10025ADF81450039560880321F7
:108A700004F0E3FF060000D1FFDF00213046FFF7DE
:108A8000BFFF68B91722ADF8142003A8CDE900058F
:108A90000295002360881946FFF707FC00B1FFDF4D
:108AA000009405AA41463846039BFDF755FCC0B229
:108AB00005281CD2DFE800F0031B13161300BDF8D5
:108AC000140000280BD003990423CDE9000160882D
:108AD00000223146FFF7A9FB002800D0FFDF06B0D7
:108AE000BDE8F081607840F010006070F7E7FFDFCC
:108AF000F5E710B504462021083012F034FA084892
:108B0000002100BF30F8112004EB8103491C1A81B9
:108B10000629F7D9208DA08410BD0000E4070020AD
:108B20003CB3010030B44FF0E02001234FF4006C5F
:108B30000021C0F880C11D02C0F880511C06C0F899
:108B40008041E54A82F80014D21E82F80014E34AFC
:108B500082F80014E24A53609360C2F84011C2F8F0
:108B60004411C2F84811C0F880C2C0F88052C0F861
:108B70008042C0F800C1C0F80041136030BC7047AB
:108B800070B401204FF0E023C6024FF0000CC3F890
:108B900080610402C3F880410506C3F88051D04AC1
:108BA00050609060CF4801680029FCD1C2F840C1F4
:108BB000C2F844C1C2F848C1C3F88062C3F8804219
:108BC000C3F8805270BC70474FF0E0204FF4006152
:108BD000C0F88012C910C0F880127047002804BF86
:108BE000C1487047012804BFC0487047022804BF2D
:108BF000BF48704700B5FFDF002000BD08B5B84989
:108C0000002298B101282FD002281CBFFFDF08BD29
:108C10004FF48020C1F80803C1F84803B54802604A
:108C2000C1F84821B2480068009008BD4FF4803078
:108C3000C1F80803C1F84803AF4B1A60C1F84021DE
:108C4000AE4BC1031960AE49C1F808034FF0E023F1
:108C50000012C3F88001AB480260C1F84021C1F89E
:108C60000022A948027008BD4FF40030C1F8080383
:108C7000C1F84803A5480260C1F844219B48006838
:108C8000009008BD70B5DFF858C204260024012505
:108C900058B1012840D002281CBFFFDF70BD9C4A9C
:108CA0004FF48020012B3CD144E0881E20F07F410E
:108CB0004FF48030CCF80803CCF84041CCF84403A2
:108CC000CCF84015012B14BF002101218E4B5970A7
:108CD0008B490D61DFF83CC2CCF800408E4C4FF060
:108CE000020CC4F800C0DFF834C2CCF80060DFF832
:108CF00014C23D32CCF80020C1F800524FF0E02CF5
:108D00008A15CCF88022C1F80403CCF800210804AD
:108D1000834908601D7070BD824A4FF40030012BFA
:108D200008D0CCF80803C2F84041CCF84403C2F89C
:108D3000401570BDC2F84041CCF80403CCF84403A0
:108D4000C2F8401570BD67480068704770B5764836
:108D50000568774975480860614CD4F840010026E1
:108D600001280AD1D4F8080310F4803F05D04FF44D
:108D70008030C4F80803C4F84061D4F844010128E5
:108D80000DD1D4F8080310F4003F08D04FF40030A0
:108D9000C4F80803C4F84461012007F0BEFBD4F80E
:108DA000480101280DD1D4F8080310F4802F08D011
:108DB0004FF48020C4F80803C4F84861022007F08B
:108DC000ACFB5C48056070BD574810B50468584955
:108DD000564808604C490878002808BF03201AD07C
:108DE000464A4FF000401060454AC00BC2F80803E5
:108DF00003124FF0E02C0020CCF88031414B18607A
:108E0000C2F84001C2F8000208704A78002A1CBF6C
:108E10004870002001D007F080FB4648046010BD78
:108E20004FF0E0214FF08070C1F8000270474FF022
:108E3000E0214FF08070C1F8800270474FF0E021D0
:108E40004FF40010C1F8000270474FF0E0214FF4DA
:108E50000010C1F8800270472949012008614FF0D5
:108E6000E0210002C1F880027047410A43F609522E
:108E70005143C0F3080010FB02F000F5807001EBD5
:108E800050207047430B48F2376C03FB0CF31B0C6C
:108E90004FEA432CC1F800C0DFF89CC003FB0C0371
:108EA00026484CF2F72C5843400D10FB0CFC0CEB01
:108EB000432303F580735B1213700A681044086043
:108EC0007047194810B5046819491848086007F038
:108ED00011FC1848046010BD0BE000E018E000E051
:108EE00000B0004004B500404081004044B1004063
:108EF00048B1004048B5004040B5004008F5014089
:108F000000800040408500402800002044B500401B
:108F100008B00040048500400885004010850040EE
:108F200004F5014004B000401005024001000001BA
:108F30001805024014050240F7C2FFFF6F0C010044
:108F400010B5EFF3108000F0010472B6EC484178E0
:108F5000491C41704078012801D108F0EDF8002C3F
:108F600000D162B610BD70B5E54CE07848B9012576
:108F7000E570FFF7E5FF08F0E7F820B1002008F002
:108F8000C3F8002070BD4FF080406571C0F80453F5
:108F9000F7E770B5EFF3108000F0010572B6D84C1A
:108FA000607800B9FFDF6078401E6070607808B9B3
:108FB00008F0C6F8002D00D162B670BDD04810B5DB
:108FC000C17821B100214171C170FFF7E2FF00209B
:108FD00010BD10B5044608F0B7F8C949C978084073
:108FE00000D001202060002010BD2DE9F05FDFF8E7
:108FF00010934278817889F80620002589F80710B7
:10900000064689F8085000782F4620B101280FD075
:1090100002280FD0FFDF08F0A4F898B108F0A8F8F4
:10902000A8420FD1284608F0A7F80028FAD047E058
:109030000125F0E7FFF784FF08F086F80028FBD051
:109040000225E8E701208407E060C4F80471AD4917
:109050000D600107D1F84412AA4AC1F3423124320B
:109060001160A8494FF0020B34310860C4F804B312
:10907000A060DFF894A2DAF80010C94341F30011B0
:1090800001F10108DAF8001041F01001CAF80010EF
:1090900000E020BFD4F804010028FAD0284608F0E8
:1090A0006BF80028FAD0B8F1000F05D1DAF80010FB
:1090B00021F01001CAF80010C4F808B3C4F8047114
:1090C00099F807004C4670B1307860B908F03CF868
:1090D000064608F027FA6FF0004116B1C4E9031004
:1090E00001E0C4E9030115B12771BDE8F09F01203B
:1090F0002071BDE8F05F00F0E1B810B5040000D1C8
:10910000FFDF4FF080414FF0FF30C1F8080300222D
:10911000C1F80021C1F80421C1F80C21C1F81021C7
:1091200008F018F828B176490120C8704878401C2A
:1091300048702046BDE8104057E72DE9F041012571
:10914000AF077D616E4CE079F0B1012803D0217A40
:10915000401E814218DA07F0F7FF064608F0E2F9F0
:10916000E179012902D9217A491C21720EB12169C4
:1091700000E0E168411A022902DA11F1020F0EDC67
:109180000EB1206100E0E060FFF7DAFE07F0DCFFDF
:1091900010B13D61A57000E0257000202072BDE88F
:1091A000F0812DE9F05F5948D0F800B0574A58498E
:1091B000083211608406D4F8080110B14FF001089C
:1091C00001E04FF00008D4F8000100B10120814611
:1091D000D4F8040108B1012600E00026D4F80C01FF
:1091E00000B101208246D4F8100108B1012700E047
:1091F000002748EA090126EA010020EA0A00B843EC
:1092000000D0FFDF0025B8F1000F04D0C4F80851EA
:10921000012007F079FFDFF8E880B9F1000F13D0E3
:10922000C4F8005198F8050020B188F805500020D6
:1092300007F06AFF98F8000030B107F085FF18B119
:10924000012088F8020020610EB1C4F80451BAF17F
:10925000000F0AD0C4F80C5198F80200464600B935
:10926000FFDFB5703570FFF794FE37B1C4F81051C9
:1092700098F8040008B1FFF760FF2449091DC1F800
:1092800000B032E770B51E4DE87808B907F058FF16
:1092900001208407A061A87858B100BFD4F80C0160
:1092A00020B9002007F068FF0028F7D10020C4F89B
:1092B0000C014FF0FF30C4F8080370BD2DE9F041F8
:1092C0001926B507C5F808630124AC610020C5F86C
:1092D0000001C5F80C01C5F8100107F035FF084F73
:1092E00010B1BC702C6100E03C70FFF729FE05490D
:1092F000B87920310860C5F804636C614FE700005D
:109300002C0000201805004010ED00E01005024080
:109310000100000110B50D2000F06FF8C4B26FF02D
:10932000040000F06AF8C0B2844200D0FFDF3A497E
:109330000120086010BD70B50D2000F048F8374CD2
:109340000020C4F800010125C4F804530D2000F0EA
:1093500049F825604FF0E0216014C1F8000170BDAC
:1093600010B50D2000F033F82C4801214160002198
:10937000C0F80011BDE810400D2000F033B82848B7
:1093800010B5046826492748083108602349D1F8F8
:109390000001012804D0FFDF2148001D046010BD3A
:1093A0001D48001D00680022C0B2C1F8002107F06E
:1093B000D4FFF1E710B51948D0F800110029FBD00F
:1093C000FFF7DDFFBDE810400D2000F00BB800F006
:1093D0001F02012191404009800000F1E020C0F807
:1093E0008011704700F01F02012191404009800068
:1093F00000F1E020C0F880127047002806DA00F083
:109400000F0000F1E02090F8140D03E000F1E020DF
:1094100090F800044009704704D5004000D0004097
:10942000100502400100000110B5202000F075F881
:10943000202000F07DF84449202081F800044349B1
:1094400000060860091D42480860F7F75BFF3F49C6
:10945000C83108603F48D0F8041341F00101C0F85A
:109460000413D0F8041341F08071C0F80413364996
:1094700001201C39C1F8000110BD10B5202000F0FA
:109480004CF8324800210160001D01602F4A481E3F
:10949000E83A10602F4AC2F808032C4BC833196011
:1094A000C2F80001C2F860012B490860BDE8104015
:1094B000202000F03DB825492848EC390860704765
:1094C00022492648E8390860704770B51F4A80690C
:1094D000E83A224911601F49D1F800610023204D6C
:1094E0001D4A5C1E1EB1A84206D300210FE0D1F830
:1094F000606186B1A84209D2C1F80031C1F860317B
:109500001460BDE87040202000F012B81168BDE87A
:10951000704011F05ABDFFDF70BD00F01F02012145
:1095200091404009800000F1E020C0F880117047B0
:1095300000F01F02012191404009800000F1E0206D
:10954000C0F880127047000020E000E000060240F2
:1095500084120020000002400004024001000001CB
:1095600000C001004FF0E0214FF00070C1F8800111
:10957000C1F88002384B802283F80024C1F8000132
:10958000704700B502460420344903E001EBC003F4
:109590001B792BB1401EC0B2F8D2FFDFFF2000BD07
:1095A00041F8302001EBC00100224A718A7101228A
:1095B0000A7100BD294A002102EBC0000171704709
:1095C00010B50446042800D3FFDF244800EBC40490
:1095D0002079012800D0FFDF6079A179401CC0B25A
:1095E000814200D060714FF0E0214FF00070C1F86F
:1095F000000210BD2DE9F0411948056818491948C5
:10960000083108601448042690F80004134F4009FC
:10961000154C042818D0FFDF16E0217807EBC100B5
:109620000279012A08D1427983799A4204D0427999
:10963000827157F8310080472078401CC0B22070FA
:10964000042801D300202070761EF6B2E5D204482B
:10965000001D0560BDE8F08119E000E0F40700207E
:109660001005024001000001400000200F4A12686E
:109670000D498A420CD118470C4A12680A4B9A428B
:1096800006D101B507F022FFFFF715FFBDE8014045
:10969000074909680958084706480749054A064B1B
:1096A0007047000000000000BEBAFECA980000200B
:1096B000040000208811002088110020F84B586019
:1096C00019721A80C90011F04EBC00210180704748
:1096D0004FF6FF720280032008F02BB970472DE986
:1096E000F04F0E46017804464FF0010A0AFA01F0E5
:1096F00047F2FF1100EA01086168154697B0088833
:10970000A0F57F42FF3A06D0B8F1000F07D047F22C
:10971000FE12104203D0012017B0BDE8F08F40EADE
:10972000080008804FF00009A5B185F80090237863
:109730000027052003220221DFF864B3102B75D225
:10974000DFE803F0740D131C2F4A515A31A5A1759F
:10975000A9F1F0EF20780B28E9D00420DCE729708C
:10976000A089A5F8010032801DE104212970A1899A
:10977000A5F80110E189A5F8031082E00620287001
:10978000A089A5F80100E089A5F80300208AA5F8C2
:109790000500A28AE81DA16911F04CFBA08AC01D3A
:1097A0006FE0082129702178082901D11021297042
:1097B000A189A5F80110E189A5F8031030806A1D80
:1097C000694604F1100005F02CFE00287ED1308897
:1097D0009DF80010084454E00A202870A089A5F8DC
:1097E00001003280AAE00C212970A189A5F801109E
:1097F000E189A5F80310B7E0A2890AEB420081B223
:109800003088884262D3052960D30E20287000205A
:1098100008E0236905EB400C33F81030401CACF82D
:10982000013080B29042F4D33180BCE0CAE09BF8B2
:1098300009005A46002873D0401E5072227BDBF884
:109840000400236900EBC205AA882868D3F800C089
:109850000244A2F1080042F808CC5A6842608DF830
:1098600000108DF8019028680290A888ADF80400D7
:1098700000216846FBF776FCA5F80490002E01D085
:10988000484630808FE0287840F0800129702878A1
:1098900040F040012970287820F03F0012302870F5
:1098A000A189A5F80110E289E81C216911F0C2FA2A
:1098B000E089C01C3080287841063FD5000672D56B
:1098C0008DF800A08DF80190308800E026E0001DA2
:1098D000ADF804000295E189E81C08440390001DDE
:1098E00004909BF808008DF8140000216846FBF7EF
:1098F00039FC074630880C303080022F01D007B386
:1099000063E09DF81420DBF804109BF808305846FB
:1099100001EBC2019A4201D28A882AB1042754E09D
:1099200030E02BE022E00DE0427A521C8BF8092057
:109930000D6030888880A6F8009046E06168A089B4
:10994000888030E0287820F03F0016302870A08909
:10995000A5F80100E089A5F80300228A681D616965
:1099600011F068FA208A401D3080E7E7287820F05F
:109970003F0018302870207B687055E760680188C8
:10998000090401D4052720E0C088A189884201D0BC
:1099900006271AE01E202870A6F800A0606801883B
:1099A00021F400410180B8F1000F0ED0BBF8000097
:1099B000002283000320A16807F01EFF6168207861
:1099C000887007E0A6F8009003276068018821EA04
:1099D0000801018038469FE62DE9FF4F97B00C46FD
:1099E000249E70B117280CD83288A2F57F43FF3B24
:1099F00007D02278530601D4120604D508201BB0E4
:109A00008BE60720FBE74FF000098DF800908DF8FA
:109A100001902278831E02F03F0CA0F1010A611C24
:109A20004D461FFA8AF702AABCF1200F79D2DFE86F
:109A30000CF089107861786C78AA78CD78F778FC8A
:109A400078F478F378F2787878F178F078EF78EE47
:109A50007889052876D104208DF80000B0788DF83B
:109A600004006088ADF8060020798DF80100607868
:109A700000F03F000C282BD00ADCA0F102000928DE
:109A800060D2DFE800F0145F175F1C5F1F5F2200E9
:109A9000122826D006DC0E281DD01028DAD11DE0B1
:109AA0001408002016281FD01828D3D11FE03078C2
:109AB000800701E030784007002843DA37E130784A
:109AC0000007F9E73078C006F6E730788006F3E75C
:109AD00030784006F0E730780006EDE73088C005C2
:109AE000EAE73088C004E7E730888004E4E730889C
:109AF0004004E1E73178890724D50328AAD105205D
:109B00008DF80000B4F80100D2E031784907F3D5B0
:109B1000062817D3617898B2012903D0022999D178
:109B200002E01FE1022700E0102706218DF8001057
:109B300061788DF80610ADF80490A11C904607F1ED
:109B400002091BE097E000BF31F8022BA0F1020AE6
:109B5000A8F800208B463A4608F1020011F06AF995
:109B600008EB070202F10208BDF80420AAEB070087
:109B7000521C0BEB070180B2ADF804208145E3D9FC
:109B8000002878D1D3E03078000774D507208DF80D
:109B900000001FFA8AF1ADF80490601C0DF1060276
:109BA0000FE000BF30F8023B22F8023B30F8023BE6
:109BB00022F8023B091FBDF8043089B25B1CADF8E6
:109BC00004300429EED2002955D1B0E03178C9061D
:109BD00051D502284FD308208DF80000ADF806902B
:109BE00061789BB28DF80410A01C0CE0078822F865
:109BF000047B871C80C25B1ABDF8067008447F1C7A
:109C00009BB2ADF806709942F0D9A3BB8FE070E02B
:109C100075E065E04FE042E01DE012E005E0FFE79F
:109C20003078800627D5092003E03078400622D519
:109C30000A208DF80000B088ADF80400ADF8067079
:109C400007E03078000616D50B208DF80000ADF83F
:109C5000047002916BE03188C9050CD502287FD3CE
:109C60000C208DF8000099B2ADF8069063788DF85D
:109C70000430A01C10E073E0078822F8027B4788BC
:109C800022F8027B071D80C2C91ABDF8067018446D
:109C90007F1C89B2ADF806708B42EDD993E731880D
:109CA000C9045DD501285BD10D208DF80000B08876
:109CB000ADF804003BE03188890451D505284FD325
:109CC0000E218DF80010B188ADF80410B4F803101F
:109CD000401FADF80800601DADF80610039026E0A7
:109CE000318849043CD501283AD10F208DF8000075
:109CF0001DE03188090433D4B4F80110F180032841
:109D00002ED3217801F03F011B2925D011218DF898
:109D10000010318841F40041A6F80010B4F8011099
:109D2000ADF80410C01EADF80600E01C02902078CB
:109D300000F03F001B2809D01D2807D003201A99E6
:109D400007F0F7FD308800F400403080684619992C
:109D5000FBF708FA284652E610218DF80010DDE7DF
:109D60000725F7E70825F5E700B597B0032806D1E2
:109D70008DF80000019100216846FBF7F3F917B058
:109D800000BD00002DE9FF4F8DB09346DDE91A5666
:109D9000DDF8749004464FF0000A082A06D0E06906
:109DA00001F02CF858B110203070BCE0288809214F
:109DB00040F01000288089F80010022717E0E169C0
:109DC00001208871E2694FF420519180E169887225
:109DD000E06942F601010181E16900208873288869
:109DE00040F020002880112089F8000004273078F6
:109DF00009900A20307004F1180009F102080225C8
:109E00000B9001F063FA002066E000BFBBF1100F79
:109E100006D1022D04D0A8EB0A00BDF80C20428028
:109E2000BDF80E001099884203D9F649097A0E91BF
:109E300004E003D1099909B131701FE0A8F80000CE
:109E40001C980088A0EB0500A0EB070083B2C7F1C7
:109E5000FF00984200D203460E980AAA08EB0701B9
:109E60008DE8070094F82010BDF80E00002201F0E4
:109E70009AFA307030B1C0B2832858D0BDF80E00C5
:109E800020833DE0089828B1DE48006800790A2860
:109E90002BD335E0BDF82800C11901F0FF0A022DCF
:109EA0000ED099F80110514503D1BDF81820824217
:109EB00008D0D4488A4600680178032908D021E0F8
:109EC00089F801A0CF4800680178042906D008E08D
:109ED00000790A2816D20120089006E0BDF80E107D
:109EE000818005EB0A00D04485B203AA0E990B9835
:109EF00001F0EFF920B91C980088401BB84285DAC0
:109F0000022D0BD0BBF1100F04D1A8EB0A01BDF854
:109F10000C0048801C98058000203070B94800680B
:109F20000078032803D0002011B0BDE8F08F022094
:109F3000FAE72DE9F0410546406B1346002758B378
:109F4000491F8EB2698FA1F57F42FF3A05D04218B2
:109F500092881144891D8CB200E00024A1192A8F37
:109F60000831914216D82044B3F8011020F8021BA2
:109F7000B3F8031020F8021B324620F8026B591D7B
:109F800010F058FF6C87696B00202144B61D3144E6
:109F9000088002E0092700E083273846BDE8F08109
:109FA00010B50B88048F9C420CD9446BE0180488D0
:109FB00044B1848824F40044A41D23440B80106021
:109FC000002010BD822010BD2DE9F04788B000258B
:109FD000904689468246ADF81050072745E0039821
:109FE00006888088000440D4A8F8006005A800977F
:109FF000CDE901504FF4007300224946304601F08C
:10A00000D2F9040038D1BDF81000ADF8180003985B
:10A0100004888188B44214D10A0412D4CDE90057CF
:10A0200021F40041029541F480434288494620468C
:10A0300000F0C8FF04000BD10398818841F400416F
:10A04000818003AA06A95046FFF7AAFF0400DED0CC
:10A05000CDE9005703980295BDF81430008800221E
:10A06000494600F0AFFF822C06D103AA04A950464E
:10A07000FFF796FF0400B2D0ADF8105004E003984B
:10A08000818821F40041818003AA04A95046FFF78A
:10A0900087FF0028F3D0822C03D0204608B0BDE80B
:10A0A000F0870020FAE730B50446406B97B00025F2
:10A0B00070B10B208DF80000208FADF80800606BA8
:10A0C0000391019000216846FBF703FE8DF80050D4
:10A0D0004FF6FF7065636087258717B030BD2DE9A7
:10A0E000F041044686B00E46616B00200C9D174679
:10A0F00000292AD0012B28D12A4631462046FFF7D5
:10A1000063FF002821D1002F1FD0A046344600262F
:10A11000ADF8106007270EE00398008828800398A8
:10A120000296811DCDE90017838842880088214668
:10A1300000F048FF30B903AA04A94046FFF730FFFA
:10A140000028E9D0822800D1002006B026E72DE9BA
:10A15000F0411546DDE906644A1D378892B2974200
:10A1600001D206201AE73280172204F8012B0A4692
:10A17000208065801946201D10F05CFE00200DE750
:10A1800000220280C262831D0263C36142634FF6F4
:10A19000FF734387028780F8201070474FF6FF72E5
:10A1A0000280042007F0C5BB30B597B00D460446C9
:10A1B000FFF779FF208E48B101208DF80000E06A9A
:10A1C000CDE9010500216846FBF783FD0020E06230
:10A1D000206382E70146002009880A0700D5012094
:10A1E00011F0F00F01D040F00200CA0501D540F097
:10A1F00004008A0501D540F01000490501D540F062
:10A2000020007047200800202DE9FF4FA7B01F460F
:10A21000349E299D379C5FEA000817D028784106B4
:10A2200010D400F03F011E290AD0218811F4FE6FDE
:10A230000CD13A88172A09D3A1F57F42FF3A05D0FD
:10A24000010606D500F03F00122802D004202BB0F2
:10A250006BE6FE4928984FF0000908728DF81090BF
:10A260008DF834900DAA0A60359A4A60ADF81490C2
:10A27000ADF890902878032200F03F038646711CC9
:10A2800004F1180CCB464FF0040AA8F10500CDF8F4
:10A2900098C01F2B7DD2DFE803F07C7C107C1C7CF7
:10A2A000867CEF7CEE7CED7CEC7CEF7CEB7C7C7C3C
:10A2B000EA7CE97C7C7C7C7CE800B8F1030F02D06E
:10A2C0008DF810A0EFE232701720A6F801003A8056
:10A2D000BEE2B8F1050FF3D1B5F801002083ADF867
:10A2E0001400B5F80310618300287DD088427BD824
:10A2F00084F808B0A4F806B04FF6FF706084269882
:10A3000000F0E4FF05203070B01C00904FF0020A0E
:10A3100008AA2899269800F0DCFF00287ED19DF835
:10A320002600012803D002207070102002E00120D6
:10A33000707002208346002201A909A805F071F877
:10A3400030BB9DF80400834522D13A88801CA2EBE3
:10A350000A0181421CDB0098BDF822100AF1020AB2
:10A360000180009909A8891C0A46009101A905F0FD
:10A3700058F89DF80400009908AA014450441FFAB7
:10A3800080FA00912899269800F0A3FF0028D2D0E7
:10A3900000E069E2BAF1020F40D0A7F800A057E24E
:10A3A0008DF8100054E2B8F1070F89D3B5F8010019
:10A3B0002083ADF81400B5F803106183A0B1884282
:10A3C00012D84FF0010A84F808A0B5F80500E08023
:10A3D00000202073E06900F011FD90B9E16981F877
:10A3E00006A04FF4205100E078E0E26942F6010057
:10A3F0009180E16981F80AA0E1690881E1690020A2
:10A400008873A8F107006084E81D6062269800F058
:10A410005DFF0720307006F1010A00E06FE00020C8
:10A420004FF0010BADF8220018E000BFBBF1010FA7
:10A430000CD0E069807901281FD03AF8021C00BFD7
:10A440000BF102002AF8021B1FFA80FBBDF8221054
:10A450000BF102002AF8021B1FFA80FB08AA2899B8
:10A46000269800F036FF58B10FE0DAE16BE10AE11F
:10A47000AEE0D2E17BE05AE01EE0BDF82010DFE75D
:10A480003988A1EB0B000428D0DABBF1010F36D0DC
:10A49000E069807901280CD0BDF82010A1F57F403B
:10A4A000FF3806D03AF8021CAAF800100BF102009F
:10A4B000B1E1BDF82010F7E7B8F1070F03D0B8F10C
:10A4C000150F7FF4FDAEB5F801102183ADF814101F
:10A4D000B5F80320628309B1914201D901205FE7F9
:10A4E00001212172A4F806B084F80CB0B8F1050F70
:10A4F00007D0C0B2691DE26904F074FF08B10A20F8
:10A500004EE74FF6FF70608404A824A9CDE900103F
:10A51000CDE902762878002300F03F0220462899F2
:10A52000FFF730FC8146208BADF8140090E1B8F1C4
:10A53000030FC6D14020ADF89000B5F8010020838C
:10A54000ADF81400289ACDE900210AAB02933988AE
:10A550000022491E8BB294F8201000F024FF8DF8E1
:10A56000100058BB0B203070BDF828002EE0B8F169
:10A57000050FA6D18020ADF89000B5F8010020832A
:10A58000B5F803206284ADF81400B2F5007F01D95C
:10A59000072005E742F47C426284289BCDE9003124
:10A5A0000DF12C0CCDF808C03988491E8BB294F8F7
:10A5B000201000F0F8FE8DF8100018B18328B5D1F6
:10A5C0000220BEE00D203070BDF82C00401C22E1BE
:10A5D0004FEADE1000EB400002EB8000404505D959
:10A5E0005FEA4E607FF56CAE584614E1B5F801C0E5
:10A5F000ADF814C02978490608D505218DF8341026
:10A600002978090605D58DF834B031E106218DF899
:10A610003410E91C289BA8EB000ACDE90013CDF803
:10A6200008B009911FFA8AF394F8201000226046BE
:10A6300000F0C8FC8DF810008DF834B02978490678
:10A6400010D52088C00509D5208B01E02008002006
:10A65000BDF81410884201D1C4F824B058468DF8D2
:10A6600010B0D8E0832801D14FF002094FF4807078
:10A67000ADF89000BDF814002083A4F822A009983A
:10A6800060621320C5E0B8F1050FFFF419AEB5F80C
:10A6900001C0ADF814C0218F41B3A1F57F42FE3A4D
:10A6A00024D007218DF83410289A6B1DCDE9003293
:10A6B00080B2CDF808B040F40043DA46B5F8032084
:10A6C00094F82010604600F07DFC4FF400718DF886
:10A6D00010008DF834A0ADF89010832810D0E8B1A8
:10A6E000218FA1F57F40FE3807D0DCE00A218DF8EC
:10A6F00034104FF6FE712187D6E7A4F838A0A7E002
:10A700002A4641462046FFF714FC8DF8100008B198
:10A71000832848D1BDF81400208351E72A464146DA
:10A720002046FFF706FC8DF81000E0BB618F606BE0
:10A73000CDE9007643185A88998833F8060BFFF75D
:10A7400006FD814684E095F801A0B8F1020F7CD1A6
:10A750005FEA0A0002D0BAF1010F76D108208DF825
:10A76000340005A800908DF838A094F820105346C6
:10A7700000222046FFF7B3FC8DF839008DF83AB07F
:10A7800050B9BAF1010F12D0BAF1000F04D1218FE4
:10A79000A1F57F40FF380AD0208F40B18DF834B04A
:10A7A0004FF4806000E053E0ADF890000DE00DA89C
:10A7B0003599FBF78EFA81464FF480608DF834B0FE
:10A7C000ADF89000B9F1020F06D0FD48006880791D
:10A7D00028B18DF8100043E0A4F818A038E0B9F1D2
:10A7E000000F03D081208DF8100043E005A80090F1
:10A7F00094F82010534601222046FFF770FC8DF894
:10A80000100020463699FFF74EFC9DF81000F8B96D
:10A8100019203070012038801AE006208DF81000D1
:10A8200041E02078000723D5B8F1010F20D109209D
:10A830008DF83400A088ADF838000420369907F070
:10A8400078F80820ADF8900000E011E0A7F800B01B
:10A850009DF8340020B10DA83599FBF73AFA8146EE
:10A86000B9F1000F1CD005E05FEA4E607FF528AD1E
:10A870004FF004092088BDF8901008432080BDF8EF
:10A88000900080050AD5218FA1F57F40FE3805D1C3
:10A890002998E062A4F830804FF003094846D6E4D6
:10A8A0009DF8100058B10120307028787070BDF804
:10A8B000140070809DF810003071052038802088C9
:10A8C000BDF8901088432080E8E72DE9FF4F01781C
:10A8D000A5B080464FF0010B0BFA01F04FF60901CD
:10A8E000349C0840ADF86C0021884FF00009A1F5B8
:10A8F0007F42FF3A02D028B1080703D5012029B0D2
:10A90000BDE8F08F289F4FF0000A04A887F800A048
:10A910002799269A55460988ADF87C10A8498DF8E4
:10A9200068A00A728DF810A008603298486098F804
:10A930000000012830D0022809D0032876D13878C9
:10A9400020F03F001D303870B8F80400A08098F85F
:10A950000000022804D1387820F03F001B30387006
:10A9600021AAF91C07208DE80700BDF87C0094F8A7
:10A970002010C01E83B2B8F80400002200F013FDBE
:10A980000028DBD1B8F80400A7F80100BDF8840066
:10A99000C01CADF87C005FE198F805108DF86810D8
:10A9A00098F804004FF40079012802D00228C5D19C
:10A9B00033E1208808F1080600F4FE60ADF86C0071
:10A9C00010F0F00F1BD010F0C00F05D03088228B94
:10A9D000904201D005257DE189B9B078C0070ED03D
:10A9E000B2680720CDE90020CDF808A0F388B2882E
:10A9F00094F82010308800F0E5FA00286FD12899EB
:10AA0000BDF86C00491C802845D006DC10280ED00B
:10AA100020280CD0402891D122E0B0F5807F5FD073
:10AA200048457DD0B0F5806F88D1CBE029E1C006E4
:10AA300001D5082000E0102081460420ADF814A0C4
:10AA40001BAA8DF8100000921FA81AA90397CDE940
:10AA5000011033884A4607212046FFF793F992E018
:10AA60009DF868004FF00A09002894D121AA072018
:10AA70008DE80700BDF87C0094F82010401E83B2DA
:10AA8000208B002200F08FFC8DF868000B203870BE
:10AA9000BDF8840019E09DF868004FF00C0900280B
:10AAA0001CD123AA07208DE80700BDF87C00628C2A
:10AAB000401E83B294F82010208B00F074FC8DF8B7
:10AAC00068000D203870BDF88C00401CADF87C008B
:10AAD00004208DF81000208BADF81400BCE057E086
:10AAE0003188208B814253D19DF868104FF01209B4
:10AAF000002918D1616A81B1B178C90748D0B3681B
:10AB00000722CDE90032CDF808A0F388B28894F886
:10AB1000201000F057FA8DF868001320387000E01C
:10AB200002E0ADF87CB097E0B6F800C0208B844519
:10AB30002ED19DF868004FF016090028606B08D0F0
:10AB4000E0B34FF6FF7000215646ADF808A0019023
:10AB500027E060B1B178C9071AD1618F43181FA8E7
:10AB6000CDE900075A88998833F8060B09E0B078D8
:10AB7000C0070DD01FA8CDE90007B288F188604654
:10AB8000B368FFF7E4FA050066D0062D7AD03FE0FF
:10AB900005253DE0019021AA02A92046FFF700FA11
:10ABA0000146628FBDF80800824201D00029F1D031
:10ABB000608F616B08440680019860874CE000005C
:10ABC000200800209DF868004FF0180940B1208B44
:10ABD000C8B13088208320463399FFF764FA3BE000
:10ABE00004F118000090237E94F8201001222046E2
:10ABF000FFF775FA8DF868000028ECD1192038703D
:10AC0000ADF87CB0E7E7052520463399FFF74BFA0E
:10AC10009DF81000032857D05CE0208800F40070F5
:10AC2000ADF86C0048452CD1208FA0F57F41FE394E
:10AC30007FF4D0AED8F808004FF0160948B1606331
:10AC4000B8F80C1021874FF6FF716187A0F800A0BB
:10AC500002E04FF6FF702087BDF86C0030F4FE6113
:10AC600016D0782300220420339906F0C5FD98F809
:10AC70000000A0702088BDF86C10084320800AE016
:10AC800000E006252088BDF86C108843208021E074
:10AC90002188814321809DF8100028B15F484168D8
:10ACA00004A8FBF716F805469DF8680090B187F8F0
:10ACB000019087F800B0208B78809DF8680038718B
:10ACC0000520ADF87C0005E05448416804A8FBF776
:10ACD00000F80546208810F4FE6F22D1208E00B3C4
:10ACE0002799289B01AD0988ADF87C10DDE9321267
:10ACF000009385E816001FABE26A2699FFF784FAF5
:10AD0000054603280DD08DF810B0E06A0590339801
:10AD10000690002104A8FAF7DCFF00B10546A4F86C
:10AD200030A02798BDF87C1001802846E7E500B5E3
:10AD300097B0042807D102208DF80000019100216E
:10AD40006846FAF7C6FF17B000BD70B5334C0378FC
:10AD500000222168012B02D0022B44D129E00B787C
:10AD60000BB1042B03D10A712268032111702168F1
:10AD7000062582880B7905EBC303CA522168082394
:10AD80000A250A7903EBC2021144C2880A802168AD
:10AD900002890B7905EBC303CA52418920680C2351
:10ADA000027903EBC202815220680179491C0171CA
:10ADB0001DE00A7482888A802168C288CA8022685D
:10ADC00001891181226841895181C1682068C1606F
:10ADD0006168FAF77EFF0146022806D02068007CF1
:10ADE000002801D119B1812070BD832070BD0020E1
:10ADF00070BD406B002800D0012070478178012988
:10AE000009D10088B0F5205F03D042F601018842E5
:10AE100001D1002070470620704700002008002064
:10AE200010B58B7883B102789A4205D10B885BB15B
:10AE300002E08B79091D4BB18B789A42F9D1B0F8B9
:10AE400001300C88A342F4D1002010BD812010BD38
:10AE500007282BD012B1012A2CD103E0497801F048
:10AE6000070102E04978C1F3C201052922D2DFE8D7
:10AE700001F0031D081017000AB1032070470220DB
:10AE80007047042812D0052810D006280ED058B1DB
:10AE90000EE005280AD0062808D0022808D003E0D2
:10AEA000062803D0032803D00520704700207047F0
:10AEB0000F2070478120704710B513880B800B78E6
:10AEC0001C061FD5FE4CA47A844204D843F010001F
:10AED0000870002010BD94682478C44064F3041303
:10AEE0000B701378D17803F0030341EA032140F299
:10AEF0000123B1FBF3F403FB1411926800FB012062
:10AF0000401C10BD906810BD37B5BDF8041011800D
:10AF10009DF8045029061BD5E94901239468897AD4
:10AF2000814209D8FE280FD1E80602D58B405B1E6E
:10AF300000E00023237007E0217883409943C5F3A4
:10AF40000013834019432170107820F01000107016
:10AF50003EBD2DE9F0410746C81C0E4620F0030017
:10AF6000B04202D08620BDE8F081082A01D90E2027
:10AF7000F9E7D34D002034462E60AF802881AA72B5
:10AF8000E8801AE0E988491CE980810614D4E17858
:10AF900000F0030041EA002040F20121B0FBF1F291
:10AFA00001FB1201206800F0E3FA2989084480B20D
:10AFB0002881381A3044A0600C3420784107E1D44D
:10AFC0000020D0E72DE9FF4F85B01546DDE912B628
:10AFD0008046994623F4404700F0BAFA04000BD0AB
:10AFE000207800060AD5B648817A0698814205D8AD
:10AFF000872009B0BDE8F08F0120FAE722466946B4
:10B000000698FFF759FF824600208DF80400072EAE
:10B0100018D0012221463046FFF71AFF0028E8D158
:10B02000207840060ED502208DF80400ADF8088087
:10B03000BDF80000ADF80C50ADF80A00ADF80E7088
:10B04000CDF810B05FEA094004D500273D46B84668
:10B0500001260CE02178E07801F0030140EA0120AC
:10B0600040F20121B0FBF1F2804601FB12865FEA5B
:10B07000494009D5B04507D1A178207901F00301F5
:10B0800040EA0120A84201D3B54201D90720B0E728
:10B0900078191FFA80F9B14501D90D20A9E79DF86B
:10B0A000040020B101A8FAF712FE0028A1D1B04592
:10B0B00007D1A0784FEA192161F30100A07084F84C
:10B0C0000490149800B10780BBF1000F15D00AEB73
:10B0D00005003A4659460FF0ADFE224669460698ED
:10B0E000FFF7EAFE9DF80000224620F010008DF8E0
:10B0F000000000990698FFF707FF002079E72DE987
:10B10000FF4FDFF8BC9182461746B9F80610D9F810
:10B11000000001EB410100EB810440F20120B2FB91
:10B12000F0F183B000FB11764D46DDF844803146E6
:10B13000049800F01DFA29682A898B46611A0C319F
:10B1400001441144AB8889B28B4202D8842007B0F5
:10B1500050E70499CDB2290603D5A90601D585206B
:10B16000F5E7B9F806C00CF1010C1FFA8CFCA9F840
:10B1700006C0129909B1A1F800C0A90602D5C4F809
:10B18000088007E0104480B2A9F80800191A01EB02
:10B190000B00A0602246FE200499FFF7B5FEE77081
:10B1A00026712078390A61F30100320AA17840F053
:10B1B000040062F30101A17020709AF8020060712E
:10B1C000BAF80000E08000262673280602D599F818
:10B1D0000A7000E00127A80601D54FF000084D468F
:10B1E00000244FF007090DE0CDF80080CDE901966D
:10B1F000E8882146109B069AFFF7E4FE0028A6D1B6
:10B20000641CE4B2BC42EFD30020A0E72DE9F04774
:10B21000804600F09DF9070005D000264446284DE1
:10B2200040F2012916E00120BDE8F087204600F039
:10B230008FF90278C17802F0030241EA0222B2FBE0
:10B24000F9F309FB1321006800F092F93044641C03
:10B2500086B2A4B2E988601E8142E7DCA8F1010051
:10B26000E8802889801B288100203870DCE720B125
:10B27000401E10809170002070470120704710B56B
:10B280000F4904460088CA88904201D3822010BD2D
:10B29000096800EB400001EB80025079A072D08871
:10B2A00020819178107901F0030140EA0120A0810A
:10B2B000A078E11CFFF700FE20612088401C01E01F
:10B2C0002C0800202080E080002010BD0121018298
:10B2D00070472DE9FC474FF6FF780546A2F800803D
:10B2E000406817468A4680788DF8020068680088B2
:10B2F000ADF8000000208DF80600288A2C88A042B6
:10B3000000D304462C822DE0288A401C2882701D20
:10B310006968FFF785FD18BB3988414501D1601E7A
:10B3200038806888A04222D3B178307901F00301D7
:10B3300040EA01296946701DFFF772FD80B96989ED
:10B34000414519D0002231465046FFF781FD38B9FA
:10B350006A894A4504D1E968B0680FF03FFD58B1E9
:10B36000641CA4B2204600F0F3F80600CCD1641EA1
:10B370002C828220BDE8FC877C807079B871F088CF
:10B38000B8803178F07801F0030140EA012078813B
:10B39000A7F80C90287A324607F10801FFF78CFDD8
:10B3A00038610020E6E72DE9F04F85B01D46904654
:10B3B0000F468346DDF838A0DDF8409000F0C8F86D
:10B3C000040009D02078000608D57148807AB84278
:10B3D00004D8872005B00DE60120FBE7C8F3090675
:10B3E000224669463846FFF767FD07465046BAF1E0
:10B3F000070F1AD000222146FFF72AFD0028E9D1C5
:10B400002078400611D501208DF80400ADF808B071
:10B41000BDF80000ADF80A00ADF80C60ADF80E50B4
:10B4200001A8FAF754FC0028D4D12178E07801F083
:10B43000030140EA0121A278207902F0030240EAE8
:10B440000220464507D0B1F5007F04D9691E81422C
:10B4500001DD0B20BEE7864201D90720BAE7801B39
:10B4600082B2AA4200D92A46B9F1000F01D0A9F848
:10B4700000200F9810B1B9190FF0DCFC0020A9E7EB
:10B480002DE9F0411D4617460E4600F061F8040014
:10B4900008D02078000607D53D48807AB04203D80E
:10B4A000872060E501205EE5224639463046FFF7F9
:10B4B00003FD65B12178E07801F0030140EA012045
:10B4C000B0F5007F01D8012000E0002028700020A6
:10B4D00049E52DE9F0411D4617460E4600F038F8C3
:10B4E000040008D02078000607D52948807AB042A9
:10B4F00003D8872037E5012035E522463946304616
:10B50000FFF702FDFF2D14D02178E07801F003024F
:10B5100040EA022040F20122B0FBF2F302FB1300EA
:10B5200015B900F2012080B2E070000A60F3010159
:10B530002170002017E510B50C4600F009F828B17D
:10B54000C18821804079A070002010BD012010BD6D
:10B550000F49CA88824209D340B1096800EB400014
:10B560006FF00B0202EB8000084470470020704728
:10B57000C0B2820609D4000605D50548807A484342
:10B58000401C80B27047084670470020704700009A
:10B590002C08002010B506F08BFB05F026FEFBF70B
:10B5A00011FF0EF04FFB06F083FABDE8104006F0E5
:10B5B0000FBB10B50C4601F0C1FC80B3204600F073
:10B5C000ACFA68B322780E2A09D00F2A07D0022AD3
:10B5D00005D0032A03D0102A2ED0FFDF1DE0A0786B
:10B5E0001E282BD00FDC0C2824D008DC092825D2FB
:10B5F000DFE800F013241724241E1E1A1C00122852
:10B600001CD1072010BD302818DDA0F13A00032816
:10B6100014D2DFE800F011130B00002010BD11E080
:10B620000EE043F20200F9E70420F7E70D20F5E70A
:10B630000F20F3E70820F1E71120EFE70320EDE703
:10B64000FFDFEAE7FFDFE8E700F067BA70B503461F
:10B65000002002466FF02F050EE09C5CA4F130063E
:10B660000A2E02D34FF0FF3070BD00EB800005EBD7
:10B670004000521C2044D2B28A42EED370BD30B595
:10B680000A240AE0B0FBF4F304FB13008D183030F9
:10B6900005F8010C521E1846D2B2002AF2D130BD74
:10B6A00030B500234FF6FF7510E0040A44EA00208D
:10B6B00084B2C85C6040C0F30314604005EA003403
:10B6C0004440E0B25B1C84EA40109BB29342ECD34E
:10B6D00030BD000010B509F0DBFB042803D009F0F1
:10B6E000D7FB052802D108F0D4F950B909F05CFC69
:10B6F000032803D009F05EFC032804D107F0AEFA5A
:10B7000008B1012010BD002010BD70B50C460546E3
:10B71000062102F092F9606008B1002006E00721DE
:10B72000284602F08AF9606018B1012020700020DC
:10B7300070BD022070BD2DE9FC470C4606466946E7
:10B74000FFF7E3FF00287DD19DF8000058B107F016
:10B75000E7F9B0427ED00022214630460BF0F9FCDA
:10B76000002874D116E007F042FFB04272D00022E8
:10B77000214630460BF0E0F8002868D1019D95F88D
:10B780009800303518B9687E08B1012000E000202B
:10B79000804603E0019D95F8498030354FF0010A5D
:10B7A00095F82D004FF00009A0B195F82E00800704
:10B7B00010D584F8019084F800A084F80290A68047
:10B7C00095F82F10A171298E2181698E618185F8EC
:10B7D0002D903CE0304602F0A8FA070000D1FFDFD0
:10B7E000384601F049FD10F0FF0008D084F80190C0
:10B7F0000D212170A680E08084F802A027E0304669
:10B8000002F081FA070000D1FFDFB8F1000F21D06C
:10B81000384601F0BCFDA8B19DF8000038B9019888
:10B82000D0F8BC004188B14201D180F80090304688
:10B8300007F0DBF884F801900A21217084F8029067
:10B84000A68000E006E0A97EA17185F8199001208C
:10B85000BDE8FC870020FBE71CB56946FFF755FFF4
:10B8600000B1FFDF684601F0B1FBFD4900208968A7
:10B87000A1F89A001CBD2DE9FC4104460E460620A5
:10B8800002F086F80546072002F082F82844C7B285
:10B890000025A8463E4417E02088401C80B2208046
:10B8A000B04202D34046A4F8008080B2B84204D32C
:10B8B000B04202D20020BDE8FC816946FFF725FFB7
:10B8C0000028F8D06D1CEDB2AE42E5D84FF6FF70FF
:10B8D00020801220EFE738B54FF6FF70ADF800007A
:10B8E0000DE00621BDF8000002F0B9F8044607217A
:10B8F000BDF8000002F0B3F80CB100B1FFDF002189
:10B900006846FFF7B8FF0028EBD038BD2DE9F041BD
:10B91000D4A0D64C06790025076884F8425001F07F
:10B920004EFB84F8435004202087102060874FF698
:10B93000FF70A4F80A0184F80C51A4F80E0184F8F1
:10B94000315004F8EE5BC94804F8C05C04F8BA5CF6
:10B950008030A57340F87D7FC4490671FD31481ED3
:10B960000BF095F80A20207503206075A075E0752E
:10B970000E20207606206076A076E076BDE8F08185
:10B980002DE9F041B64C0D466060217007F015F8C6
:10B99000FFF7A1FFFFF7BAFF207809F01CF8B349C1
:10B9A000C431A1F181000F46064607F041FF6068EF
:10B9B0000BF038F820780CF0C9FB284609F0C1FEDE
:10B9C0003946304607F0E8F860680BF04DFC01F0AE
:10B9D000F6FAA649002081F84300CFE710B501240C
:10B9E0000AB1002010BD21B1012903D00024204656
:10B9F00010BD02210DF096FBF9E72DE9F047040098
:10BA000000D1FFDF994D002695F8310058B16670DE
:10BA10001020207095F83200A07095F83300E07087
:10BA200085F831606AE0287840B12C22A91C2046B4
:10BA30000FF000FA0E2020702E705FE095F82E00B7
:10BA400060B10120E07095F82F00A07095F83000EB
:10BA500060700F20207085F82E604FE0844802212E
:10BA60008246FFF708FF00B1FFDFB5F80E91062010
:10BA700001F08EFF0746072001F08AFF3844C7B265
:10BA8000781C00F0FF0800BFB5F80E01B84213D1D2
:10BA90000021204607F05EFD58BB95F8340080B3C6
:10BAA0006670132020701C21A01C0FF03AFA0220AF
:10BAB000A07085F8346021E040451BD1002120466C
:10BAC00007F000F8E8B12078132817D1A0783C28B7
:10BAD00014D1A088072101F0B0FF050000D1FFDFDD
:10BAE000288806F082FFA088072101F0B8FF00B186
:10BAF000FFDF03E02146FFF71EFE10B10120BDE885
:10BB0000F087FFE702215046FFF7B5FE18B9B5F8F8
:10BB10000E114945B8D10020F1E76EE710B508F0E5
:10BB2000C8FE00B1FFDF0AF07BFF00B1FFDF07F0C6
:10BB300035FE09F0EFFD00B1FFDF0BF093FB00B124
:10BB4000FFDF06F0F7FF00B1FFDF0CF0F9FA00B1FC
:10BB5000FFDFFFF7C0FEFFF7D9FE06F017FF02F088
:10BB6000C1F801F02CFA4148002180F8431001711E
:10BB7000012141710222C270017010BD10B53B4C11
:10BB8000207828B10A21BDE810400E2001F0E4B968
:10BB9000FFF7A0FD08B10C2002E001F010FA002030
:10BBA0002071012060710A21E170207010BD70B514
:10BBB0002E4C0546207828B1BDE8704039210E2072
:10BBC00001F0CAB9FFF786FD08B10C2012E094F825
:10BBD000430008280DD204EB0010102229464430FF
:10BBE00001F0C7F994F84300401C84F8430000209A
:10BBF00000E007202071012060713921E170207080
:10BC000070BD70B5194C0546207828B1BDE870406C
:10BC10000B210E2001F0A0B9287818B1012801D01D
:10BC2000122016E094F8C400082823D2FFF752FD32
:10BC300008B10C200DE00E482B7894F8C4106A1C53
:10BC4000463806F01AF994F8C400401C84F8C40081
:10BC500000202071012060710B21E170207070BD07
:10BC600044000020FFFFFFFF1F00000038080020F5
:10BC7000460900200720ECE710B5FE4C207828B1DB
:10BC80003821BDE810400E2001F066B9FFF722FD13
:10BC900008B10C2002E0002084F84300207101204C
:10BCA00060713821E170207010BDF248017819B13F
:10BCB0000F210E2001F050B9002101710E21817079
:10BCC0000F21C170FF2181714FF6FF710181EA4997
:10BCD00049680A7882728A8882814988C1810121F3
:10BCE000417101707047E3490A781AB13B210E2077
:10BCF00001F032B90088A1F80A01012081F80C0195
:10BD000000220A7148713B22CA700870704710B552
:10BD1000D84C207828B12B21BDE810400E2001F02E
:10BD20001BB90821A01D05F0F9FA0020207101209F
:10BD300060712B21E170207010BD70B5CD4C217861
:10BD400029B1BDE8704031210E2001F005B990F90C
:10BD50000000042814D098B1011D11D010F1080F73
:10BD60000ED010F10C0F0BD010F1100F08D010F105
:10BD7000140F05D010F1280F02D01220207103E01B
:10BD8000002506F0BBF825713120E07001206071BC
:10BD9000207064E730B5B74D04468DB0287828B1DF
:10BDA0002A210E2001F0D8F80DB030BD1022214616
:10BDB000684601F0DEF8102204F1100104A801F039
:10BDC000D8F868460DF0D6FF10222C46A81D08A909
:10BDD00001F0CFF8002020710E20A0702A20E07022
:10BDE000012060712070DFE72DE9FF41A14C207830
:10BDF00028B13A210E2001F0AFF8BDE8FF814FF0E5
:10BE0000000884F80680B4F80A01ADF8040002A91D
:10BE1000FFF77BFC20B1002101A8FFF72CFDE8BB58
:10BE2000BDF80400ADF8000002A980B2FFF76DFC78
:10BE300000B1FFDFBDF8000001F077FF050000D181
:10BE4000FFDF2846039F01F0A9FA80F0010697F86A
:10BE50004950BDF8000001F056FF070000D1FFDF98
:10BE6000384601F094FA80F0010255EA020019D038
:10BE7000A179BDF8000004EB410108817D49A37957
:10BE80001831585C65F300005854A37962F34100FF
:10BE90005854A27966F38200505400E00DE0A07976
:10BEA000401CA07100216846FFF7E5FC28B9BDF8E9
:10BEB0000000BDF804108842B6D1012084F8048047
:10BEC00060713A21E170207097E770B5694C0546C2
:10BED000207828B1BDE8704034210E2001F03CB834
:10BEE00008F0D6FF052804D0284608F061FD0020A0
:10BEF00000E00C202071012060713421E17020707D
:10BF0000ADE65C48017819B10E21084601F024B86D
:10BF10005949CA68C0F80620098A41810021017187
:10BF2000012141710E22C2700170704770B5514CF1
:10BF30000646251D207828B1BDE8704032210E202C
:10BF400001F00AB83146002006F00EFF287058B9FB
:10BF500000213246084607F053FD287020B94648B4
:10BF60003168C160B1880182012060713221E170C5
:10BF7000207074E670B53F4C0546207828B1BDE8C6
:10BF8000704030210E2000F0E7BF08F0C4FD10B96A
:10BF900009F064FE68B1287809F034FC287807F0CD
:10BFA000A7FD00202071012060713021E170207018
:10BFB00055E60C20F6E72DE9F0412E4C0646251DEE
:10BFC000207828B1BDE8F04117210E2000F0C4BF51
:10BFD0003146012006F0C8FE2870012768B93246B4
:10BFE0000121002007F00CFD287030B93068E063B3
:10BFF000B088A4F8400084F8427067711720E070A0
:10C000002770BBE438B51B4D0446287828B1BDE83D
:10C01000384030210E2000F09FBF227961798A429A
:10C0200015D0A079E379984211D01F2A0FD81F2983
:10C030000DD8002211460EF03DF940B90022E079FA
:10C0400011460EF037F910B9207A072801D91220CD
:10C050001BE04FF6FF70ADF8000008F0A5FFD8B95F
:10C0600008F0A8FFC0B908F013FFA8B9002168467E
:10C0700004E000003808002044000020FFF7FBFB2C
:10C0800050B1204605F032FE002028710120687171
:10C090003E21E970287038BD0C20F6E72DE9FC47F9
:10C0A000FE4C054694F82E0028B128210F2000F000
:10C0B00053FFBDE8FC87282084F83000012184F874
:10C0C0002E10A8784FF000091A2825D00EDC16286B
:10C0D00031D2DFE800F030303030302130303030D5
:10C0E0003030303030303030302121212A2822D0F9
:10C0F0000BDCA0F11E000C281DD2DFE800F01C1C98
:10C100001C1C1C1C1C1C1C1C1C0D3A38042812D2A4
:10C11000DFE800F0110211022888B0F5706F0AD232
:10C120001F20884684F82F0028886946FFF7EDFA1B
:10C1300018B1022019E0122017E09DF80000019FBD
:10C14000002806D007F1CE07019E05D106F1B506FD
:10C1500004E007F1B407F7E706F1CF06684600F000
:10C1600023FF08B1387818B10C2084F82F00A0E71D
:10C1700087F80080A878307084F82F90684600F027
:10C1800025FF96E77CB5C54C0546207820B12521D2
:10C190000E2000F0E1FE7CBD28886946FFF7B5FA65
:10C1A000002168B102202071BC4881600173E180E8
:10C1B0000E20A0702520E0700120607120707CBDF1
:10C1C000019A104612F1300282F836108368A3609B
:10C1D000037B237392F83630002BF5D12888E0805A
:10C1E000E6E72DE9FC41AD4C064694F82E0028B157
:10C1F00010210F2000F0B0FEBDE8FC811F2084F864
:10C200002F00102084F83000012784F82E70308829
:10C210006946FFF77AFA70B9684600F0C5FE50B17A
:10C22000019D9DF8000030350028019805D0E230CE
:10C23000017841B904E0022006E0D0F8BC00F7E73D
:10C2400095F82D1019B13A2084F82F00D4E795F80D
:10C250002E1089070CD1042101709DF8000020B92F
:10C2600001993088D1F8BC104880684600F0AEFED5
:10C27000002084F82F0085F82D70BDE72DE9F047E8
:10C28000864D0646287828B1BDE8F0471D210E20CE
:10C2900000F062BE4FF01F0985F80490012068711C
:10C2A0001D21E970287008F0F3FD0C2704284ED0FA
:10C2B00005284CD0B0791224012800D0E8B9307894
:10C2C00008B1012819D1F07908B1012815D1708879
:10C2D00043F6FD71021F30248A420ED2B288121F2B
:10C2E0008A420AD22887B0886887B0794FF0000860
:10C2F0004446012803D050B111E02C710CE495F8AC
:10C30000420020B3654A3C320121084602E0644AFB
:10C310000021012007F074FB040000D0FFDFF0795A
:10C32000012800D010B907F093FB044614B185F83A
:10C330000490E3E73078012801D018B109E000212A
:10C34000022001E00021012007F097FB08B12F71C6
:10C35000D4E785F80480D1E770B5504C217829B135
:10C36000BDE870401E210E2000F0F6BD1F21217196
:10C37000012161711E22E270217002781221012ACE
:10C3800000D01AB9407818B1012801D0217166E4B3
:10C3900000260C25012A08D008F07AFD052802D0D5
:10C3A00008F034FA30B1257159E4618F208F08F01C
:10C3B000BFFBF7E7267152E42DE9FE4F0546AFF2C9
:10C3C0005C71D1E90001354E01908A4696F82E0045
:10C3D00030B103B02121BDE8F04F0F2000F0BCBD0B
:10C3E0001F2086F82F00212086F830004FF001082A
:10C3F00086F82E80298843F6FD730A1F30209A4262
:10C400007ED26A88141F9C42FAD28A4278D8EA897E
:10C4100040F67B43911F9942F2D2298A8C1F9C429D
:10C42000EED28A42F2D86A8AB2F5FA7FE8D2AA8AB4
:10C4300040F67744A2F10A03A342E1D2B2EBD10F56
:10C440005ED9E98A2A8B9142E0D82979122011B16C
:10C45000012955D102E069790029F9D1297B09B177
:10C460000129F6D108F014FD4FF00C0905286ED013
:10C4700008F00EFD0428FAD096F83400002866D1A2
:10C4800007F0B5F8A0F57F41FF39F8D1062102A8E1
:10C4900001F0A4FA040050D0032103E03808002082
:10C4A000500000200CF02CFB96F8030100901B229A
:10C4B00096F802312088114601F070FB04283ED026
:10C4C00000B1FFDF208806F08FFA04F10D07B4F801
:10C4D00000B00421384604F021FF594638460CF0DC
:10C4E00004FCFDA03F1D006800900321684604F095
:10C4F000A0FE002069460A5C3A54401CC0B200E02D
:10C500006FE00328F7D3288A6080688AA080A88A11
:10C51000E08096F8051196F8040108F0C8FA014683
:10C52000204608F0F0FA002784F8367084F8377057
:10C53000687968B101280FD10CE0092051E020880A
:10C54000062101F08CFA00B1FFDF072049E071E01D
:10C55000677601E084F81980D5F80600C4F81A005F
:10C560006889E0830198A06084F80CA084F8C480F6
:10C570008DF800700121684604F05BFE9DF8000014
:10C5800000F00701C0F3C1021144C0F34010084499
:10C590008DF80000401D2076092801D20830207651
:10C5A000002120460CF0ACFA287B18B1012805D0F8
:10C5B000FFDF24E00021C94A012005E096F842008F
:10C5C00098B10121C64A084607F01AFAB8B1208886
:10C5D00006F00BFA2088062101F041FA00B1FFDFD6
:10C5E0001F2086F82F00BDE8FE8F208806F0FDF999
:10C5F0002088062101F033FAE0B1FFDF1AE0287944
:10C60000012800D010B907F023FA50B921460320C1
:10C6100007F033FA28B96A882988204608F005FA15
:10C6200058B1208806F0E1F92088062101F017FAB8
:10C6300000B1FFDF86F82F90D5E784F8B87086F850
:10C640002F70D0E738B5A64C3C3C207820B1222191
:10C650000E2000F081FC38BD1F202071012565717E
:10C660002220E070257008F013FC052802D00C2071
:10C67000207138BD00202071684608F090FA00282B
:10C68000F7D10098008806F0B0F9009806210088DC
:10C6900001F0E5F900B1FFDF904884F834500C3820
:10C6A0000078FCF78DFF38BD2DE9F0418C4D044634
:10C6B0003C3D95F82E0028B1BDE8F04123210F2024
:10C6C00000F04ABC1F2085F82F00232085F8300099
:10C6D000012085F82E00618840F67B438A1F3020B8
:10C6E0009A4251D2A288961F9E424DD291424BD877
:10C6F000E188B1F5FA7F47D2218940F67746A1F16A
:10C700000A03B34240D2B1EBD20F3DD96189A2896D
:10C71000914239D84FF000082088062101F08DF9A8
:10C7200006004FF0020707D000F030FC20B1D6F829
:10C73000BC00017839B902E085F82F7061E4D6F8C1
:10C74000D010097809B13A201EE005218171D6F890
:10C75000BC004146A0F80880D6F8BC20A0885081D3
:10C76000D6F8BC20E0889081D6F8BC202089D08102
:10C77000D6F8BC00028943899A4204D88279082AF3
:10C7800001D89A4203D3122085F82F0039E4228879
:10C790004280D6F8BC00077085F82F1031E42DE9EF
:10C7A000FE434F4C06463C3C207830B103B0242178
:10C7B000BDE8F0430E2000F0CFBB012565712420B9
:10C7C000E070257030460CF0B2FA08B1002000E0AD
:10C7D0001220207100282DD1414884F8FC504430AB
:10C7E000316840F87D1F317901714FF0000884F8FD
:10C7F000FC806946062001F0ACF800B1FFDF684616
:10C8000001F085F8A0B9BDF8047000BFBDF80400C0
:10C81000062101F012F9060000D1FFDF86F8C450AE
:10C82000684601F074F818B9BDF80400B842EDD1BB
:10C8300084F80480BDE8FE8370B5294D06463C3D72
:10C8400095F82E0028B1BDE8704026210F2000F099
:10C8500083BB1F2085F82F00262085F8300001209B
:10C8600085F82E003088062101F0E7F8040007D093
:10C8700000F08CFB20B1D4F8BC00017831B901E0A4
:10C8800002200CE0D4F8D010097809B13A2006E073
:10C8900005210170D4F8BC1030884880002085F84C
:10C8A0002F0074E50E483C38017819B106210E209E
:10C8B00000F052BB002101710E2282700622C2706C
:10C8C000C0F80610C0F80A10817941F001018171A9
:10C8D0000121417101707047112233005000002086
:10C8E0007408002070B5F84E054696F82E0028B161
:10C8F000BDE870402C210F2000F02EBB1F2086F8D1
:10C900002F002C2086F83000012086F82E00288881
:10C91000062101F092F8040007D000F037FB20B1A7
:10C92000D4F8BC00017831B901E0022020E0D4F84D
:10C93000D010097809B13A201AE094F86410D1B106
:10C94000D5F802104160D5F80610816054F8BC0F8C
:10C95000698910228181206805F10C010E300EF0EA
:10C9600069FA21680320087021682888488000201F
:10C9700086F82F000BE50C20FAE770B5D24E04467E
:10C980000C25307828B1BDE8704018210E2000F049
:10C99000E3BA08F009FB032852D008F00BFB032888
:10C9A0004ED0607908B1012829D1A07908B10128B9
:10C9B00025D1A07B28B1012803D0022801D003286B
:10C9C0001DD1607BD8B1C00819D162884FF4804076
:10C9D000824202D82188814203D9207901280ED1D0
:10C9E00018E0207930B1012814D0022805D003289E
:10C9F00005D102E0202A0BD30CE0A0290AD220792D
:10CA0000042805D12088202802D36188884201D9D2
:10CA1000122515E0207986F83600607910B10128DA
:10CA200004D00DE0A94A0021204606E096F8420015
:10CA300030B1A54A01213C32204606F016F90546E0
:10CA40000120357170711821F17030709FE410B5BC
:10CA50009D4C217829B11A21BDE810400E2000F02C
:10CA60007BBA01781F2902D91220207106E000212B
:10CA700021710278411C104606F0A8F9012060716E
:10CA80001A21E170207010BD10B58F4C217829B1AA
:10CA90002021BDE810400E2000F05EBA01781F2969
:10CAA00002D91220207106E0002121710278411C78
:10CAB000104606F07AF9012060712021E1702070A3
:10CAC00010BD2DE9FC41804C217829B1BDE8FC4125
:10CAD0001B210E2000F040BA012767710C21217143
:10CAE00000780026012803D000286AD012205CE0DC
:10CAF00006F085F800287ED094F83600A0B1012811
:10CB000012D0042810D008F055FA002873D108F08C
:10CB10004BFA18B108F048FA02286CD1002008F04E
:10CB200074FEE0B3FFDF4AE008F03EFA002862D16D
:10CB300008F040FA00285ED105F0F2FFA0F57F4131
:10CB4000FF3958D1072101A800F048FF5F49054689
:10CB50000C398860280000D1FFDF032128460BF044
:10CB60001DFF284606F0FCF994F8091194F8080115
:10CB700008F023FA0146284608F04BFA94F807011A
:10CB800000901B2294F806312888114601F006F81F
:10CB900068B1042800D0FFDF2888072100E00EE0FC
:10CBA00000F05DFF00B1FFDF0720207123E028883F
:10CBB00005F01AFF284608F028FE00B1FFDF2671B5
:10CBC00019E008F0F1F9032803D008F0F3F903287D
:10CBD00011D108F0ECF90546002008F027FD50B906
:10CBE000267145B1288805F000FF2888072100F04C
:10CBF00036FF00B1FFDF1B20E0702770BDE8FC812D
:10CC00002DE9F041304C0646207828B1BDE8F041CE
:10CC10002D210E2000F0A0B93088072100F00DFF73
:10CC200005004FF0010720D095F8D10040B995F8E4
:10CC30003C000F2801D0102802D195F8040150B112
:10CC40000C2020710E20A0702D20E0703088E08034
:10CC50006771277072E51022B11C05F1D2000EF049
:10CC6000E9F885F8D1700020EBE70220E9E770B51C
:10CC7000154C0546207828B1BDE870402E210E20C5
:10CC800000F06AB92888072100F0D7FE022178B1A8
:10CC900090F8D1202AB990F83C200F2A04D0102A0D
:10CCA00002D00C20207104E080F8D1100020F9E7B8
:10CCB00021710E20A0702E20E0702888E0800120D5
:10CCC00060712070EDE50000380800205000002061
:10CCD0007CB5C54C0546207820B137210E2000F0E8
:10CCE0003BF97CBD28886946FEF70FFD38B102206C
:10CCF0002071012060713721E17020707CBD0198A6
:10CD00007F22014680F8382080F83920002280F800
:10CD10003A20A87801F8280FE878487028798870B8
:10CD20002271E6E71CB5B04C217821B113210E2009
:10CD300000F012F91CBD00886946FEF7E6FC08B158
:10CD4000022005E0019890F82810012902D00C205B
:10CD5000207106E0382100222271095C21720088CE
:10CD6000E080012060711321E1700E21A17020701C
:10CD70001CBD2DE9F0419C4C0546207828B1BDE84A
:10CD8000F04135210E2000F0E7B8A87808B101285D
:10CD900003D1A888B0F5FA7F01D912202071288824
:10CDA000072100F04AFE0126A0B1002780F8C870D4
:10CDB000A988A0F8CA1080F8A460A978012900D039
:10CDC000002180F8C81090F8A50008B108F01CFEFA
:10CDD000277101E00220207166713520E070267015
:10CDE000ACE42DE9F041804C0546207828B1BDE83F
:10CDF000F0413C210E2000F0AFB82888072100F058
:10CE00001CFE012358B382886D88C688418803EBD5
:10CE10004207BD4217D342F210777E43BF107943D9
:10CE2000B6FBF1F1491E89B24FF4FA76B14200D94E
:10CE300031468D4200D22946491C521CB1FBF2F109
:10CE40005143491E8AB290F8F01001B90284E28081
:10CE50000020207163713C20E07023706EE402209A
:10CE6000F7E770B5604C0546207828B1BDE8704002
:10CE700033210E2000F070B808F096F808B10C20AD
:10CE800017E0297889B10A290FD014290DD01E295D
:10CE90000BD0282909D0322907D04B2905D0642985
:10CEA00003D0FF2901D0122003E0284608F04FFDEF
:10CEB00000202071012060713321E1702070F0E4C6
:10CEC00049490A781AB13F210E2000F045B80022E6
:10CED0000A710278454B4AB1012A0CD01220087120
:10CEE000012048713F22CA700870F4E4D0F80100B4
:10CEF000C3F80200F4E7D0F80100C3F80600EFE73A
:10CF000070B5394C0546207828B1BDE870403D2108
:10CF10000E2000F021B808F047F810B908F04AF8E0
:10CF200008B10C2003E0287805F060FF0020207194
:10CF3000012060713D21E1702070B2E410B50178EC
:10CF4000402907D22A4A52F8211019B1801C88477B
:10CF5000012010BD002010BD234A92F83130002B73
:10CF600006D182F8320082F83310012082F83100B5
:10CF7000B1E430B5134606E0CC18D51A14F8014CCC
:10CF80005B1E4455DBB2002BF6D130BD90F8491042
:10CF900041B990F8981029B190F89800042801D070
:10CFA000012098E4002096E40178406821B190F8CF
:10CFB000490010B100208EE4E8E701208BE40A4824
:10CFC0000021C0F8F81080F8C41084E40178012929
:10CFD00009D1406890F8A510002904D0002180F8FC
:10CFE000A51008F011BD76E43808002038090020AB
:10CFF0004CB301003D3070470844C01D424301F16D
:10D000003D00104480B2704770B51C460546A0181C
:10D01000049BC01D00FB03F204F13D00104486B2E6
:10D02000B14238BFFFDF1C2128460DF07AFFA6F180
:10D030001C0080B22C752880B0F5004F88BFFFDF40
:10D0400070BD008870472DE9F04F0E468188044678
:10D0500000F11C0AC088154620F4004221F4004368
:10D06000002721F4004820F400499A4208D100F436
:10D07000004001F4004188421CBF0020BDE8F08F51
:10D08000C14517D9207DA9EB0801091AC91F8D4296
:10D0900027DCC11D0AEB08000144C91E71603581FF
:10D0A000F7603782011D3160058047800120A07440
:10D0B000BDE8F08F2088217DA0EB0800401AB0F178
:10D0C000070B0ED4BBF11B0FB8BFFFDF5D45D4BF0C
:10D0D00028461FFA8BF0291A0A04120C18BF4A4579
:10D0E00003DDA7740020BDE8F08F217DCB1D0AEB86
:10D0F00008010B44DB1E7360308104F11C03F360F4
:10D1000032820B1D336008804A800120A074BDE884
:10D11000F08F2DE9F041044600F11C02808820F4D4
:10D120000043A07C002808BFBDE8F081D018028829
:10D13000438813448B423CBF0020BDE8F0810027A8
:10D1400091429CBF0180478013D9891A0D042D0C90
:10D1500045800ED0A088261D20F40040854288BF5F
:10D16000FFDF30884FF4004121EA0000284330807F
:10D1700008E0217D0088CB1D184481B22288201D43
:10D1800000F09AFAA7740120BDE8F08130B4B0F83D
:10D1900002C08488034600F11C052CF4004028449A
:10D1A000A44503D10020D88130BC7047B3F80AC031
:10D1B0000488A44509D34088ACEB040CA0EB0C0018
:10D1C00084B20CEB0500C01E06E0A4EB0C041D7D30
:10D1D000A4B2AC446044001DB1F800C0A44588BFAF
:10D1E0000C80B3F80AC0BCF1000F0CBF4FF0010C6B
:10D1F0004FF0000C82F800C00988D98130BC70471C
:10D200002DE9F041044600F11C01408820F4004063
:10D210004518E089002808BFBDE8F081618908440D
:10D2200080B2608129886A881144814238BFFFDF5B
:10D2300028886D88628941190027914218D175B1FB
:10D240006088A61C20F40040A84238BFFFDF308869
:10D250004FF4004121EA00002843308007E0217D9F
:10D260002288CB1D184481B2A01C00F025FA6781EA
:10D27000E7810120BDE8F0812DE9F0470189B0F890
:10D2800002800027044600F11C0A414518BF4FF4F4
:10D29000004938D021F400400AEB00014E886EB1FD
:10D2A000208904F1080520F40040B04238BFFFDFB8
:10D2B000288829EA0000304328801FE0207D238948
:10D2C000C21D088823F4004510442188284480B2F8
:10D2D00004F1080C88420AD2091A89B21B32914221
:10D2E0002CBF03F4004129EA030004D204E0401AF1
:10D2F00080B229EA03010843ACF80000781C2189B8
:10D3000087B24145C6D13846BDE8F0872DE9F047E0
:10D31000B0F806800B46044600F11C01B0F80890F6
:10D32000408828F4004C01EB0C05804504BF002028
:10D33000BDE8F087002A1CBF281D106023B1227DA4
:10D34000291D18460DF076FD2F886D8885B1E819E6
:10D3500087B2E088A61D20F40040A84238BFFFDF56
:10D3600030884FF4004121EA00002843308007E074
:10D37000207D2288C31DD81981B2A01D00F09CF920
:10D38000C84504BFE08820813846BDE8F087418861
:10D39000808881420CBF0120002070474188C088EE
:10D3A00088420CBF01200020704730B44488828836
:10D3B00000F11C0324F4004C22F400416344944225
:10D3C0001BD04289C48915191C885A88A3189D420C
:10D3D00016D312B18A4210D212E0037D0CF1070C71
:10D3E0001A196244008892B2801A80B2223398429D
:10D3F00001D211B104E08A4202D130BC0020704752
:10D4000030BC012070472DE9F0078588C48800F101
:10D410001C06024625F4004C24F4004925F4004A79
:10D42000002024F4004306EB0C074FF00108D1451F
:10D430000AD104F4004405F40045AC4204D0108243
:10D44000BDE8F00700207047634506D9147DA3EBC3
:10D450000C031B1BDD1F002305E01488157DA4EBC6
:10D460000C04641BE51F002DE9DB94895CB13C884A
:10D470007F8847B1DB1BD0748B42E0DB908930445E
:10D48000001BC01E12E02D1BD0748D4206DB107DE8
:10D490009389C01D60443344184406E08B42CEDBC0
:10D4A00082F8138090893044001BC01E1182BDE8B1
:10D4B000F00770472DE9F05F044600F11C088088F2
:10D4C000924620F4004B208A894608EB0B0608B1EF
:10D4D000484502D20020BDE8F09FA089002804BF83
:10D4E00000273D4605D0378875887919884218BFCE
:10D4F000FFDFE07C50EA050101D078B338E0A08975
:10D5000050B1217D4044C91D59440844B4F8151058
:10D5100020F8031DE17D8170A18907EB09004944D2
:10D52000A181308000257580207DBAF1000F09D0DF
:10D53000C31D30882288184481B2201D00F0BCF839
:10D54000A5813AE0A189C01D58444144084430F8FF
:10D55000031DA4F815108078E0752EE0FFE7A08980
:10D56000B4F815104044C01B20F8031DE17D817004
:10D5700005EB090085B2A089BAF1000F4844A081EB
:10D580003780758010D0A088261D20F40040A84266
:10D5900038BFFFDF30884FF4004121EA0000284304
:10D5A00030800020A08108E0A0894044C01B30F8F2
:10D5B000031DA4F815108078E07500202082A07467
:10D5C0000120BDE8F09F10B4B0F802C0848800F1DB
:10D5D0001C022CF400431344A44504D0B0F80AC044
:10D5E000BCF1000F02D010BC0020704703F1040C06
:10D5F000C1F800C0007D00F1070C0CEB0300C01E59
:10D60000486018880881CA605B880B8220B9D01EE8
:10D6100048600B810020088210BC0120704770B563
:10D62000044600F11C018288408820F4004319441C
:10D63000904205D06289002A04BFE289002A01D005
:10D64000002070BD0A884D8885B1A61C20F40040DA
:10D65000A84238BFFFDF30884FF4004121EA0000C4
:10D66000284330800020E081012070BD207DC31D53
:10D67000981881B22288A01C00F01EF8F2E7002161
:10D680008181C1740182817470478289002A04BF3C
:10D6900000207047828800F11C0322F400421A44E3
:10D6A000B2F800C0BCF1000F1DBF037D121D1A446B
:10D6B000DA1E4A608089704710B4B0F800C02CF4BC
:10D6C0000044214489B24FF4004491420AD2521AD4
:10D6D00092B21B339A422CBF0CF4004224EA0C0194
:10D6E00004D204E0891A89B224EA0C0211430180B1
:10D6F00010BC70472DE9F04188464FF6FC7102F1ED
:10D7000003021E46040002EA010509D00027E01CBE
:10D7100020F00300A04200D0FFDF201D01210CE01B
:10D720000127F4E7024628442FB9B14201D203464B
:10D7300000E000231360491CC9B2B142F2D9011BB9
:10D74000C8F80010002F04D10EB1201D00E0002009
:10D750002060BDE8F081024600201168002902D057
:10D76000084609681160704702680A6001607047E6
:10D770004FF6FC73C91C1940101A001F90FBF1F002
:10D78000C0B270474FF6FC73C91C1940001D01FB65
:10D7900002007047F8B5D24D04460E46A878A04264
:10D7A00000D8FFDF05EB8607B86A50F8240000B107
:10D7B000FFDFB868FFF7CFFF05000DD0B86A062E6F
:10D7C00040F824500AD0082E00D3FFDFC548294670
:10D7D00050F82620204690472846F8BDC048C24B46
:10D7E0007A30A0F12E0200902946204609F08FF8E9
:10D7F000F2E72DE9F84F8046DDF828901E4603EB4E
:10D80000090093468A46C4B25FEA080707D000259C
:10D81000FF2800D9FFDFBAF1000F03D101E0012595
:10D82000F6E7FFDF08F1030020F00301414500D0D7
:10D83000FFDFCB4500D9FFDF65B9A94A00204C3294
:10D840004FF6FF7110705180A74A1070A44A7A32C7
:10D8500010705180A24880F800B046708470C47087
:10D860000471447180F80690DFF878B2C671002622
:10D870000BF1400B8146FF1C27F003000746002DEB
:10D8800002D109EB860188603BF8162019F80630B2
:10D8900001D04FF000006946FFF72CFF0098761C7E
:10D8A000F6B20744082EE6D3FF1C27F003002346F8
:10D8B000064675B1002002226946FFF71BFF00985B
:10D8C0003118002003464E46C91C21F003021DB149
:10D8D00010E0C9F84800EEE706EB80070021BA62C5
:10D8E00006E000BFD7F828C04CF82130491CC9B267
:10D8F000A142F7D3401CC0B202EB84010828E3D355
:10D90000A1EB0800AAF800000020BDE8F88F10B5D0
:10D91000044604F075F808B1102010BD2078704A54
:10D92000618802EB800092780EE0836A53F8213020
:10D9300043B14A1C6280A180806A50F82100A06037
:10D94000002010BD491C89B28A42EED861800520B2
:10D9500010BD70B505460C46084604F051F808B1F4
:10D96000102070BD082D01D3072070BD2570002048
:10D97000608070BD0EB56946FFF7EBFF00B1FFDFB9
:10D980006846FFF7C4FF08B100200EBD01200EBDA0
:10D9900010B50446082800D3FFDF5148005D10BDD4
:10D9A0003EB5054600246946FFF7D3FF18B1FFDFF7
:10D9B00001E0641CE4B26846FFF7A9FF0028F8D034
:10D9C0002846FFF7E5FF001BC0B23EBD44498978F9
:10D9D000814201D9C0B27047FF2070472DE9F04164
:10D9E0000C460546062901D0072C10D13C4FB86CD7
:10D9F000FFF7B1FE02004FF6FF7604D00221B86CAB
:10DA0000FFF7B6FE00E030462880B04202D1002089
:10DA1000BDE8F0812146FFF7BDFE040002D1288851
:10DA200000F050F82046F3E7A0F57F42FF3A01D01E
:10DA3000082901D300207047ACE6A0F57F42FF3AE9
:10DA40000BD0082909D2264A9378834205D902EBE4
:10DA50008101896A51F820007047002070472DE944
:10DA6000F04104460D46A4F57F4143F20200FF3920
:10DA7000CED0082D01D30720CAE719494FF000087E
:10DA80008A78A242C4D901EB85072146BA6A52F8C6
:10DA90002460002EBCD0134A08462032314652F88A
:10DAA00025209047B96A062D41F8248001D0072D22
:10DAB00002D1204600F006F83146B868FFF754FE60
:10DAC0000020A5E710B5064CC2B20221A06CFFF7FA
:10DAD00059FE0146A06CBDE81040FFF745BE0000AE
:10DAE000480900204CB40100560000200146A0481F
:10DAF000002200680260037A00EB830040F80C2FDC
:10DB00008180114600F025B92DE9F05F9846DDF8D7
:10DB100030B0DDF828A01546894604004FF0000615
:10DB200025D00027E01C20F00300A04200D0FFDF3A
:10DB30007DB30120FFF75EFA00FB05620AEBCB0024
:10DB4000104486B20120FFF755FA00FB05620B99DD
:10DB500008EBC100104405EB450100EB4100143017
:10DB600000EB850000EB850086B217B111E00127BC
:10DB7000D8E7A6EB85000C3887B27D48A900046081
:10DB8000257204F10C0060600DF0EDF93846FFF7E6
:10DB9000ADFFA9F800600020BDE8F09F2DE9FF4F20
:10DBA000734C814681B020689A468B4600B9FFDFEE
:10DBB0002068027A4A4503D9426852F8291021B1F7
:10DBC00043F2020005B0BDE8F08F006800B9FFDF46
:10DBD00001210E9A0398FFF70FFAC61C4FF6FC7549
:10DBE0002E40584601215246FFF706FAC01C00EAB3
:10DBF000050808EB0600001D85B25D480027006897
:10DC0000046801E027460446206838B1A188A9428B
:10DC1000F8D13946204600F0A4F813E005F10800D9
:10DC2000A18880B2814229D33946204600F099F874
:10DC3000A0880022411B601902608180394600F0F3
:10DC400088F8A580A08860802680251D0E9F01236E
:10DC5000039A314628460097FFF7D6F920884146B7
:10DC600028445A460123CDF800A0FFF7CDF94048DB
:10DC700000684168002041F82940A3E70420A1E79B
:10DC800070B53B4C0546206800B9FFDF2068017A7B
:10DC9000A94210D9426852F8250060B1418800239A
:10DCA00042F8253003608180194600F052F821685F
:10DCB00000200A7A08E043F2020070BD4B6853F876
:10DCC00020306BB9401CC0B28242F7D8002002E07D
:10DCD0008A88104480B209680029F9D1FFF706FF4D
:10DCE000002070BD70B5224D286800280AD000249D
:10DCF00004E02046FFF7C4FF641CE4B22868007A01
:10DD0000A042F6D870BD70B5194E054600243068A3
:10DD100000B9FFDF3068017AA94204D9406850F8A1
:10DD2000250000B1041D204670BD70B5104E05469B
:10DD30000024306800B9FFDF3068017AA94206D9B3
:10DD4000406850F8251011B131F8040B44182046F2
:10DD500070BD19B10A68026008607047044909681B
:10DD6000F8E7006809B10860704701490968FAE7F7
:10DD70005C00002070B5044600780E4601281AD0D9
:10DD8000072802D00C281AD115E0A068216905786F
:10DD90000B2D0CD0052003F0CCFD052D0FD07823E2
:10DDA00000220520D4F8101003F026FD07E07823A8
:10DDB00000220620F8E70520216903F0BAFD31466C
:10DDC0002046BDE8704001F0BDB910B500F1390240
:10DDD000C3799478411D64F003042340C371DB07C9
:10DDE0000DD04B79547923404B710B791279134044
:10DDF0000B718278C9788A4200D9817010BD0022E7
:10DE00004A710A71F5E74178012900D00C210170AF
:10DE100070472DE9F74F86B000208C698DF800001F
:10DE20000878012617460D464FF0070B4FF01109F1
:10DE30004FF00A0A2A2878D2DFE810F02A001A03E5
:10DE400058036D03A703B603D203FF03160440046F
:10DE500068048704A004DD04EE04110519053905E2
:10DE60005E058905AC05D705F505FF0521063206D7
:10DE7000440676069806EA0621072F075A077A070E
:10DE80008E079F07D80710083C08F807FC07020810
:10DE900014B120781D2829D0D5F808805FEA080041
:10DEA00043D001208DF80000686A049003208DF8AB
:10DEB00004008DF805A0286A0290A8880028EFD0F9
:10DEC00098F8001091B10F2910D27DD2DFE801F04F
:10DED0007C144BDCFEFDFCFBFAF9F8089EF7F6001B
:10DEE000022822D124B120780C2801D0002676E324
:10DEF00002208DF80000B7E10620696A03F019FDE1
:10DF0000A8880728EDD1204601F017F9022809D08A
:10DF1000204601F012F9032808D9204601F00DF936
:10DF2000072803D20120207005E016E2002CB7D0AC
:10DF300020780128D5D198F80400C11F0A2902D3FE
:10DF400085F81CA093E2A070D8F80010A163B8F87F
:10DF50000410A18798F8060084F83E00012028707C
:10DF60000320207046E00728BBD1002C98D02078F1
:10DF70000D28B6D198F8031094F83B20C1F3C000E7
:10DF8000C2F3C002104201D00E2000E00F2089072A
:10DF900007D198F805100142D2D198F80610014235
:10DFA000CED194F83D2098F8051020EA02021142E3
:10DFB000C6D194F83E2098F8061090430142BFD194
:10DFC00098F80400C11F00E04FE20A29B8D2617F2F
:10DFD000814201D90620C9E3D8F800106160B8F881
:10DFE0000410218198F80600A072012028700E20EC
:10DFF000207003208DF80000686A049004F1390055
:10E000000190601D029017300390E1E0B5F806B072
:10E0100041288FD1204601F090F8042802D1E07801
:10E02000C00704D1204601F088F80F289CD1CBF11D
:10E030004002164608F10101606A0CF0FBFE606ABE
:10E040005A463044E9680CF0F5FE0E208DF80000C9
:10E05000686A0490606A019000216846FFF78AFEB2
:10E060002078042808D0A07F48B1012807D00328D1
:10E0700008D010202070A2E00520207015E284F85E
:10E08000009033E71220F5E71128C2D1204601F0B5
:10E0900054F8042802D1E078C00719D0204601F0D6
:10E0A0004CF8062805D1E078C00711D1A07F0228DE
:10E0B0000ED0204601F041F8112808E0B9E089E0CF
:10E0C000A1E178E158E110E1EFE0D5E01DE0A0D159
:10E0D000102208F1010104F148000CF0ABFE607859
:10E0E000012809D012202070E078C0076BD0A07FF3
:10E0F000A0B3012863D066E0607FA17888423FF634
:10E1000069AF00BF84F800B059E011288ED12046D5
:10E1100001F013F8082804D0204601F00EF8132867
:10E1200084D12869D8B16869C8B104F17800102297
:10E1300008F1010106460CF07DFE2078082812D077
:10E1400014202070E078C0070FD0A07F022818D0DC
:10E150006178022912D0032831D034E02FE000206A
:10E160008DF80000F9E00920EBE70B202870296901
:10E1700002204870206CC1E9010695E208B101282F
:10E1800079D10B202870296908204870606A48609E
:10E19000206AC1E902067BE2206CE2780068C2F3E3
:10E1A0004402521ED04000F0010040F0800000E028
:10E1B00000200874E06A48617FE20646FEE304201E
:10E1C00028700520EBE185F800A08DF800A0B9E3E8
:10E1D0003946F4E31128C5D1204600F0AEFF0A28E5
:10E1E00002D1E078C00704D1204600F0A6FF152830
:10E1F000B8D1102208F1010104F148000CF01AFE18
:10E2000020780A2810D01620207012202870296942
:10E2100004F1580081F801A048602030886010386F
:10E22000C860206C0861AFE30B202070E1E2287029
:10E23000D4E1022896D1204600F07FFF042804D3C1
:10E24000204600F07AFF082809D3204600F075FF29
:10E250000E2887D3204600F070FF12287DD2A07FC1
:10E260000228B8D18DF80090686A049098F80100EF
:10E270008DF80400FEE367E20228ACD1204600F0EE
:10E280005CFF002869D0204600F057FF0128F9D034
:10E29000204600F052FF0C28F4D005208DF8040031
:10E2A00098F801008DF805005CE71128FCD1002CDE
:10E2B000FAD020781728F7D16178E06A022912D0C5
:10E2C0005FF0000101EB4101182606EBC1011022AD
:10E2D000405808F101010CF0ADFD0520696A00F01D
:10E2E0001FFF267002E60121ECE70B28DCD1002C91
:10E2F000DAD020781828D7D16178E06A02292DD0A9
:10E300005FF0000101EB4101102202EBC101415815
:10E31000B8F8010008806078E16A022821D0002066
:10E3200000EB4002142000EBC2000958404650F8B0
:10E33000032F0A60406848600520696A00F0F0FE1B
:10E340006078022810D04FF000002044407A20F07E
:10E3500001010CD14FF001000BE0D3E14FF00101BE
:10E36000D0E74FF00100DBE74FF00100EDE74FF0A1
:10E3700000002044417281E3112895D1002C93D0F4
:10E380002078192890D16178E06A022911D0002103
:10E3900001EB41011C2202EBC1011022405808F19F
:10E3A00001010CF047FD0520696A00F0B9FE1A2052
:10E3B000E9E00121ECE7082898D1002C98D02078DA
:10E3C0001A2893D1E16A98F801000870E16AD8F838
:10E3D000022041F8012FB8F8060088800520696AFC
:10E3E00000F09EFE6078022807D04FF00000204425
:10E3F000407A20F002002CD034E04FF00100F6E724
:10E40000214448723AE31128B7D1002CB7D02078C4
:10E410001B28B2D16178E06A02291DD05FF00001AB
:10E4200001EB4101202202EBC1011022405808F10A
:10E4300001010CF0FFFC0520696A00F071FE6078B4
:10E4400002280CD04FF000002044407A20F0040055
:10E4500008D14FF00101D3E74FF00101E0E74FF0A1
:10E460000100F1E74FF00001CAE785F81CB0F4E3C2
:10E470003878012886D11C2204F11C0079680CF040
:10E480001EFDE079C10894F83B0001EAD001E07874
:10E4900061F30000E070217F09B1297732E1217832
:10E4A00003290AD0C0073FF4E6AD032028708DF899
:10E4B00000A0686A04904120A7E302262671E17952
:10E4C000204621F0E001E171617A21F0F0016172F2
:10E4D000A17A21F0F001A172FFF777FC2E708DF880
:10E4E00000A0686A04908DF804B071E638781228AC
:10E4F000D4D18DF800B0696A049191680291ADF8A9
:10E5000004B008466168016021898180A17A817127
:10E5100004202070AEE23878B7F806801228BDD10A
:10E520008DF800B0686A0490381D01AB07C883E815
:10E5300007004120ADF8040008460C2100F8011B3B
:10E54000C8F140063246216A0CF074FC206A42464B
:10E550008119F8680CF06EFC00216846FFF70AFC90
:10E56000E07820F03E00801CE0702078052801D083
:10E570000F2008E0A07F00283FF4C4AD0128FBD0A5
:10E58000032870D108202070B0E43878032885D1A2
:10E5900078680168A1664068E066052028708DF8FB
:10E5A0000000686A049013E638780328A0D17868E0
:10E5B0000168216740686067206C68B9A07F28B156
:10E5C000012803D0062028700420E8E785F800B071
:10E5D000FE482064606401E085F800B00326F0E3A3
:10E5E0003878022884D13879E0BBA07F02280BD08C
:10E5F0000328F1D1607801280BD0A07994F83A1063
:10E6000001280AD0F1480BE0B86800287AD02064CD
:10E6100011E0A17994F83A00F2E7B8680028F5D043
:10E620002064E078C00701D0012901D0E74802E06A
:10E63000F8680028EAD06064CEE78DF800A0696A27
:10E640000491E1785046C90709D06178022903D1C5
:10E65000A17F29B1012903D0A17F032900D008207F
:10E66000287046E101E1BFE0387812288FD1B86800
:10E67000286209202870E0782969C0070DD0082099
:10E680004870206A4860606A886004F16800C86069
:10E69000A07F02287FF48CAD7EE502204870206CBC
:10E6A000486004F16800886004F13800C860201DEB
:10E6B0000861206B4861606B88612EE2E1783878F0
:10E6C000C90701D0072100E00B2188428AD12078B8
:10E6D000072818D084F800908DF800B0686A04907C
:10E6E000286A0290ADF80490032100F8011B5168DC
:10E6F00010220CF09FFB00216846FFF73BFB002037
:10E700002862BEE44CE208202070E5E73878122841
:10E71000ACD18DF800B0686A049090680290ADF8B2
:10E720000490042100F8011B102204F168010CF090
:10E7300081FB00216846FFF71DFB2078092801D0E6
:10E74000132020E784F800A016E0E1783878C907A4
:10E7500001D0072100E00B21884287D1102204F16B
:10E76000480079680CF03AFB10B104202877B1E337
:10E77000207809283FF4BFAC0C2058E5E078C107A9
:10E7800037D0A17F012902D002291BD02EE00D2015
:10E79000287029690B2048706078012809D0206A08
:10E7A0004860606A886004F16800C86010300861E1
:10E7B00000E5606A4860206A886004F17800C860FB
:10E7C0001038F4E7C0F3440114290FD24FF0006170
:10E7D00001EBB0104FEAB060E0706078012803D020
:10E7E00010202070042061E10620CCE6607801282A
:10E7F00087D00E201BE538780A2889D185F800A03B
:10E8000010208DF80000686A049050680190002183
:10E810006846FFF7AFFAE9E7E078C0070AD0A07FC3
:10E82000012803D10F202870042041E11020287016
:10E830000F203DE115202870296903204870206CC5
:10E8400048606078012805D004F1780088601038AD
:10E85000C86062E104F1680088601030F8E7387839
:10E860000228CAD138790028E0D0287730E33878F8
:10E870001428FBD185F80090296909204870786830
:10E880004860607801280DD004F16800886010307D
:10E89000C860206B0861606B486104F158008861B2
:10E8A000A06A22E004F1780088601038F0E7387838
:10E8B0000828DBD16078012801D0132043E2A17839
:10E8C000A06A0844C1F110010CF02BFB1220287043
:10E8D000296904F1580081F801A04860203088605F
:10E8E0001038C860206C086147E0C861E06A0862BF
:10E8F00013E18DF80490DFE038780928B6D11022B2
:10E9000004F1480079680CF069FA08B10B202DE792
:10E9100020780B2812D02046FFF757FAA178A06A7A
:10E920000844C1F110010CF0FCFA162028700820F0
:10E930008DF80000686A049000206FE013202870B2
:10E940008DF800A0686A04908DF8049040E438784F
:10E9500012288BD1B868286214202870296904F124
:10E96000580081F801A04860103088601030C860FD
:10E97000606C08616078012806D004F139004861B4
:10E98000206B8861606BB0E7601D4861606B8861D7
:10E99000206BAAE7387809288BD18DF800B0686A17
:10E9A0000490286A0290ADF804900D2100F8011B34
:10E9B000102279680CF03EFA002101E077E27CE059
:10E9C0006846FFF7D7F90020286201E06AB5010028
:10E9D0006178012901D01520D5E51621297008217B
:10E9E0008DF80010696A049118E038780C2885D1F8
:10E9F000162028706078022802D12046FFF7E5F93A
:10EA0000A07879680A18C0F1100110460CF089FA54
:10EA100008208DF80000686A049078680190A0785A
:10EA20008DF8080061E53878102892D1E079C007A8
:10EA300079D01720287009203AE03878112888D139
:10EA40001422391D04F11C000CF039FAE16A208D02
:10EA5000A1F80900E16AA078C871E179E26A01F0E1
:10EA600003011172E16A627A0A73E16AA07A81F89D
:10EA7000240000E045E26078012876D0B4E16078B7
:10EA8000022801D0012000E000202044407AC00785
:10EA900004D0E078C00701D1192054E11E206CE6B3
:10EAA000387812287CD1B86828621A20287005208E
:10EAB0008DF80000686A049011466846FFF75AF91D
:10EAC000FFF77BBB387803286AD16078E16A0228B7
:10EAD00001D0012000E0002000EB4002142000EBF8
:10EAE000C20289587A6813680B6052684A601B2119
:10EAF0002970D5E9041206234B70636A4B6066786F
:10EB0000E36A022E01D0012600E0002606EB46064D
:10EB100000EBC6001858C1E90202686A486206980C
:10EB200000F027FBCCE788E138780F2838D16078EF
:10EB3000E26A022801D0012000E0002000EB400042
:10EB4000102101EBC00002231058093279680AF045
:10EB50006DFC1C202870296905204870206A4860D7
:10EB6000E06A09308860FA4872E65BE138780E287E
:10EB700016D16178E06A022901D0012100E000216C
:10EB800001EB4101182606EBC101A27840587968D3
:10EB90000CF050F96178E06A022902D0012101E00D
:10EBA000B8E0002101EB410106EBC1014158A0781A
:10EBB0000A18C0F1100110460CF0B3F98DF800B03E
:10EBC000686A0490286A0290ADF8049006210170EA
:10EBD0006278E16A022A01D0012200E0002202EB01
:10EBE000420206EBC202401C895810220CF022F9A6
:10EBF00000216846FFF7BEF8002028621D2028701B
:10EC00008DF800A0686A04900B208DF804006CE475
:10EC1000387812287ED18DF800B0686A0490906828
:10EC200002900B20ADF80400029880F800B06278E2
:10EC3000E16A022A01D0012200E0002202EB420236
:10EC4000102303EBC20289580988A0F801106178EB
:10EC5000E26A022902D0012101E03BE1002101EB3F
:10EC60004103142101EBC30151580A6840F8032FF6
:10EC70004968416000216846FFF77CF80EE760783C
:10EC8000022801D0012000E000202044407A8007C3
:10EC900001D51F2057E021206FE53878122839D19F
:10ECA0008DF800B0686A0490B8680290ADF80490DE
:10ECB000082606706278E16A022A01D0012200E08B
:10ECC000002202EB42021C2303EBC202401C8958C3
:10ECD00010220CF0AFF800216846FFF74BF8202017
:10ECE00028708DF800A0686A04908DF804605AE4DA
:10ECF000387812280ED18DF800B0686A04909068B8
:10ED000002900820ADF80400029809210170E16921
:10ED1000097800E093E04170E16951F8012FC0F8F3
:10ED200002208988C18000216846FFF723F8B2E7F6
:10ED30006078022801D0012100E000212144497AB5
:10ED4000490706D5222028708DF800A0686A049033
:10ED5000CFE5012848D067E0387812286FD1B8682D
:10ED6000286223202870296905204870206A48609D
:10ED7000E06A0930886077486AE538780E285ED105
:10ED80006178E06A022901D0012100E0002101EB55
:10ED90004101202606EBC1014058516810220CF0B9
:10EDA00049F88DF800B0686A0490286A0290ADF8BE
:10EDB000049080F800A06278E16A022A02D0012261
:10EDC00001E0A4E0002202EB420206EBC202401C7A
:10EDD000895810220CF02EF800216846FEF7CAFF71
:10EDE000002028626078B4E72420C6E46078022816
:10EDF0000BD000202044407AC10702D0E178C90737
:10EE000005D0810705D519209BE40120F2E71720E2
:10EE100097E4400701D51B2093E41C202070607804
:10EE2000012801D01820A8E42720A6E42820287073
:10EE30000B203DE6387813284AD129209DE40CE0C8
:10EE40002078012844D00C2842D02046FEF7DBFF72
:10EE50000C208DF80000686A049039E038784FF093
:10EE60002608122805D013201070032685F800808C
:10EE70004DE08DF800B0686A0490B86802900220F6
:10EE8000ADF80400029805210170297F417000212E
:10EE90006846FEF76FFF0B208DF80000686A04904B
:10EEA00039466846FEF766FF064685F80080012E63
:10EEB0000ED02CE001208DF80000686A0490042038
:10EEC0008DF80400287F8DF805000020287712E0D7
:10EED000287F80B11D202070252028708DF800A08B
:10EEE000686A049002208DF8040039466846FEF7EF
:10EEF00041FF06460BE00CB1FE2020709DF800009B
:10EF000028B100216846FEF735FFFEF7EFBF09B0D4
:10EF10003046BDE8F08F2DE9F04F0C4601274E69D1
:10EF2000097885B09046BA464FF00209072021B112
:10EF300001294FD0022920D1C9E0217901290BD024
:10EF4000022916D0032911D0042916D11CE0000093
:10EF500062B501009CB40100707801280CD1062034
:10EF6000616A02F0BFFC002807D11AE01D20307052
:10EF700017E07178022901D0052796E031780C2935
:10EF800027D18DF804000EE03078011F042902D348
:10EF90000E3803281DD2B07F02281AD120890228FA
:10EFA00017D38DF8049084F800A020899DF80410F0
:10EFB000884203D20A208DF800003FE01221083475
:10EFC00088F8001094E80E00C8E901120327C8F879
:10EFD0000C306AE098F80010122966D18DF8000014
:10EFE000616A0491D8F80850029521794FF00B0B13
:10EFF000012906D0022929D0032911D0042954D18E
:10F000005AE0ADF8049085F800B0207E4F4600F03D
:10F010001F00687000216846FEF7ACFE377043E0C1
:10F02000ADF8049005202870207E68704E460021BF
:10F030006846FEF79FFE26708DF800B0606A049067
:10F0400041466846FEF796FE07462EE0ADF80400FE
:10F0500085F800A0207F6870607F00F00100A87034
:10F06000A07F00F01F00E870E17F2971C0071FD06A
:10F0700094F8200000F00F00687194F8210000F06F
:10F080000F00A87100216846FEF774FE2868B0637F
:10F09000A888B087A87986F83E00A0694078707784
:10F0A0002879B0700D2030700027384605B030E761
:10F0B0000020A8716871E5E7ADF804900E20287073
:10F0C000207E687000216846FEF754FEECE7FE20C3
:10F0D00030708DF800A0606A049004208DF8040060
:10F0E000207E8DF80500EDE700B50023012285B0F4
:10F0F00005280FD006280BD102208DF8002004919E
:10F100008DF804008DF8053000216846FEF732FEC8
:10F1100005B000BD8DF8002004918DF80420F1E7C2
:10F1200070B50C46054602F004FC21462846BDE8B1
:10F1300070407823002202F05FBB08B1007870476E
:10F140000C20704770B50C0005784FF000010CD012
:10F1500021702146F4F70EF973482178405D88420A
:10F1600001D1032070BD022070BDF4F703F9002027
:10F1700070BD027B032A05D000220A704B780C2B4D
:10F1800002D003E0042070470A770A62027B9300F2
:10F19000521C0273C15003207047F0B585B00F4672
:10F1A00005460124287B05EB800050F8046C70783C
:10F1B000411E0D290AD25C493A46123101EB80000A
:10F1C000314650F8043C2846984704460CB1012CBF
:10F1D00011D1287B401E10F0FF00287301D00324BA
:10F1E000E0E70D208DF80000706A04900021019680
:10F1F0006846FFF7A7FF032CD4D005B02046F0BD2A
:10F2000070B515460A46044629461046FFF7C5FF65
:10F21000064674B12078FE280BD1207E30B1002044
:10F220002870294604F10C00FFF7B7FF2046FEF7CF
:10F23000EAFD304670BD704770B50D460446882122
:10F240000BF091FE012D03D0022D03D0052070BDDF
:10F25000012000E0022060702046FEF7D4FD00206F
:10F2600070BD28B1027E1AB10A4600F10C01C7E751
:10F270000120704730B5044687B00D46062002F0E5
:10F2800058FB2946052002F054FB2078FE2806D0C2
:10F2900000208DF8000069462046FFF7E2FF07B026
:10F2A00030BD7FB50E4600218DF80C1041780C2939
:10F2B00003D00D2903D0002405E0846900E04469EF
:10F2C0000CB1217E91B16D4601462846FFF751FFF2
:10F2D000032809D1324629462046FFF791FF9DF8C1
:10F2E0000C10002900D0042004B070BD04F10C05FE
:10F2F000EAE710B590B00C4607900B480521801E38
:10F3000008900A488DF8191009900F92694606A8CE
:10F31000FFF7C7FF002805D11022204601990BF006
:10F3200089FD002010B010BDA2B4010062B501003B
:10F3300070B50D46040011D085B1210128460BF0AF
:10F34000F0FD10224E4928460BF074FD4C48012177
:10F350000838018044804560002070BD012070BDE8
:10F3600070B5474E00240546083E10E07068AA7B41
:10F3700000EB0410817B914208D1C17BEA7B914272
:10F3800004D10C2229460BF029FD30B1641C3088D1
:10F390008442EBDB4FF0FF3070BD204670BD70B58E
:10F3A0000D46060006D02DB1FFF7DAFF002803DB7B
:10F3B000401C14E0102070BD314C083C208862884D
:10F3C000411C914201D9042070BD6168102201EBFB
:10F3D000001031460BF02EFD2088401C2080287044
:10F3E000002070BD70B514460D0018D0BCB10021CE
:10F3F000A170022802D0102811D105E0288870B130
:10F400000121A170108008E02846FFF7A9FF00281D
:10F4100005DB401CA070A8892080002070BD012061
:10F4200070BD70B5054614460E000BD0002030703C
:10F43000A878012808D005D91149A1F108010A8846
:10F4400090420AD9012070BD24B128782070288804
:10F45000000A5070022008700FE064B14968102261
:10F4600001EB0011204610390BF0E4FC28782073E2
:10F470002888000A607310203070002070BD0000E2
:10F48000680000202DE9F041FE4C207EE17D88429D
:10F4900008BFBDE8F0810126FB4D0027E07D215C1F
:10F4A00001EB810205EB8200037C052B10D0037C6D
:10F4B000062B1BD0037C072B27D0437C012B18BFC6
:10F4C000FFDF30D0207EE17D8842E7D1BDE8F081CA
:10F4D0000674E07D16281ABFE07D401C0020E07510
:10F4E000481CC0B255F8222002210CE00674E07DD1
:10F4F00016281ABFE07D401C0020E075481C55F816
:10F500002220C0B203219047DCE70674E07D162874
:10F510001ABFE07D401C0020E075481CC0B255F8C1
:10F5200022200821EFE74774E07D16280EBF002057
:10F53000E07D401CE075481CC0B255F82220072130
:10F54000E1E770B5D14E00240C2086F82900A6F51D
:10F550003B70254680F8CD4180F8CC4100F5F47031
:10F560000476C47506F12C000AF0B2FDA6F58E7083
:10F57000057586F82B50601EB06086F8255086F819
:10F58000225086F8235086F8245086F82150C0482F
:10F5900005704570A6F1E80004EB840100EB8101E1
:10F5A0000D74611CCCB20B2CF6D30120F9F726FBAD
:10F5B0000020F9F723FB012086F82600F9F7D2FF97
:10F5C000B448F9F7DEFFB44C2070B448F9F7D9FF1E
:10F5D0006070BDE87040F9F7A5BA10B5F9F7D0FA38
:10F5E000AD4C2078F9F7E6FF6078F9F7E3FFA74C18
:10F5F00094F82800002808BF10BDF9F7CAFC0020C5
:10F6000084F8280010BD0B20704770B5F9F79BFBFC
:10F610009E4C054694F8260000281CBFFFDF70BDF5
:10F6200094F82B00002808BFFFDF6FF07F4260696D
:10F630000026291AB1F5800F24BF431BB3F5800FB4
:10F640000DD38A4203D2101A2844411C07E09A4283
:10F6500028BFFFDF05D2511B0844401C414200294E
:10F6600000DBFFDF012584F8265084F82B6094F836
:10F6700029100420844A01EB810102EB8101087406
:10F68000A068B0F1FF3F04D0A81EA0600120F9F7E8
:10F69000B5FA0020F9F7B2FAF9F796FA0AF0A6FEE1
:10F6A000F9F7DAFB7E48066006604FF0E0214FF480
:10F6B0000040C1F88002F3F780FC7548007802280A
:10F6C00004D0032805D194F8230010B184F8225007
:10F6D00001E084F82260BDE87040F9F7A1BB034661
:10F6E00069490B2000EB800201EB820212F8042C26
:10F6F00022B1401E10F0FF00F4D1704700EB8002F1
:10F7000001EB8201012241F8143C01F8042C7047FE
:10F71000012804D0032808BF002926D000E021B327
:10F720005A4B4FF0000C83F821C0594A00289070C2
:10F7300014BF022882F803C00BD0072915D2DFE8D6
:10F7400001F01404060C0E1012001B2000E03A20F9
:10F75000D070012083F8210070475820F8E7772007
:10F76000F6E79620F4E7B520F2E700207047484816
:10F7700010B54078F9F779FB80B210BD421E10B584
:10F78000414900EB800001EB80040A2A02D814F8FA
:10F79000040C00B9FFDF14F8040C012818BFFFDFC8
:10F7A000002004F8040C10BD70B53E4C94F8CD0157
:10F7B00094F8CC1188420CBF01250025F9F7C3FA53
:10F7C000F9F753FB94F8CD1194F8CC2191420CBF7A
:10F7D00001210021A942E9D170BD2DE9F05F8046E9
:10F7E0004B1E1746DCB2284804EB840200EB82056E
:10F7F0002E1D287CDFF88C9007282DD199F8170052
:10F80000002299F818C0844524D000BF19F800C020
:10F81000A44508BF012200D04AB116280CBF4FF002
:10F82000000C00F1010C19F80CC009F800C01628F2
:10F830000CBF0020401CC0B299F818C08445E5D127
:10F8400042B199F818204846002A0EBF1622027EBF
:10F85000521E0276012028740A2B10D80A4801EBA8
:10F86000810100EB810010F8040C40B1287C0128D4
:10F8700006D0287C012802D0B87A012816D0FFDFF4
:10F88000B87A11E0BC0B0020D80B0020C00C00207F
:10F890007A000020A51601007800002085F4000001
:10F8A00000F50040D409002001284AD1FE49287CF7
:10F8B000022816D099F8180016284AD099F818008E
:10F8C00099F81710401C884200D1FFDF01206874AE
:10F8D00099F8180009F8004099F8180016283DD04A
:10F8E0003EE0DFF8C8C39CF829000246A04207D0DA
:10F8F000024600EB820001EB8000807CA042F7D141
:10F900009CF8293083420CD19CF8292002EB82021A
:10F9100001EB8202927C8CF8292001228CF82A20AB
:10F9200009E000EB800301EB830302EB820201EBB1
:10F9300082029B7C937400EB800001EB80000C2220
:10F940008274387A062825D2DFE800F012211E1BC7
:10F95000181599F817000028B8D1B6E7002002E082
:10F9600099F81800401C89F818000020BDE8F09FA5
:10F970004FF0000A11E04FF0B40A0EE04FF0730AA6
:10F980000BE04FF0320A08E04FF00A0A05E04FF0B2
:10F99000060A02E0FFDF4FF0000A3868A0EB0A0019
:10F9A0003060397A00290CBF04210221401A20F06E
:10F9B0007F423260D7E90001084420F07F40706048
:10F9C000B87A022818BF387B7ED1387A00280CBF5D
:10F9D0000420022000EB0A037868591D00EB010B9C
:10F9E000B3484078504503D9B04991F8231011B17C
:10F9F0000BF1060003E0A0EB0A005844801DAB4960
:10FA000091F829C0BCF10C0F24D08E4691F8291032
:10FA100001EB810CA44901EB8C0CDCF804C06245BD
:10FA200018D0DFF890C29EF8292002EB820201EB89
:10FA300082014A688968A2EB080222F07F42A1EBAA
:10FA4000080121F07F41904298BFB2F5800F49D262
:10FA50008C4547D34044A0EB0B0020F07F41316040
:10FA60001944F86821F07F410A1A6FF07F43B2F51C
:10FA7000800F24BFA0EB010CBCF5800F0DD3934287
:10FA800003D2181A0844421C07E0634528BFFFDF71
:10FA90001FD2591A0844401C4242002A19DD052091
:10FAA000287499F8180016282DD099F8180099F89C
:10FAB0001710401C884200D1FFDF99F8180009F8A0
:10FAC000004099F8180000E00BE016287FF448AFDA
:10FAD00044E73068ABF10501084420F07F407060D6
:10FAE000002030727068401D20F07F407060787A8E
:10FAF000B072387A0627707203280DD260B101F017
:10FB000023FB28B108E099F817000028D5D1D3E7E6
:10FB1000CAF138074FF0320A65480178012918BF49
:10FB200003290AD14078504507D9604991F823103C
:10FB3000002904BFA0EB0A0007445E4B3068A0EB2D
:10FB40000802706822F07F41A0EB080020F07F4C93
:10FB50008F4298BFB1F5800F1CD263451AD3534929
:10FB600091F829300C2B32D091F829704FF00C0B02
:10FB70004FEA0B0A4C4907EB870301EB8303D3F8E9
:10FB800008C0ACEB080C944531D8BB469F7C0C2FC9
:10FB9000F0D199E00520287499F81800162811D0A2
:10FBA00099F8180099F81710401C884200D1FFDF1F
:10FBB00099F8180009F8004099F8180016287FF401
:10FBC000CFAECBE699F817000028F1D1EFE702207D
:10FBD000287491F829000C2818BF91F82900A874FE
:10FBE00081F82940012081F82A00BDE8F09F0C2F00
:10FBF0001CBFBA46002267D00AEB8A0301EB8303DD
:10FC0000D3F804C0ACEB080C844528D29A7B96F854
:10FC10000AC094451CD30520287499F818001628AA
:10FC200011D099F8180099F81710401C884200D19B
:10FC3000FFDF99F8180009F8004099F81800162815
:10FC40007FF48EAE8AE699F817000028F1D1EFE72D
:10FC500093F812A00122BAF10C0FCDD103E0002AD3
:10FC600008BFBA4630D03E460F4806EB860200EB8E
:10FC70008208062188F8101099F81800162836D046
:10FC800099F8180099F81710401C884200D1FFDF3E
:10FC900099F8180009F8006099F8180016280CBFA8
:10FCA000002099F8180007E0D80B0020C00C0020B5
:10FCB0007A000020FFFF3F0018BF401C89F81800A1
:10FCC00098F81260B245CFD10220FE4E287406F19A
:10FCD000E80090F82910B9420ED185F812A080F8FA
:10FCE0002940012180F82A100120BDE8F09F99F8F1
:10FCF00017000028CCD1CAE70C2F0BD0BBF10C0F9A
:10FD000008BFFFDF0BEB8B0006EB8000847485F8E7
:10FD100012A0E9E7BBF10C0F08BFFFDF0BEB8B0074
:10FD200006EB800084740C20A874DDE730B50D4626
:10FD3000E54A44190021101A71EB010038BFFFDFBA
:10FD4000E2488542C8BFFFDFE1488542B8BFFFDF18
:10FD5000E0488442A8BFE04804DA002CAABF20464D
:10FD6000DC4830BD201830BD401E70B5C0B200EB7D
:10FD70008001D44800EB8104607B062810D2DFE8C4
:10FD800000F0030D0B090705002033E0B4200BE061
:10FD9000732009E0322007E00A2005E0062003E096
:10FDA000FFDF617B002029B3022108446168084419
:10FDB00020F07F40F9F759F894F90C50C24A4419E1
:10FDC0000021101A71EB010038BFFFDFBF488542E8
:10FDD000C8BFFFDFBE488542B8BFFFDFBD488442D1
:10FDE000A8BFBD4804DA002CAABF2046B94870BDA0
:10FDF000201870BD0421D8E72DE9F04F0646B7481A
:10FE000085B00068C005C00D11D0103840B2002880
:10FE1000B8BF00F00F0000F1E020B4BF90F8140D5F
:10FE200090F80004400908BF4FF0010A01D04FF0DC
:10FE3000000A3078002817BF01283079002005B06B
:10FE400018BFBDE8F08F062810D2DFE800F0030DE0
:10FE50000B090705002015E0B4200BE0732009E032
:10FE6000322007E00A2005E0062003E0FFDF3179B9
:10FE7000002039B15FF0020100EB0109BAF1000F77
:10FE800006D101E00421F7E79549002081F8270019
:10FE90006C4602AA2146B068F8F7F4FF9DF90820E5
:10FEA000F068211D10440122C01C1F28B8BF019218
:10FEB00008DB03AAF8F7E6FF9DF80C0010B10198E3
:10FEC000401C0190DDE900100844401D20F07F40F7
:10FED0000190A1EB090020F07F40009070798DF82F
:10FEE0000A0000980390F8F72EFF0099019B091A69
:10FEF000181A7C4A21F07F4120F07F40B1F5800F35
:10FF000010D282420ED3764890F82950009CAB461E
:10FF1000191B21F07F486FF07F41091BA0F1E80712
:10FF2000049101E0002080E00C2D26D005EB850037
:10FF300007EB80026FF07F435068011BB1F5800F23
:10FF400010D3A4EB000CBCF5800F0BD38B4203D273
:10FF500004990844411C05E063450DD2181A204459
:10FF6000401C4142002908DA5D48AB46957C90F878
:10FF700027000028D8D04CE0FFDF5D4525D00BEBF3
:10FF80008B0007EB80036FF07F429968081BB0F588
:10FF9000800F12D3A4EB010CBCF5800F0DD382426D
:10FFA00003D204980844401C07E0624528BFFFDFE5
:10FFB0000BD2521A1019401C4042002805DD9DF852
:10FFC0000A009A7B904228BF0C460C2D1CBF9DF85E
:10FFD0000A10434A14D000BF05EB850007EB8000F0
:10FFE00043681B1B23F07F43434509D2837B99421F
:10FFF00028BF8468857C92F8270050B90C2DEBD17E
:020000040001F9
:100000000098A04205D004EB080020F07F40009447
:10001000019000990398814206D001EB090020F07D
:100020007F40F8F722FFB06001202D4991F827109A
:10003000002904BF05B0BDE8F08FBAF1000F3FF40E
:1000400023AF05B0BDE8F08F2DE9F04F814687B0B2
:100050000C4625480AF044F8244901274FF00008CF
:1000600001EB090500287DD0A1F5887898F81400E7
:10007000002818BFFFDF2078012800F0238200BF8E
:1000800088F810902078022808BFFFDF184E2079EA
:1000900006F10C023072607970723146A068F8F790
:1000A000F1FE96F90C000F2804DD1F38307330681C
:1000B000401C306096F90C00E168351D0844C01CF6
:1000C0001F2817E0D80B0020FF7F841E0020A10707
:1000D00000E05EF80080841E00807BE104ED00E01B
:1000E000C00C0020FFFF3F00EC0C0020B40C0020EF
:1000F000A40B0020B8BF2F6009DB6A462946F8F739
:10010000C1FE9DF8000010B12868401C28602078CE
:10011000B07288F81470F64D95F8CD0195F8CC11B1
:10012000884204BF07B0BDE8F08FF24890F829403C
:100130000C2C00F0CF81F8F706FEEF4904EB8402A7
:1001400001EB82010A7C042A19BF0A7C032A07B04A
:10015000BDE8F08FE94B4A688968121A22F07F42A5
:10016000081A00E01BE020F07F40062A3CBF07B0E1
:10017000BDE8F08FB2F5800F24BF07B0BDE8F08F67
:1001800083423CBF07B0BDE8F08F95F8CD0195F8EC
:10019000CC11884240F0A78107B0BDE8F08FD44E63
:1001A00096F8CD01162855D096F8CD0196F8CC11C9
:1001B000401C884200D1FFDF207801284FD0CC4876
:1001C00090F8CD1101EB810100EB810080F81090D7
:1001D000207802284BD0C64890F8CD1101EB810160
:1001E00000EB8105207928726079687205F10C02B4
:1001F0002946A068F8F746FE95F90C000F2804DDA3
:100200001F3828732868401C286095F90C00E168A5
:100210002E1D0844C01C1F28B8BF376009DB6A4682
:100220003146F8F72FFE9DF8000010B13068401CF1
:1002300030602078A872AE4991F8CD0116280EBF23
:10024000002091F8CD01401C81F8CD01AC4809F0A7
:100250005DFF60E796F8CC010028ADD1ABE715F85B
:10026000010C002818BFFFDF05F8017CA7E7A548AF
:100270000068C005C00D0FD0103840B20028B8BFCC
:1002800000F00F0000F1E020ACBF90F8000490F8FF
:10029000140D400908BFFFDF954890F8CD1101AA61
:1002A00001EB810100EB8106E068CDF800808DF85C
:1002B00004806946F8F7E6FD9DF904000F28CCBFDD
:1002C000012000200099351D084401900220B072E1
:1002D0002079307260797072A068C01C1F28B8BF86
:1002E0002F6009DB6A462946F8F7CCFD9DF800002F
:1002F00010B12868401C2860307A062810D2DFE848
:1003000000F0030D0B09070500200BE0B42009E005
:10031000732007E0322005E00A2003E0062001E018
:10032000FFDF0020217900290CBF042102210844AD
:1003300002907168401D08440199009001440298A0
:10034000081A05906B4C002084F82700F8F7FBFC96
:10035000804630600198404420F07F40F06094F87F
:1003600029000C287ED0204690F8291001EB81024C
:10037000A0F1E80101EB82025468009A274622446A
:1003800022F07F42039296F809B090F82950121B90
:1003900022F07F4A6FF07F42121BA94604920C2D77
:1003A00027D0554805EB850100EB81036FF07F42B4
:1003B0005868011BB1F5800F24BFA4EB000CBCF5FD
:1003C000800F0BD38A4203D204990844411C05E0F4
:1003D00062450DD2111A0819401C4142002908DA61
:1003E0004448A9469D7C90F827000028D7D04DE0CE
:1003F000FFDF4D4525D0404809EB890100EB810125
:100400006FF07F438868021B8146B2F5800F24BFDE
:10041000A4EB000CBCF5800F0DD3934203D2049AD9
:100420001044421C07E0634528BFFFDF09D21A1AB7
:100430001019401C4242002A03DD887B834528BFF7
:100440004C460C2D1CBF2B4BA3F1E80116D000BF6E
:1004500005EB850001EB80025068001B20F07F4017
:10046000504500E026E009D2907B834528BF946880
:10047000957C93F8270048B90C2DE9D1A74205D007
:1004800004EB0A0020F07F4027460390039AA7EB75
:10049000080121F07F41A2EB0802059822F07F427B
:1004A000B1F5800F06D2904204D30298384420F070
:1004B0007F4030600F4890F8270000287FF442AF5B
:1004C000B9E600BF15F8010C002818BFFFDF05F8DA
:1004D000017CD5E595F8CD0195F8CC11884204BF93
:1004E00007B0BDE8F08F07B0BDE8F04FF8F798BC53
:1004F000D4090020C00C0020D80B0020FFFF3F00D3
:10050000EC0C002004ED00E00020F8F767BB0120B0
:10051000F8F764BBFD48007870472DE9F0410546C7
:1005200002282DD0FA4C94F829000C2808BFFFDFD0
:10053000002784F82670012684F82B6094F829108F
:100540000320DFF8D08301EB810108EB81010874FF
:10055000F8F76DFCD5B1012D39D0032D1CBFFFDF9D
:10056000BDE8F08194F8290094F82910401CC0B22D
:1005700001EB810158F82120BDE8F0410521104729
:10058000E2480078BDE8F041F9F71AB8207F00286A
:1005900018BFFFDF84F8256000202760F8F72EFBE6
:1005A000A168B1F1FF3F04D0012300221846F8F7FB
:1005B00069FB94F8290094F82910401CC0B201EBA3
:1005C000810158F82120BDE8F041012110470120A8
:1005D000F8F714FB94F8250000281CBFA068B0F1C0
:1005E000FF3F0DD094F8290094F82910401CC0B2A8
:1005F00001EB810158F82120BDE8F04106211047A8
:10060000207F012815D002281FD0032833D00428CA
:100610001CBFFFDFBDE8F08194F820106068012363
:10062000411A00221846F8F72DFB94F82800B8BBB1
:1006300037E094F8240028B184F82470F8F7FEFB22
:1006400084F823602777BDE8F08194F8280018B972
:10065000F8F776FC84F8286094F8290094F82910BB
:10066000401CC0B201EB810158F8212000219047C5
:100670002777BDE8F081217B60680123411A0022C1
:100680001846F8F7FFFA94F8240028B184F824708B
:10069000F8F7D4FB84F8236002202077BDE8F081CE
:1006A00003E0F8F74DFC84F8286094F8290094F8EA
:1006B0002910401CC0B201EB810158F82120002113
:1006C00090472677BDE8F08110B5914C94F8290049
:1006D0000C2808BFFFDF94F8290094F82910401C6B
:1006E000C0B28C4A01EB810152F82120BDE81040D4
:1006F000042110472DE9F05FF8F725FB844C814673
:100700004FF00C0B94F829000026A4F1E8084FF0F4
:10071000010A0C282CD094F82910204601EB810105
:1007200008EB8101097C042922D090F8291001EB03
:10073000810108EB8101097C032908BFBDE8F09F16
:10074000754922696069A2EB090222F07F42A0EBA1
:10075000090020F07F40062A38BFBDE8F09FB2F5BF
:10076000800F28BFBDE8F09F814238BFBDE8F09FF1
:10077000A068B0F1FF3F18BFFFDF84F8256094F850
:100780002900664F0C2806D194F8210018B1F8789A
:100790007870B87838705E4890F829000C281ED020
:1007A0005B4890F8291001EB810108EB8101097C7D
:1007B000042914D190F829B090F8291001EB810197
:1007C00008EB810181F810A090F8291001EB81015C
:1007D00008EB8101897C80F8291080F82AA0504C10
:1007E00094F8CD0194F8CC1104F2DF2588424ED064
:1007F00094F8CC0100EB800004EB8000007C405DAD
:10080000012894F8CC0100EB800004EB800004D0B8
:10081000007C405D022878D018E0807A01280DD055
:1008200094F8CC11022001EB810104EB8101097CD9
:10083000485594F8CC01162820D01BE094F8CC0140
:1008400000EB800004EB8000007C465594F8CC015E
:1008500000EB800004EB800294F8CC0100EB8000F8
:1008600004EB8000017C4846FEF7B7FF94F8CC010A
:10087000162803D094F8CC01401C00E0002084F836
:10088000CC0194F8CD0194F8CC118842B0D1254C1C
:10089000207D70B1207C415D012966D0405D022839
:1008A0006BD0207D28B1217C1E4A4846FEF795FF7B
:1008B0002675BBF10C0F06D00BEB8B0008EB80000C
:1008C000017C012961D0124C94F829000C2800F019
:1008D000388194F82A00002800F0428184F82A60C8
:1008E00094F8290000EB800008EB8003A4F53B702E
:1008F000D3E90112DB68C0F80433C0E9BF12607E9F
:1009000000280CBF042502250EE01CE07800002022
:10091000C00C0020D80B0020FFFF3F007A00002011
:10092000D4090020A40B002094F82900C34600EB52
:10093000800108EB8100407B06284DD2DFE800F003
:10094000404A4846444294F8CC0100EB800004EB56
:100950008000807A012818BFFFDF94F8CC0100EBFB
:10096000800004EB8000867268E7A17A01291DBF30
:10097000022141552675465593E7A07A012818BFF4
:10098000FFDFA672207C46558BE707210174FE4CE1
:10099000207E162810D0207EE17D401C884200D1A8
:1009A000FFDF207E04F800B0207E16280EBF002056
:1009B000207E401C207686E7E07D0028F1D1EFE71D
:1009C00000200BE0B42009E0732007E0322005E0AE
:1009D0000A2003E0062001E0FFDF00202073617E93
:1009E000022918BF012911D121690144A1EB090293
:1009F00022F07F42382A09D903206076A1F1320023
:100A000020F07F4020613220207309E0322807D295
:100A100094F8280058B9F8F793FA84F828A006E06B
:100A200094F8280018B1F8F7B4FA84F828607978B7
:100A300084F8201038780622012818BF032806D130
:100A400084F824A0207B814284BF081A821D94F878
:100A50002230002B18BF921C94F82400002808BFF5
:100A6000002B6AD0D4F810806069A8EB0908DFF881
:100A70001CC328F07F48A0EB090020F07F404245CE
:100A800098BFB8F5800F41D284453FD3207B884280
:100A900015D22369A1EB0002A3EB020222F07F42F0
:100AA0001144294421F07F412261616000280CBF7C
:100AB00001200320207710F0FF0F36D114E00AD96F
:100AC000226900291044284420F07F4060600CBF58
:100AD00002200420EEE7002B08BFFFDF2069284436
:100AE00020F07F40606026770120F8F787F800BF8C
:100AF00094F82900012300EB80010BEB8100616871
:100B000090F90C200020F8F7BDF829E084F8246063
:100B100084F82260207B0028E0D021690844284422
:100B200020F07F4060600220207720690123411976
:100B300000221846F8F7A6F8DAE7207B0028ECD167
:100B4000CCE70120F8F75AF80020F8F757F8F8F743
:100B50003BF894F8280018B1F8F71BFA84F82860DD
:100B600094F8220028B1F8F769F984F8236084F832
:100B7000226094F8210018B1F8787870B87838704D
:100B800094F8240030B184F823603878002808BF36
:100B900084F824607C48017EC07D814203D07C487B
:100BA0004078F8F70DFD84F827A0BDE8F09F70B5F8
:100BB000784C054682B094F829000C2808BFFFDF66
:100BC00094F8290000EB8000734E06EB8000007C57
:100BD000032818BFFFDFA068B0F1FF3F18BFFFDF99
:100BE00094F82900002100EB800006EB800001AAA8
:100BF00090F90C0000918DF8041028446946F8F72C
:100C000041F99DF904000F28CCBF01200020009974
:100C100008446168084420F07F41A16094F82500F1
:100C2000002804BF02B070BD012302B00022BDE85D
:100C300070401846F8F726B8584A0B1A02F1010C12
:100C4000B3EB9C0F3CBF1846704710B5441AB4EB89
:100C50009C0F3CBF184610BD9A4203D2101A08449C
:100C6000401C10BD94429EBFFFDF002010BD511AF2
:100C70000844401C404210BD0123002201460220CE
:100C8000F8F700B80220F7F7B9BFF8F75CB8F0B58D
:100C9000404C054683B094F82B00002808BFFFDFC6
:100CA000642D50D33E490020491B80414BD33D4821
:100CB00090F8CD1190F8CC01814244D13A48007DA2
:100CC000002840D194F82900334F00EB800007EB57
:100CD0008006206801AA28446946F8F7D3F89DF9F0
:100CE0000400002802DD0098401C0090B2680099C2
:100CF00073685018C01A20F07F40B0F5800F22D2E0
:100D0000B07C0C2809D000EB800007EB8000406825
:100D1000801A20F07F40884215D3A068B0F1FF3FD1
:100D200005D00120F7F76AFF4FF0FF30A060206880
:100D300028442060B0680099084420F07F4060613A
:100D400003B00120F0BD03B00020F0BD2DE9F0415B
:100D50000646401EC5B2104805EB850100EB810434
:100D6000207C002808BFFFDF0E4A92F8CC1192F8D1
:100D7000CD01814221D000BF01EB810302EB83034F
:100D80001B7CB34220D011E0BC0B0020FFFF3F00D2
:100D900078000020C00C0020D80B0020FF7F841EAC
:100DA000FF1FA107D4090020A40B002016290CBFA7
:100DB0000021491CC9B28142DED13A48017D002997
:100DC00062D0007CB0425FD10020BDE8F081217C80
:100DD00005291FBF217C0629217C07292CD12774D6
:100DE000C27D0023017E914218BF014624D000BF7E
:100DF00011F80280A84508BF012300D04BB1162A84
:100E00000CBF4FF0000802F1010811F8088001F84A
:100E10000280162A0CBF0022521CD2B291F8188010
:100E20009045E5D143B10A7E002A08BF81F818C079
:100E300002D00A7E521E0A76617C21B36674C27D9E
:100E40000021037E934224D0835CAB4208BF012182
:100E500000D029B1162A0CBF0023531CC35C835455
:100E6000162A0CBF0022521CD2B2037E9342EBD151
:100E700049B1027E0146002A08BF81F818C008D097
:100E80000A7E521E0A7604E00127074800264FF02A
:100E9000160C217C012904BF617C002997D1012017
:100EA000BDE8F081A40B0020BC0B0020F0B5734A14
:100EB000D2F80032724D002401212E7856B9714EBD
:100EC0003460704F03263F1D3E606E4F04260C3782
:100ED0003E602970C2F80042D1601160694C48340C
:100EE000D16425688542FBD35160D160C2F80032DD
:100EF000F0BD2DE9F041044680074FF000054FF0AA
:100F0000010604D560480560066024F00204E00490
:100F10004FF0FF3705D55D484660C0F8087324F4EC
:100F20008054600003D55A48056024F08044E005F1
:100F30000FD55248C0F80052C0F8087351490D60EF
:100F4000091D0D604F4A04210C321160066124F422
:100F50008074A00409D54F484660C0F80052C0F81C
:100F600008734D48056024F40054C4F38030C4F382
:100F7000C031884200D0FFDF14F4404F14D04748FE
:100F80004660C0F8087346488660C0F80052C0F852
:100F9000087344490D600A1D16608660C0F8087326
:100FA0000D60166024F4404420050AD53E48466092
:100FB0008660C0F80873C0F848733C48056024F4A4
:100FC000006409F0EDF93A48044200D0FFDFBDE8C3
:100FD000F08170B5202500224FEA020320FA02F1C9
:100FE000C90719D051B201F01F060124B4404E09BF
:100FF000B60006F1E026C6F88041C6F88042002916
:1010000006DA01F00F0101F1E02181F8143D03E05F
:1010100001F1E02181F80034521CAA42DED370BDF8
:1010200070B5174C0D466060FFF763FF6068FFF70F
:10103000D0FF2846F8F761F808F004FE00F0D5F874
:1010400009F0AEF909F0FBF8F8F78CFABDE870404A
:1010500008F09ABE10B50A4C6068FFF74AFF606856
:10106000FFF7B7FF09F09CF9F8F70CF90020606072
:1010700010BD034840687047022070470080004060
:101080008000002004850040FC1F004000C000409C
:1010900004E5014000D0004004D5004000E00040DD
:1010A00000F0004000F5004000B0004008B50040EE
:1010B000FEFF0FFC70B51F490A68BAB100231D4638
:1010C00001244A68521C4A60092A00D34D600E79F7
:1010D00004FA06F20E6816420AD072B60B68934301
:1010E0000B6062B649680160002070BD052070BDCC
:1010F0005B1C092BE5D3FFDFF8E74FF0E0214FF44D
:101100008000C1F800027047EFF3108111F0010F69
:1011100072B64FF0010202FA00F20648036842EA92
:101120000302026000D162B6E7E7024800210160D5
:1011300041607047880000200120810708607047E7
:10114000012081074860704712480068C00700D03E
:10115000012070470F48001F0068C00700D0012021
:1011600070470C4808300068C00700D00120704765
:10117000084810300068704706490C310A68D203ED
:1011800006D5096801F00301814201D101207047B1
:10119000002070470C040040C84911F8210F49781D
:1011A000884201D3401A02E0C1F121010844C0B2D3
:1011B0007047C249233111F8210F4978884201D381
:1011C000401A02E0C1F121010844C0B27047BB4996
:1011D000463111F8210F4978884201D3401A02E0C4
:1011E000C1F121010844C0B27047B54910B5802053
:1011F00081F80004B1490020233101F8210F487023
:10120000AE4901F8210F4870AC49463101F8210F71
:101210004870AC4808F05CFFAA48401C08F058FF32
:10122000F8F778F8BDE8104000F03DB9202070478D
:10123000B2E770B50C4605460026FFF7ADFF014644
:101240009E48A14212D30022641EE4B20DD390F84E
:101250002210435C491CC9B205F8013B80F82210FA
:101260002129F1D180F82220EEE7012600F01BF9B8
:10127000304670BD202070479BE770B50C46054690
:101280000026FFF796FF01468C482330A14212D377
:101290000022641EE4B20DD390F82210435C491C76
:1012A000C9B205F8013B80F822102129F1D180F85C
:1012B0002220EEE7012600F0F6F8304670BD20212E
:1012C00001700020704710B50446FFF780FF2070C2
:1012D000002010BD70B50C460546FFF778FF0146AB
:1012E00076484630A14213D30022641EE4B20DD3E7
:1012F00090F82210435C491CC9B205F8013B80F804
:1013000022102129F1D180F82220EEE7002401E00B
:1013100042F2070400F0C7F8204670BD70B50C46D5
:101320000546212900D9FFDF67480068103840B220
:1013300000F0A0F8C6B20D2000F09CF8C0B28642C2
:1013400004D2FFDF02E000BFF8F734F82146284658
:10135000FFF76FFF0028F7D070BD2DE9F047DFF8E9
:101360006481564CA8F101080746233498F8000020
:10137000DFF84891002604F1230A38B994F82210C6
:1013800094F82100212200F084F890B14D4699F89C
:10139000221099F82100212200F07BF8B8B15546BF
:1013A0009AF822109AF82100212200F072F848B32E
:1013B00035E094F82100275494F82100401CC0B275
:1013C00084F8210021282AD184F8216027E095F8AB
:1013D00021002F5495F82100401CC0B285F821004F
:1013E000212801D185F8216098F800004746B0B166
:1013F00095F8221095F82100212200F04AF870B1EA
:101400003E700CE095F821002F5495F82100401C07
:10141000C0B285F82100212801D185F8216094F817
:10142000221094F82100212200F033F800281FD068
:1014300099F8221099F82100212200F02AF80028BA
:1014400016D09AF822109AF82100212200F021F8F3
:1014500000280DD0F7F784FF1A4808F041FEB0F5D8
:10146000005F00D0FFDFBDE8F047164808F04EBE31
:10147000BDE8F087002806DA00F00F0000F1E02058
:1014800090F8140D03E000F1E02090F8000440090A
:101490007047401C884204D0904200D109B100201E
:1014A00070470120704710B5064808F019FE002863
:1014B00003D1BDE81040F7F73EBF10BDF00C00208F
:1014C0000DE000E09100002004ED00E013490878F1
:1014D0004A78401CC0B2904205D0114B01221A60DC
:1014E000BFF34F8F0870704770B54FF0E0250B4C7D
:1014F000F7F7E6FF20BF40BF20BF6078217861701A
:10150000D5F8001229B9D5F8041211B92178814211
:10151000EED0F7F7D0FF002070BD00009300002050
:10152000180502402DE9F041012528034FF0E02184
:101530000026C1F880011E4CC4F800610C2000F0A8
:101540002CF81C4801680268C94341F3001142F0BD
:1015500010020260C4F804532560491C00E020BF5B
:10156000D4F80021002AFAD019B9016821F010013D
:101570000160114807686560C4F80853C4F8006149
:101580000C2000F00AF83846BDE8F08110B504469A
:10159000FFF7C8FF2060002010BD00F01F020121EE
:1015A00091404009800000F1E020C0F880127047AF
:1015B00000C0004010ED00E008C500402DE9F047F4
:1015C000F84C0646FF21606800EB06121170217886
:1015D000FF2916D04FF0080909EB011109EB061796
:1015E0004158C059491E21F07F4100F0DDF918B182
:1015F00094F80080454614E06168207801EB0611FC
:1016000008702670BDE8F087626809EB0510D159B3
:10161000105800F0C9F930B96068A84600EB08100E
:101620000578FF2DF0D1606800EB061100EB081083
:101630000D700670E6E7F0B5DA4B04460020012590
:101640005A680C261B7A0BE005EB0017D75DA74202
:1016500004D106EB0017D7598F4204D0401CC0B20A
:101660008342F1D8FF20F0BD70B5FFF70EFBCD4CE3
:10167000014608252278606805EB0212805800F0C8
:1016800093F9012808D92178606805EB01114058C9
:10169000BDE87040FFF7F0BAFEF73CFFBDE87040D0
:1016A000F7F78EBF2DE9F041BE4C2578FFF7EDFA34
:1016B0000146FF2D6FD04FF00808626808EB051651
:1016C000905900F071F90228606801D980595EE0F4
:1016D00000EB051109782170022101EB0511425C34
:1016E0005AB1521E4254815901F5000121F07F4147
:1016F00081512846FFF762FF34E00423012203EB07
:10170000051302EB051250F803C0875CBCF1000F13
:1017100010D0BCF5806F10D9CCF3090250F806C088
:101720000CEB423C2CF07F4C40F806C0C3589A1A90
:10173000920A09E0FF2181540AE0825902EB4C32FF
:1017400022F07F428251002242542846FFF736FFA2
:101750000C21606801EB05114158E06850F8272022
:10176000384690472078FF2815D0FFF78EFA0146BB
:101770002278606808EB02124546805800F014F9A0
:10178000012891D92178606805EB01114058BDE826
:10179000F041FFF771BABDE8F081F0B51D4614467F
:1017A0000E460746FF2B00D3FFDFA00700D0FFDF68
:1017B0007C48FF210022C7604460057206740170F6
:1017C00042701046012204E002EB0013401CE15479
:1017D000C0B2A842F8D3F0BD70B5724C0646657829
:1017E000207C854200D3FFDFE06840F82560607808
:1017F000401C6070284670BD2DE9FF5F1D468B467A
:101800000746FF24FFF741FADFF89891064699F85A
:101810000100B84200D8FFDF00214FF001084FF06F
:101820000C0A99F80820D9F804000EE008EB01131F
:10183000C35CFF2B27D0BB4205D10AEB011350F844
:1018400003C0DC4521D0491CC9B28A42EED8FF2C26
:101850001BD008EB04110AEB0412475440F802B005
:101860000421029B0022012B01EB041111D04250F4
:101870004FF4806808234FF0020C454519D9A9059B
:10188000890D08D008E00C46DDE7FF2004B0BDE874
:10189000F09F4550ECE7414606EB413203EB041361
:1018A00022F07F42C250691A0CEB0412890A81545B
:1018B0000BE005B9012506EB453103EB041321F0DC
:1018C0007F41C1500CEB0411425499F8005020465E
:1018D000FFF774FE99F80000A84201D0FFF7C4FE9C
:1018E0003846D3E770B50C460546FFF7CEF90646F5
:1018F00021462846FFF79FFE0446FF2817D0294DB2
:10190000082101EB041168684058314600F04CF89A
:1019100000F58050400B02216A6801EB0411515C14
:1019200009B100EB8120002800D1012070BD00200A
:1019300070BD2DE9F0410F468046FFF77CFEFF2881
:101940001BD0184E357871682A462C4605E0844233
:1019500006D0254601EB05131C78FF2CF7D10CE0CF
:10196000FF2C0AD0A5420CD101EB02100078307098
:10197000FF2804D0FFF778FE03E000200BE7FFF715
:1019800081F939464046FFF7ADFFFF220123716818
:1019900003EB0413CA5401EB041201EB0511127896
:1019A0000A70F8E65C0D0020401A20F07F40B0F588
:1019B000000F00D90020704770B50446A0F5000064
:1019C0002C4EB0F1786F02D23444A4F500042A48BA
:1019D000844201D2012500E0002500F041F830B139
:1019E000B4420BD32548006804E0284370BDB442DC
:1019F00004D32348844201D20120F6E70020F4E713
:101A000010B50446A0F50000B0F1786F03D2194874
:101A10000444A4F5000400F023F84FF0804130B1F5
:101A20001648006804E08C4204D2012003E0144808
:101A30008442F8D2002080F0010010BD10B520B122
:101A4000FFF7DEFF08B1012010BD002010BD10B56A
:101A500020B1FFF7B1FF08B1012010BD002010BD7B
:101A6000084809490068884201D1012070470020D8
:101A7000704700000000002000C001001C00002092
:101A80000800002098000020BEBAFECA0548064A99
:101A90000168914201D100210160044901200860E0
:101AA0007047000098000020BEBAFECA40E5014021
:101AB000404800210170417010218170704770B55D
:101AC000054616460C460220F5F789FC39490120E7
:101AD00008703949F01E086038480560001F04602E
:101AE00070BD10B50220F5F77AFC3249012008706C
:101AF00033480021C0F80011C0F80411C0F80811E3
:101B000030494FF40000086010BD2A480178C9B17F
:101B10002D4A4FF4000111602949D1F8003100220B
:101B2000002B1CBFD1F80431002B02D0D1F80811D2
:101B300011B14270102103E001214170234909686D
:101B4000817002700020F5F74ABC1A48017800291C
:101B500004BF407870471A48D0F80011002904BF2C
:101B600002207047D0F8001100291CBFD0F80411E2
:101B7000002905D0D0F80801002804BF01207047D3
:101B8000002070470B480178002904BF8078704717
:101B90000B48D0F8001100291CBFD0F8041100290F
:101BA00002D0D0F8080108B110207047074800683B
:101BB000C0B270479C00002010F5004008F50040BE
:101BC00000F0004004F5014008F5014000F4004039
:101BD0003148002101704170704770B506461446C7
:101BE0000D460120F5F7FBFB2B49012008702B481F
:101BF0000660001D0460001D056070BD2DE9F04108
:101C000004460120F5F7EBFB234901200870244925
:101C10000C60244D0026C5F8046123494FF040773D
:101C20000F60A1F1040844B1012C18BFFFDFC5F813
:101C30000062C8F80070BDE8F081C5F800024FF0FE
:101C40008070C8F80000BDE8F0811348017879B1D0
:101C5000154A4FF0407111601249D1F8042100215A
:101C6000002A08BF417002D0104A12684270017009
:101C70000020F5F7B4BB08480178002904BF40787C
:101C800070470848D0F80401002808BF704707488B
:101C90000068C0B2704700009F00002008F50040B7
:101CA00004F5004000F0004008F5014000F4004059
:101CB00070B5FE4C002501266570257025626572A1
:101CC000A572E67284F82950256304F13C00A563EF
:101CD00008F0FEF9002818BFFFDF84F82450F4480C
:101CE00009F062FAF3480660657770BD30B4EF49D9
:101CF0000268DFF8C8C34A6142688A61007A0877DF
:101D00000A7DED4BACF1040401204AB10A7E00FAD1
:101D100002F21A608D7D002D0CBF2260CCF80020ED
:101D20004A7D002A04BF30BC70474A7E904018604C
:101D3000C97D00290CBF2060CCF8000030BC704782
:101D4000DF4900B50A1D40B101281CBFFFDF00BDFF
:101D5000DC480860DC48106000BDDC480860DC48F6
:101D6000F9E7F0B502264FF0E02701240025C7F877
:101D70008061D8490D600C60D7490A6822F077026B
:101D800042F0880242F000420A60CD490A1DD0B1FB
:101D9000012818BFFFDF1AD0D04940F25B6008600D
:101DA000091F40F203100860081F0460CC4903209B
:101DB0000860CC4996200860BC4C94F9240010F0CF
:101DC000030F09D033E0C1480860C14802E0BD48B4
:101DD0000860BD481060DFE780100A300C2826D26A
:101DE000DFE800F021252525251D1915110D0A060E
:101DF000BD49042008601BE0BB48056018E0BA49F3
:101E0000FC20086014E0B849F820086010E0B649EA
:101E1000F42008600CE0B449F020086008E0B24902
:101E2000EC20086004E0B049D820086000E0FFDF43
:101E3000607F002814BF4FF4C020AC48AC49086054
:101E4000AD49AC480860091FAC480860C7F880621B
:101E5000AB491020C1F80403F0BD944A0368C2F8EE
:101E600002308088D08011727047904890F8290025
:101E700070478E4A517010707047F0B50D46044699
:101E800004EB4501908808841078D2F801100127EE
:101E900040EA012044F8250005F1080007FA00F6A1
:101EA000002B04BF206BB04304D0012B18BFFFDF11
:101EB000206B304307FA05F108432063F0BD30B5CD
:101EC0000D460446082988BFFFDF0022002D11D9E6
:101ED00054F82210900000F1804000F58050C0F8C6
:101EE000001604EB4201098CC0F82016501CC2B247
:101EF0009542EDD8206B8349086030BD10B504468B
:101F000010F0030F2BD1A0100A300C2827D2DFE8E5
:101F100000F022262626261E1A16120E0A067249DE
:101F2000042008601CE070490020086018E06E4939
:101F3000FC20086014E06C49F820086010E06A4951
:101F4000F42008600CE06849F020086008E0664969
:101F5000EC20086004E06449D820086000E0FFDF5E
:101F6000524880F8244010BD504890F83400704723
:101F7000654AC178116000686449000208607047D2
:101F8000252808BF02210ED0262808BF1A210AD012
:101F9000272808BF502106D00A2894BF0422062211
:101FA00002EB4001C9B25A4A11605A4908607047B1
:101FB0003E49086270473D498A7A012A49D0022A7F
:101FC00018BF70474B7D002B08BF7047DFF848C132
:101FD000012A42D0CA7D4B7E002A18BF01227D30E3
:101FE000CCF80000DFF834C10020CCF84C01180216
:101FF00082F0010240EA025040F00312087F8300A1
:1020000003F1804303F5C043C3F81025444A02EBB3
:102010008002887EC30003F1804303F5F833C3F8E0
:102020001425DFF800C1C3F810C5C97ECB0003F149
:10203000804303F5F833C3F81425304AC3F810255C
:10204000012202FA00F002FA01F108433649086061
:1020500070470B7D002BB9D170478A7D0B7E002A1B
:1020600018BF01227E30BBE72DE9F84F00280CBFD6
:10207000012002200D4C224D0322A072C5F800223F
:10208000627F002A14BF4FF4C022184A264F3A60DC
:102090004FF00108002976D0012973D002291CBF16
:1020A000FFDFBDE8F88F206A00283FE0700D0020B8
:1020B000840D0020A0050040180500500C050050BC
:1020C00014150040050103001F0003020601020071
:1020D00025000302FC1F00403C170040381500405B
:1020E00010150040441500400C1500400000040489
:1020F00008F5014040800040A4F501401011004067
:102100000010004040160040241500401C150040FF
:1021100008150040541500404C85004000800040E8
:10212000006000404C81004004F5014008BFFFDF23
:10213000216A206B0844FB490860FC49FA480860A2
:10214000A17AFB4801290EBF0560FA490160A06B26
:1021500040F40020A063D5F800924FF0100AC5F8B3
:1021600008A30026C5F80062F3484FF4802BC0F89E
:1021700000B0FF208DF80000C5F81061C5F8108090
:102180003DE000E01CE0012813D0C5F804800228DF
:1021900018BFBDE8F88F607D002808BFBDE8F88F44
:1021A000E648C0F84C80E6480068BDE8F84F0A30C1
:1021B00001E7C5F80080207D0028F1D1BDE8F88F47
:1021C000E0490128896B07D0022818BFFFDF09D03A
:1021D000BDE8F84F0A20EEE641F48010A0634FF40A
:1021E000801004E041F40010A0634FF40010386048
:1021F000EEE700BF9DF80000401E8DF800009DF83E
:10220000000018B1D5F810010028F3D09DF80000A7
:10221000002808BFFFDFC5F80C61C5F81061C5F8DC
:102220000461C5F81461C5F81861C5F82861C6488D
:1022300000680090C5F80092C7F800B0C5F804A384
:102240004FF400203860216A206BBDE8F84F084445
:102250000A30B0E62DE9F847BC4CD4F8000220F073
:102260000309D4F804034FF0100AC0F30018C4F8AF
:1022700008A30026C4F80062B24D687F002814BF8E
:102280004FF4C020B248AC490860A87A0127012861
:1022900002D0022803D014E0287D10B911E0687D37
